:020000040800F2
:1000000088EE0024A504000841A000082D8F0008F8
:10001000759D0008151F00085DC90008000000005C
:10002000000000000000000000000000B103000814
:1000300063310008000000000D04000885B20008CC
:10004000C3040008C3040008C3040008C304000874
:10005000C3040008C3040008C3040008C304000864
:10006000C3040008C3040008C3040008D12A000820
:10007000DD2A0008C3040008C3040008C304000804
:10008000C3040008C3040008C3040008A531000825
:10009000BD310008B1310008C9310008C3040008AF
:1000A000C3040008C3040008C3040008C304000814
:1000B0000DB40008C3040008C3040008C30400080A
:1000C000C3040008C3040008C3040008C3040008F4
:1000D000F5A40008C3040008C3040008C304000812
:1000E00065310008C304000800000000C3040008D4
:1000F000C3040008C3040008C3040008C3040008C4
:10010000C3040008C3040008C3040008C3040008B3
:10011000C3040008E9C00008C3040008C3040008C1
:10012000C3040008C3040008C3040008C304000893
:10013000C3040008C3040008C3040008C304000883
:1001400000000000000000000000000000000000AF
:10015000E92A0008C3040008C3040008C304000817
:10016000C3040008C3040008C3040008C304000853
:10017000C3040008C3040008C30400080000000012
:10018000C3040008C3040008C3040008C304000833
:10019000C3040008C3040008C3040008C304000823
:1001A000C3040008C3040008C304000800000000E2
:1001B000C3040008C3040008C3040008C304000803
:1001C000C3040008C3040008000000000000000091
:1001D0000000000000000000C30400080000000050
:1001E000000000000000000000000000000000000F
:1001F0000000000000000000C3040008C304000861
:10020000C3040008C304000800000000C304000881
:10021000C3040008C3040008C3040008C3040008A2
:10022000C304000800000000C30400080000000030
:10023000C3040008C304000800000000C304000851
:10024000C3040008C3040008C3040008C304000872
:10025000C3040008C3040008C3040008C304000862
:10026000C3040008C3040008C3040008C304000852
:10027000C3040008C3040008C30400080000000011
:10028000C3040008C3040008C3040008C304000832
:1002900000000000C3040008C304000800000000C0
:1002A00000000000C3040008C3040008C3040008E1
:1002B000C3040008C3040008C3040008D5310008C3
:1002C000E1310008C3040008C304000800F002F88C
:1002D00000F05EF80AA090E8000C82448344AAF182
:1002E0000107DA4501D100F053F8AFF2090EBAE880
:1002F0000F0013F0010F18BFFB1A43F0010318475A
:1003000020010100400101000A444FF0000C10F8E8
:10031000013B13F0070408BF10F8014B1D1108BF83
:1003200010F8015B641E05D010F8016B641E01F823
:10033000016BF9D113F0080F1EBF10F8014BAD1C73
:100340000C1B09D16D1E58BF01F801CBFAD505E091
:1003500014F8016B01F8016B6D1EF9D59142D6D3EB
:10036000704700000023002400250026103A28BF13
:1003700078C1FBD8520728BF30C148BF0B60704717
:100380001FB50FF010FE00F03EF91FBD10B510BDF7
:1003900000F021FA1146FFF7F3FF0DF0C3FA00F069
:1003A0003FFA03B4FFF7F2FF03BC00F043FA00008A
:1003B0002C4B19680868B0E8F04F80F30988BFF348
:1003C0006F8F4FF0000080F311887047000000002D
:1003D00008480068006880F308884FF0000080F348
:1003E000148862B661B6BFF34F8FBFF36F8F00DF23
:1003F00000BF00BF08ED00E0DFF80C00016841F429
:1004000070010160704700BF88ED00E0EFF30980E4
:10041000BFF36F8F134B1A681EF0100F08BF20ED4B
:10042000108A20E9F04F106009B44FF0500080F3BB
:100430001188BFF34F8FBFF36F8F0EF0CFFC4FF0DB
:10044000000080F3118809BC19680868B0E8F04F13
:100450001EF0100F08BFB0EC108A80F30988BFF3BC
:100460006F8F70471C000024EFF305807047000079
:100470000B49D1F800C04A685CF8043B1068184486
:1004800042F8040B8C4528BFA1F1DC0C8A4228BF3E
:10049000A1F1DC02C1F800C04A6020F000407047C2
:1004A0001CCE00240A4880470A4880470A48004773
:1004B000FEE7FEE7FEE7FEE7FEE7FEE7FEE7FEE714
:1004C000FEE7FEE705480649064A074B704700006D
:1004D0008931000835B30008CD02000888CE002419
:1004E00088EE002488DE002488DE002453EA020C13
:1004F00000F069802DE9F04B4FF00006002B1FBF84
:10050000B3FA83F503FA05F424FA05F65E4012BF48
:100510001643B2FA82F502FA05F4C5F120051EBFB2
:1005200022FA05FC44EA0C04203556EA044C4FEA52
:10053000144418BF641C4FF000084FF000099042AB
:1005400071EB030C39D3002919BFB1FA81F701FA15
:1005500007F6B0FA80F700FA07F6C7F120071EBFCA
:1005600020FA07FC46EA0C062037B6FBF4FCA7EBA2
:100570000507103F07F01F0BCBF120060CFA0BFB11
:100580002CFA06F644BFB3460026202FA4BF5E46D1
:100590004FF0000B5BEA060C08BF4FF0010B19EBA4
:1005A0000B09ABFB027C48EB0608C01B06FB02CC28
:1005B0000BFB03CC71EB0C01C1E70B460246414635
:1005C0004846BDE8F08B13B54FF000004FF0000136
:1005D000AFF30080BDE81C40704700000B4910B528
:1005E000A1F17C020A4CC2E93712372106E000EB88
:1005F000104342F82130074B00FB03400B1EA1F1D2
:100600000101F4DC10BD0120E8E70000BCCD0024AE
:10061000E119D666CD0D0100032A40F2308010F0BA
:10062000030C00F0158011F8013BBCF1020F62448D
:1006300098BF11F801CB00F8013B38BF11F8013B1E
:10064000A2F1040298BF00F801CB38BF00F8013BCB
:1006500011F0030300F02580083AC0F0088051F83B
:10066000043B083A51F804CBA0E80810F5E7121D46
:100670005CBF51F8043B40F8043BAFF30080D20765
:1006800024BF11F8013B11F801CB48BF11F8012B31
:1006900024BF00F8013B00F801CB48BF00F8012B54
:1006A000704710B5203AC0F00B80B1E81850203ADE
:1006B000A0E81850B1E81850A0E81850BFF4F5AF02
:1006C0005FEA027C24BFB1E81850A0E8185044BF8C
:1006D00018C918C0BDE810405FEA827C24BF51F8F9
:1006E000043B40F8043B08BF7047D20728BF31F8ED
:1006F000023B48BF11F8012B28BF20F8023B48BF3E
:1007000000F8012B704702F0FF0343EA032242EA9C
:10071000024200F002B84FF000020429C0F012803B
:1007200010F0030C00F01B80CCF1040CBCF1020FA4
:1007300018BF00F8012BA8BF20F8022BA1EB0C0179
:1007400000F00DB85FEAC17C24BF00F8012B00F86F
:10075000012B48BF00F8012B70474FF0000200B595
:10076000134694469646203922BFA0E80C50A0E8D4
:100770000C50B1F12001BFF4F7AF090728BFA0E882
:100780000C5048BF0CC05DF804EB890028BF40F84E
:10079000042B08BF704748BF20F8022B11F0804F90
:1007A00018BF00F8012B704770477047704710B5AD
:1007B00000F00CF8006810BD10B5044600F006F813
:1007C000046010BD0048704724CE002400487047E4
:1007D00024CE002470477546FFF7F4FFAE460500AF
:1007E0006946534620F00700854618B020B5FFF74C
:1007F00069FEBDE820404FF000064FF000074FF0C3
:1008000000084FF0000B21F00701AC46ACE8C0092E
:10081000ACE8C009ACE8C009ACE8C0098D46704737
:1008200010B50446AFF300802046BDE81040FFF746
:10083000B8BD000001491820ABBEFEE7260002004B
:1008400070B505000C464FF0FF302DED028B5AD0ED
:10085000002C58D0D4ED010AD4ED001A94ED020A10
:1008600020EEA01A61EEA01A94ED032AF7EE008A9A
:1008700000EE001A40EE021AB0EE008AF0EE680AAE
:1008800041EE480A21EE880A0CF02EFB85ED010AA4
:1008900094ED000AD4ED021AD4ED030A94ED011A86
:1008A00020EE210A00EEC10A20EE080AF0EEC00A8E
:1008B00010EE900AB0F17E5F06DB10EE101A1348BE
:1008C00060F31E01A96003E00CF08CF885ED020ACC
:1008D00094ED021AD4ED001A94ED030A21EE012AD8
:1008E000D4ED012A61EE801AF0EE680A00EE002ACB
:1008F00042EE811A42EE480A21EE880A0CF0F4FA20
:10090000002085ED000ABDEC028B70BDDB0FC93FF6
:1009100070B504000D463ED0B7EE001ADFED380A80
:10092000C1EE001A84ED001AC4ED010AC4ED020AFA
:10093000C4ED030AC4ED041A65B3D5ED000A95EDC4
:10094000010AB7EEE01AB7EEC00A0CF0E9F9B7EE0B
:10095000C00BD5ED002ADFED2B0A9FED2B1ADFED42
:100960002B1A9FED2B2AF5EEC02AB1EE400AF1EECC
:1009700010FA13D1D5ED012AF5EEC02AF1EE10FAE6
:100980000CD1D5ED022AF5EEC02AF1EE10FA05D110
:10099000C4EC040A32E04FF0FF3070BD10EE101AC4
:1009A0001C48814204DBB5EEC00AF1EE10FA0ADD04
:1009B0009FED190ADFED190A9FED191ADFED191ADB
:1009C00084EC040A1AE010EE102A17498A42DFDB91
:1009D00010EE102A8242DBDC10EE102A134882420D
:1009E000D6DB10EE102A8A42D2DC10EE101A8142B9
:1009F000CEDBB5EEC00AF1EE10FAC9DC002070BD06
:100A000000000000C5064D3F2D4A0D3C56A439BBE1
:100A1000AD47193FDB0FC93F6E597F3F0C53B039CB
:100A2000AB88BBBB8595973DDB0F49400000B442C6
:100A300000210160416081607047000030B5040012
:100A40004FF0FF302DED108BA1B07CD000297AD073
:100A5000002A78D09FEDFE0AFE4D85ED000AA3B175
:100A6000D3ED009AD3ED018A93ED029AF5EEC09A88
:100A7000F1EE10FA11D1F5EEC08AF1EE10FA0CD1B8
:100A8000B5EEC09AF1EE10FA07D121B02046BDECC8
:100A9000108BBDE8304000F011BA94ED000A92EDE1
:100AA000001AD2ED010AD2ED021A94ED013AD1ED0D
:100AB00000AA20EE014A60EE203A60EE214A23EEC1
:100AC000415AD4ED022A94ED032A91ED01AA91ED49
:100AD000028AF5EEC0AAB6EE000AF1EE10FA02EEB6
:100AE000E05A02EEA14A43EE613A43EE204A02EE9A
:100AF000615A02EE604A42EE013A42EEC14A25EEE8
:100B000000FA64EE00EA23EE80EA64EE80DA09D1AE
:100B1000B5EEC0AAF1EE10FA04D1B5EEC08AF1EE3E
:100B200010FA7CD02AEEAA0A0AEE0A0A08EE080A8F
:100B300008F0FEF96AEE801ACDED0B1A6AEE001A83
:100B4000CDED0A1A00E0B4E168EE001A29EEA90A18
:100B5000CDED091A08EEA80A09EE090A08F0E8F92D
:100B6000D4EC021AB0EE008AD4ED030A69EE80AA32
:100B700094ED021A61EEA12A20EE883A21EE88BA9D
:100B800062EE08BAF0EE629A61EE822A8DED163AB4
:100B900021EE08AACDED122A61EE812A61EEA01A9B
:100BA00068EE808ACDED192A62EE012ACDED1D1A7C
:100BB00029EE009ACDED1C2A6BEE2A2A2BEEAA7A9A
:100BC0002AEE200ACDED112A8DED1A7A60EEA21AD6
:100BD0008DED1B0A6BEE282A2AEEA90A48EEA91A07
:100BE000CDED182A62EE02CA02EEE00A6BEE092A87
:100BF00062EE20FA21EE01CA20EEA0DA42EEC21A1D
:100C000002EE810A2BEEA82A47EE011A0AEEAC0A80
:100C100048EEEC1A02EE010A48EE8C1A00E005E1FB
:100C20002BEE892A2BEE013A02EE200A2AEE092A3F
:100C300042EE201A0AEECC0A61EE200ACDED000A3F
:100C400048EECD1A0AEECD0A8DED043A20EE000AE8
:100C500001EEA10A08F06CF9DDED1C2ADDED1D1A8C
:100C6000DDED000AB7EE002A32EEE11ADDED122AC0
:100C70009DED043ADDED0A1A72EEA04AC2EE000ABA
:100C80009DED1B0A1FEE883A0CEEC82A02EE880A78
:100C90006AEE285A0CEE482A70EE612ADDED0B1A36
:100CA00073EE611AB6EE003A22EEAB0A73EE4C3ADE
:100CB00033EE6C3A61EEABBA0AEE610A21EE201A0D
:100CC00033EE4C6A9DED163A4AEE22BA73EECD3AF7
:100CD00022EE837A21EE83AA94ED013A63EEA03AE4
:100CE0000BEE617A0BEE22AADDED091ADDED192A71
:100CF000B1EE00BA72EE617A72EEAF1A7FEEE26A7E
:100D000023EE0B2ADDED182A21EEA04A20EE885AA8
:100D100063EE221A02EE67AA94ED022ADDED112A93
:100D200042EEC21A62EE0B2A49EE291AF0EE479AF9
:100D30009DED1A7A42EEE79AD4ED032A65EE427AE7
:100D400047EE221A94ED007A49EE6C1A45EEA21A8B
:100D500062EE205AB0EE65BA49EE4C1A49EE0D1A11
:100D600001EEA41A63EE214A41EEA63A01EE87BADB
:100D700001EE864AB0EE64CA62EE216A05EE62CAEE
:100D8000B0EE645A73EEEA3A22EEA16A00EEE25A3D
:100D900041EEC77A06EEE30A06EE23AA31EE686A50
:100DA00063EE204A21EE881A40EEC76AF0EE40AAB0
:100DB00022EEA08A45EE06AA27EE207A74EE490AB2
:100DC000B0EE640A47EEA39A01EEA20A0BEE06AA61
:100DD00001EE438A45EEA0AA4CEE23BA01EE427A18
:100DE00040EE069A08EE20AA2AEEAA0A46EE86BA35
:100DF00047EE209A0AEE0A0A44EEA0BA09EEA90AC2
:100E00000BEEAB0A08F094F86AEE800A2AEE001A9C
:100E100069EE801A2BEE802A95ED000A00EE60FA4A
:100E200040EE41EA00EE61EA40EE42DA94ED040A57
:100E300094ED002A94ED011AD4ED020A0FEE002A77
:100E40000EEE801A4EEE000AD4ED031A04E0000004
:100E50009EEF273DD40000244DEE801A22EE020AB8
:100E600084ED002A84ED011AC4ED020A01EE010AA4
:100E7000C4ED031A00EEA00A01EEA10A08F058F82A
:100E800094ED001A94ED012AD4ED021AD4ED030A70
:100E900021EE001A22EE002A61EE801A20EE800A6E
:100EA00084ED001A84ED012AC4ED021A002084EDBD
:100EB000030A21B0BDEC108B30BD000070B50400FA
:100EC0004FF0FF302DED0C8B7ED000297CD0002A16
:100ED0007AD09FED860A864DF6EE001A85ED000A5F
:100EE000D2ED000A92ED010A92ED021A91ED00BADC
:100EF00094ED022AD4ED032AD1ED018A91ED028A04
:100F0000B5EEC0BA94EC023A23EE204A63EE004AF2
:100F100023EE013A23EEE05AF1EE10FA02EE405AC7
:100F200002EE014A43EEC14A03EE803A02EEC15A94
:100F300002EEC04A42EEA04A02EE603A65EE21AAF5
:100F400024EE21AA64EEA19A23EE219A09D1F5EEAE
:100F5000C08AF1EE10FA04D1B5EEC08AF1EE10FAB3
:100F60007ED02BEE0B0A08EEA80A08EE080A07F05E
:100F7000DFFF94ED004AF1EE000AD4ED011AF0EE25
:100F8000003A94ED022A94ED033A2BEE001AB2EEE9
:100F9000005A68EE802A68EE004A24EE047A24EEB5
:100FA00023BA64EE20CA21EEA00A63EE035A23EEB0
:100FB000236A62EE206A22EE024A61EEA17A62EEB4
:100FC00023BA21EE85CA00E08DE021EEA3DA62EEBD
:100FD000053A27EE205A20EE257A27EEA08A64EE05
:100FE00020DA65EE020A06EE417A28EE038A6CEEFC
:100FF000848A4BEE010A0DEE418A05EE217A4BEE12
:10100000818A46EEA50A0DEE838A0BEE627A4CEEDB
:10101000A78A46EE620A0BEEE28A37EE40BA4DEE40
:10102000628A70EEE6BA0CEE27BA43EEA7BA0CEE6F
:1010300004BA43EE84BA00EE24BA28EEA80A46EEBB
:10104000A4BA0BEE0B0A0BEEAB0A08EE080A07F087
:101050006FFF28EE801A6BEE000A6BEE801A00E03C
:101060000BE028EE002A95ED000A40EE41AA00EEC2
:1010700060AA40EE619A00EE429A201D94ED002A8B
:1010800094ED040AD0EC030A0AEE802A4AEE000A24
:1010900009EE801A49EE001A22EE020A84ED002AB7
:1010A00000EEA00AC0EC030A01EE010A01EEA10A5B
:1010B00007F03EFF94ED001A94ED012AD4ED021AD8
:1010C000D4ED030A21EE001A22EE002A61EE801A06
:1010D00020EE800A84ED001A84ED012AC4ED021A84
:1010E000002084ED030ABDEC0C8B70BD022B073D84
:1010F000D4000024B1EE601AB4EEC10AF1EE10FA89
:1011000002D2B0EE410A7047B4EEE00AF1EE10FAF6
:10111000F9DDB0EE600A70470248082140680CF023
:10112000E5BD0000AC000024044A13231221002076
:1011300010B500F08DF9002010BD00008CBD00241A
:1011400001214FF0FF3202200CF00ABE9FED010A90
:10115000704700000000C8430248102140680CF0AE
:10116000C5BD0000AC000024044A06230221012072
:1011700010B500F06DF9002010BD000093BD0024F3
:1011800001214FF0FF3204200CF0EABD2DE9F041BF
:1011900006000D466FF0010726D02DB3424C207893
:1011A00018B16FF00200BDE8F0810CF025FE606020
:1011B000D0B1B622F5627E21002000F09FF9B62260
:1011C0001421012000F09AF91E2000F028FE1E21B3
:1011D000002000F061F90021084600F05DF91E28AA
:1011E0006FF0030508D101E03846DCE7002101205B
:1011F00000F052F90F2801D02846D4E7062000F06D
:101200004FFD072000F04CFD284A0121002000F08E
:10121000E3FD2749062000F071FD2649072000F074
:101220006DFDAA224021002000F068F90122412131
:10123000002000F063F908225321002000F05EF93D
:1012400004225821002000F059F904227D210020B9
:1012500000F054F9322000F0E2FD01220F21104687
:1012600000F04CF903221021012000F047F9002280
:101270001621012000F042F901221821104600F049
:101280003DF980221521012000F038F90A2000F0F4
:10129000C6FD01202070062000F010FD072000F0A0
:1012A0000DFD00207FE70000AC00002405140008BD
:1012B00019110008591100081EB5E8B324499FED23
:1012C000250AB1F80120ADF80020B1F80320ADF8EF
:1012D0000420B1F80520ADF80820BDF90020BDF9C3
:1012E000043001EE902A01EE103ABDF90840F8EE04
:1012F000E11AB8EEC11A00EE904A81EE802AF8EEAB
:10130000E00AC1EE001A80ED042A80EE801AC0EDDA
:10131000051A80ED061A4A7C897CD20042EA5111F6
:10132000B1F5806F01DBA1F5006100EE101AB4EE9B
:10133000001AF3EE070A00E007E0B8EEC00A40EE3C
:10134000010AC0ED0A0A00201EBD6FF001001EBD9B
:101350008CBD002400A0AA451EB56FF00102E8B3C1
:101360002549DFED260A9FED260AB1F80730ADF8D2
:101370000030B1F80930ADF80430B1F80B101BB2F1
:10138000ADF80810BDF9001001EE903A02EE101A07
:10139000BDF90840F8EEE11AF8EEC22A01EE104A53
:1013A00082EEA02AB8EEC11AC1EEA02AC1EE201A20
:1013B00062EE000A22EE801AC0ED070A80ED081ADC
:1013C00021EE800A80ED090AC16AD1ED001A70EEA3
:1013D000E10AC0ED070AD1ED010A00E009E071EE73
:1013E000600AC0ED080AD1ED020A30EE600A80ED15
:1013F000090A10461EBD00008CBD00246F12034276
:1014000035FA8E3C012010B500F066FC0C4C38B962
:101410000121084600F094FC606802210CF066FC93
:10142000052000F059FC002809D10121052000F019
:1014300087FC60680421BDE810400CF057BC10BD6B
:10144000AC00002401214FF0FF3218200CF088BCC2
:1014500070B514001E460D461BD010B1012807D1EF
:1014600002E00021012001E00021052000F068FCDD
:101470000849002345F0800001220870184600F05A
:10148000B9FC32462146BDE870400123002000F03F
:101490008DBC70BDAD00002470B50D460446012022
:1014A00000F0BDFC14B1012C07D102E000210120A5
:1014B00001E00021052000F043FC45F080000E4DC6
:1014C0000023012229462870184600F093FC0023CF
:1014D00029460222184600F069FC3CB1012C04D1D7
:1014E0000121052000F02CFC287870BD0121084660
:1014F00000F026FC687870BDAD00002410B50446ED
:10150000124801F07F0101704270012000F087FC59
:1015100014B1012C07D102E00021012001E00021DB
:10152000052000F00DFC002308490222184600F0B7
:1015300061FC3CB1012C08D101210520BDE810401F
:1015400000F0FEBB01210846F8E710BDAD00002405
:101550002DE9F04716008846074600D10A261F4CA1
:101560006421A0680CF043FB18B16FF00400BDE8E3
:10157000F08760684FF0FF390BE00178B94207D17E
:101580004268424504D1A0680CF08EFB4846EEE765
:1015900000690028F1D1142000F0E6FB050012D00C
:1015A0000022304654210CF0B1FAA86088B12F70A7
:1015B000C5F804802E73606828616560A0680CF02F
:1015C00073FB0020D3E7A0680CF06EFB6FF0010006
:1015D000CDE7284600F062FBD5E700009C00002420
:1015E00070470000074A526808E01378834204D12C
:1015F00053688B4201D1906870471269002AF4D178
:10160000002070479C000024D0E901014FF0804287
:10161000B1F1005F03D0904207D1012070479042A2
:1016200001D103207047022070470020704700005E
:10163000032804D228B1012805D0022805D00020B3
:1016400070470348704703487047034870470000DD
:101650004C040024EC0400248C0500242DE9F04106
:10166000164C0746984615460E46207848B15DB19F
:10167000A06864210CF0BBFA48B16FF00400BDE82B
:10168000F0816FF00200FAE76FF00100F7E73146F2
:101690003846FFF7A7FF0646A0680CF005FB56B1D9
:1016A00000224346294630460CF0FEF90028E6D0D9
:1016B0004FF0FF30E3E76FF00300E0E79C00002409
:1016C0002DE9F041694F8AB0387820B16FF00200FF
:1016D0000AB0BDE8F08166486021FFF73EF8644A31
:1016E000002420466032C1B2032908D240F291138F
:1016F000594302EBC101C1F8804CC1F8844C401C35
:101700000328F0DB5B48F86000200CF099FA002811
:10171000B8607DD001263E7002940225019401A993
:101720005548CDE9046403950694079403F03AFB09
:101730006F070197CDE902654F4801A9CDE904641F
:101740000694079403F02EFB02224B480023114617
:10175000009403F066FB49490022474803F0AAFAC7
:10176000474A0321002000F09FF80021454A08461F
:1017700000F09AF8404804F041F8029401A901945D
:101780004148CDE9045403950694079403F00AFBFD
:10179000CDE90265019701A93B48CDE904540694BF
:1017A000079403F0FFFA0222374800231146009401
:1017B00003F037FBDFF8C4800022334808F10F083C
:1017C000414603F077FA314A0521012000F06CF818
:1017D0002C4A0021012000F067F82B4804F00EF895
:1017E000029401A901942A48CDE904540395069472
:1017F000079403F0D7FACDE90265019701A92448BF
:10180000CDE904540694079403F0CCFA002300E0D9
:1018100029E002221E481146009403F002FB1C48F6
:101820000022414603F046FA184A0521022000F042
:101830003BF8144A0021022000F036F8144803F067
:10184000DDFF144C01225103204604F064F901220B
:101850002046910304F05FF901222046D10304F0F1
:101860005AF9002034E74FF0FF3031E79C000024A4
:10187000F0960024E11500084C0400240110020039
:10188000F9180008FD1B0008EC040024AD1900083D
:101890008C05002400080258024AD268002A00D0B1
:1018A000104770479C0000240C4B1B7843B152B189
:1018B00003284FF0FF3301D2082907D31846704799
:1018C0006FF0020070476FF001007047044B03EBAC
:1018D000401040F821200020704700009C000024A8
:1018E000F0960024034B1B780BB1FFF731BE6FF06D
:1018F000020070479C0000242DE9F0430024AFB0A3
:10190000E0B2FFF795FE060044D03DE040213046AE
:101910001FAB15AA03F0BEFAE0BB16980028159875
:101920003ED020F0604515A8FFF76EFE80460146C8
:101930002846FFF7B1FF81464946E0B2FFF752FE65
:10194000070021D08DF80080CDE90159189816497B
:1019500000F00F00085C8DF80C00402802D94020F0
:101960008DF80C000DF10D0040210546FEF7D3FE69
:101970009DF80C201FA92846FEF74EFE002369465D
:101980001A4638460CF0EEF84021304603F076FA5D
:101990000028BBD1641C032CB2DB2FB0BDE8F08360
:1019A000C0F30A05BFE70000700001082DE9F0430D
:1019B0000024AFB0E0B2FFF73BFE060044D03DE0AC
:1019C000412130461FAB15AA03F064FAE0BB16981C
:1019D000002815983ED020F0604515A8FFF714FEAA
:1019E000804601462846FFF757FF81464946E0B248
:1019F000FFF7F8FD070021D08DF80080CDE90159EF
:101A00001898164900F00F00085C8DF80C0040286B
:101A100002D940208DF80C000DF10D004021054643
:101A2000FEF779FE9DF80C201FA92846FEF7F4FD6D
:101A3000002369461A4638460CF094F84121304696
:101A400003F01CFA0028BBD1641C032CB2DB2FB0BE
:101A5000BDE8F083C0F30A05BFE70000700001088D
:101A60002DE9F04780465C489AB0994615460F46E6
:101A70000078229C50B1B8F1030F4FF0FF3A7DD2AD
:101A8000B9F1000F6FF0010105D008E06FF002001E
:101A90001AB0BDE8F087022F01D0032F17D1402CD8
:101AA0006CD84046FFF7C4FD060010D0642168469C
:101AB000FEF753FE4FF000005FB1012F4FF0804161
:101AC0000BD04A10022F0CD0032F73D10DE0084623
:101AD000DEE7CDE9005002900AE00095CDE9011063
:101AE00006E00095CDE9010202E00095CDE9011282
:101AF000B2684FF40011B2F5807F12D0B2F5407F8A
:101B00000AD00590069001210490CA05082CCDE961
:101B1000072109D8204620E04FF48012CDE90521A5
:101B2000F1E7CDE90501EEE70C2C01D8092014E01E
:101B3000102C01D80A2010E0142C01D80B200CE046
:101B4000182C01D80C2008E0202C01D80D2004E02E
:101B5000302C01D80E2000E00F20039009A8214668
:101B60000546FEF7FAFDB9F1000005D024B1224682
:101B700001462846FEF750FD304600E01AE003F02B
:101B8000A7FA30B12A466946304603F0D7F8002854
:101B90009ED040F29112694618FB02F00F4A02EB08
:101BA000C004D4F8800CD4F8842C401C00F01F052D
:101BB000AA4201D150466BE7D4F8800C00EBC0027A
:101BC00002EB0010642204EB8000FEF76AFDC4F80B
:101BD000805C00205CE700009C00002450970024FB
:101BE00008B539B10A794B1D00920A680021FFF748
:101BF00037FF08BD6FF0010008BD00002DE9F0417E
:101C0000DFF894800025A4B0ECB22046FFF710FD69
:101C100007003AD019A9384603F002FA0028F9D093
:101C200020E0032C684630D2D6F8801CD6F8842CED
:101C300091422AD0D6F8841C01EBC10202EB0111BB
:101C4000642206EB8101FEF72CFDD6F8840C401CC3
:101C500000F01F00C6F8840C09AA6946384603F054
:101C60006DF890B9032C10D240F2911204FB02F1EE
:101C700008EBC106D6F8800CD6F8841C884204D044
:101C8000384603F025FA0028CBD16D1C032DBBDBB1
:101C900024B0BDE8F0810000509700240CF070BE25
:101CA00010B530B1062804D0072802D04FF0FF301D
:101CB00010BD282003F0C8FF002010BD10B530B1C2
:101CC000062804D0072802D04FF0FF3010BD28208E
:101CD00003F0CBFF002010BD082810B509D206493B
:101CE00001EBC00231F83010506803F00FFF0128FB
:101CF00000D0002010BD00008000010810B521B107
:101D0000082805D34FF0FF3010BD6FF0010010BD63
:101D1000094A012432F830205FF0000004FA00F391
:101D2000134203D0054A42F8201003E0401CC0B221
:101D30001028F3D3002010BD80000108E8BC002467
:101D4000082810B502D34FF0FF3010BD054A02EB52
:101D5000C00432F830300A466068194603F0DBFEF2
:101D6000002010BD800001080CF082BC022810B5D4
:101D700002D34FF0FF3010BD044901EBC00251F80F
:101D80003000918806F0D8FC002010BDC00001088A
:101D900018B1012803D0002070470248704702485C
:101DA000704700002C060024B406002410B5022859
:101DB0004FF0FF3406D2FFF7EBFF18B123B105F067
:101DC0006DFE04E0204610BD142305F02DFD002813
:101DD000F9D0012010BD000032B1054B03EB4010DB
:101DE00040F82120002070476FF00100704700008C
:101DF00028BD002410B502284FF0FF3406D2FFF7AB
:101E0000C7FF18B123B106F065F804E0204610BD05
:101E1000142305F03EFF0028F9D0012010BD70B555
:101E200005460BF0DCFD4FF47A71B1FBF0F0B5FB29
:101E3000F0F40BF0BDFD02284FF0FF3110D005DCAF
:101E400088420BD090B1012813D10FE0032805D0B0
:101E5000042803D06FF0004290420AD1084670BDBA
:101E600004B9012420460BF07EFD02E0284602F072
:101E70000FFF002070BD2DE9F0410BF0B0FD0646CC
:101E80000DF0B4FD4FF47A784FF0E024B8FBF6F192
:101E9000A76900FB01F50DF0A9FDB8FBF6F2A169F9
:101EA000504385420AD1616900EB40034246C3EBCF
:101EB000C0105743491CB7FBF1F10AE062694FF4C7
:101EC0007A7300EB40055943521CB1FBF2F1C5EBAC
:101ED000C010C1EBC000002100F57A70BDE8F081B0
:101EE00008B100207047014870470000C408002472
:101EF0000AB128B902E06FF001007047092902D346
:101F00004FF0FF307047024840F821200020704712
:101F100068BD0024FEE7000000B593B030B3012196
:101F2000009108228DF8042002780021114B8DF8D1
:101F3000052042788DF8062082781B78D21A8DF819
:101F40000720C0788DF8080000208DF809108DF862
:101F50000A108DF80B108DF80C106946FFF740FE43
:101F6000002801D04FF0FF3013B000BD6FF001002A
:101F7000FAE70000BC000024042808D239B1084A5E
:101F800052F8200030B1026922B1806810474FF04A
:101F9000FF307047027900208854001F704700000E
:101FA000B8BD002470B50A4800F016F8084818308B
:101FB00000F012F8074D002455F8240018B1C1684C
:101FC00009B180688847641C042CF5DB002070BDD3
:101FD000F8030024B8BD002410B10179042902D30C
:101FE0004FF0FF307047024A42F82100002070474E
:101FF000B8BD0024F8B568B117A200F1100112684D
:10200000009290F87820042A07D2032A05D0525C67
:10201000D2B902E04FF0FF30F8BD04256C46002233
:10202000A35CC618367C16B180F8783004E0521CE8
:1020300080F87850032AF3DB90F8782080F87C2031
:1020400080F8902080F8A020012300F1440200F0E5
:10205000C3F80020F8BD000001000200016890ED07
:10206000210AD1ED030A20EE200A80ED210AD1EDEC
:10207000030A90ED220A20EE200A80ED220A0020B9
:10208000704700207047016890ED220AD1ED020AE6
:1020900030EE600A80ED220A0020704790F8781038
:1020A000012901D011B10AE0002100E0012180F8EE
:1020B000781080F87C1080F8901080F8A010002034
:1020C0007047016890ED210AD1ED040A20EE200A44
:1020D00080ED210AD1ED040A90ED220A20EE200ABB
:1020E00080ED220A00207047012180F8A310002013
:1020F000704790F8A110491C01F0030180F8A1106D
:1021000000207047016890ED220AD1ED020A30EEFE
:10211000200A80ED220A00207047016890ED210A14
:10212000D1ED020A30EE600A80ED210A00207047EE
:10213000016890ED210AD1ED020A30EE200A80ED0F
:10214000210A00207047042280F88020022180F8B4
:10215000811080F8941000207047002070479AB3D7
:1021600090B35368B3F1004F10D0B3F1804F13D048
:10217000B3F1005F18D03BB3806A33EA000019D096
:102180000020C9B1896A8B430CD015E090F8220079
:1021900091B191F8221004E090F8230061B191F818
:1021A000231049B1012108E090F8240021B191F8F1
:1021B0002410F6E70120E4E70021127A002A04D077
:1021C000012A03D0022A03D00020704788437047B9
:1021D00021EA0000704700002DE9F0475FEA00099E
:1021E0001E46924688461AD0B8F1000F17D00D4F00
:1021F0005FF0000407EB0415687A304209D02A46E4
:1022000051464046FFF7ABFF18B1E96809B14846AF
:102210008847641C0B2CEDD30020BDE8F0874FF0FD
:10222000FF30FAE7D000010800F080BE0078704768
:102230000022CA610A624A628A6202784A70428F48
:102240008A83828FCA8390F8402081F8222090F8F8
:10225000412081F82320B0F81F00886200207047D9
:1022600070B50C4605461821201DFEF776FA287831
:1022700001212070022295ED090A032384ED010A51
:1022800095ED0A0A002684ED020A95ED0B0A84ED0D
:10229000030A95ED0C0A84ED040A95F8390001282B
:1022A00014D0022816D0032812D0267595F83800CD
:1022B000012811D0022813D003280FD084F815600C
:1022C000002095ED0D0A84ED060A70BD2175EDE73D
:1022D0002275EBE72375E9E76175F1E76275EFE7D2
:1022E0006375EDE72DE9F04104002DED028B2AD056
:1022F000FFF7C1FD06460D460DF0DFFD00EE100AAA
:102300009FED1E8A0027C0EE080AC4ED010AE068AE
:10231000301A65EB07010DF0D0FD00EE100AC0EE9B
:10232000080AC4ED020A94F87800E66004280DD388
:1023300084F88070381F84F8947084F8A170BDEC24
:10234000028BBDE8F0814FF0FF30F8E794F8900081
:102350000B4D05EB001081682046884794F87C00FF
:1023600005EB001041682046884794F8A00005EB73
:102370000010C168204688470020E0E70024744927
:10238000B803002470B505000C460AD04CB1A42156
:10239000FEF7E3F92C60FFF705FEFFF7DEFE0020F5
:1023A00070BD4FF0FF3070BD417C79B1022180F8E3
:1023B00080109FED080A00F144020B4680ED210ACF
:1023C00080ED220A00F11001FFF706BF002180F81E
:1023D00080107047000000000168427C091D62B354
:1023E000012280F89420B0F92C2090ED020A52428C
:1023F00000EE902A0423B8EEE01AD1ED000A21EE97
:10240000001A61EE200AC0ED260AB0F92E2091EDE7
:10241000001A00EE902A00F1440200F11001F8EEDB
:10242000E00A60EE800AB7EE080A60EE810A20EE4C
:10243000800A80ED270AFFF7CFBE002180F89410B4
:102440007047417C69B1012290F8321080F8A220D7
:10245000082300F1440280F8A31000F11001FFF7F7
:10246000BBBE002180F8A1107047016890F82420BD
:102470001431012A05D0022A05D0032A0FD00021E9
:1024800002E0097800E0497880F8801090ED070AB2
:10249000D0ED080A80ED210AC0ED220A7047897844
:1024A000F2E7016890F824201431012A05D0022AAD
:1024B00005D0032A17D0002102E0C97800E009798D
:1024C00080F89410D0ED050A90ED060AF8EE001A97
:1024D000BFEE081A60EEA10A20EE010AC0ED260A3E
:1024E00080ED270A70474979EAE7037C0122002141
:1024F00013B180F8A12001E080F8A11090F82530F8
:10250000022B09D0032B02D080F8A21006E080F83D
:10251000A22080F8A320704780F8A22080F8A310A2
:10252000704710B5044600F00BF8002807D120468C
:10253000FFF760FD2046BDE81040FFF7D3BE10BD99
:1025400070B580B100F1100134220D464430FEF721
:10255000A8F800242946E0B2FFF70EFD641C042C05
:10256000F8DB002070BD4FF0FF3070BD2DE9F04169
:10257000040015460E462DED048B65D0F6B3D4E964
:1025800000020027281A67EB02010DF096FC00EE0E
:10259000900A9FED841AC4E9005780EE810A10EE7C
:1025A000100A84ED020A6FEAD05010F0FF0F9FED81
:1025B0007E9A04D0B5EEC00AF1EE10FA01D884ED8F
:1025C000029A7A49A068884203DA9FED790A84ED7D
:1025D000020A7849A068884203DD9FED770A84EDFE
:1025E000020A31782A46204600F0B2F9207C9FED9D
:1025F000738A01282ED0052831D000E024E094ED24
:10260000B70AD4ED0C0A70EE609AB0EE690A0AF0CF
:10261000C5FDF0EE400AB0EE690AF0EE608A0AF0FD
:1026200089FED6ED010A96ED021A60EEA80A40EE88
:10263000410AC4ED050AD6ED010A96ED021A20EE14
:10264000800A08EE810A10E06FF00100BDEC048BF7
:10265000BDE8F08184ED068A84ED058A07E096EDF9
:10266000010A84ED050A96ED020A84ED060A217C32
:1026700004F59C70072914D2DFE801F004040A2055
:102680002F04070084ED078A0BE096ED030A06E0AD
:10269000D4ED021AD4EDB70A94ED0C0A18E084EDDB
:1026A000070A94F911309FED460A04F11401881EBF
:1026B00004F1380207F060FB00256CE094ED0C0A91
:1026C0009FED401AD4ED021AD4EDB70A30EE010A9C
:1026D000B0EE481A07F0B6FCE1E700EE105ADFED65
:1026E0003A8ADFED3A9AB8EE400A20EE090A0AF07B
:1026F00021FEDFED370A20EE200AB0EEC00A30EEF0
:10270000280A89FEC00AD4ED0D0A20EE200AC6E789
:1027100004EB051104EB451791EDA80A04EB8506BF
:1027200007F5C67006F022FC207CF0EE400A072870
:102730001ED2DFE800F01B04040404041400C5EBFF
:102740000510D4ED021A04EB8000483096ED0E0A15
:10275000B0EE481A07F076FCF0EE408A08E096EDFD
:102760000E0ADFED1C0AC0EE208A01E0F0EE488A76
:1027700007F50370B0EE680A06F0F8FB86EDA30AD1
:10278000E16806F52370D1ED1F0AB1EE600A00F092
:1027900086F96D1CEDB294F91100A842B8DC002056
:1027A00054E7000000007A446F12833A6F12033A34
:1027B0006F12033ACDCC4C3DCDCC4C3D0000000017
:1027C0000000FA43AB611C3F9A99193FCDCC4C3FB6
:1027D000CDCC4C3E00C0DA452DE9F04104000E4658
:1027E0002DED028BF0EE408A0FD0FEF769FFE66018
:1027F00000212174042096F86010072922D2DFE816
:1028000001F00A0C171A1C211E006FF00100BDEC2C
:10281000028BBDE8F081002700E0012760740020F2
:102820009FED388A054684ED028AC4E9000037E04E
:1028300002200746F2E70327F0E70427EEE701202E
:102840000527EBE76FF00300E1E700BFC5EB0510DC
:10285000002104EB80004830B0EE680A06F1200247
:1028600007F0A4FC04EB4518D6ED190AB0EE680A8F
:1028700008F5C67006F0A8FBD6ED1A0AB0EE680A95
:1028800008F5037006F0A0FB04EB0510691C80ED51
:10289000A88A80EDA98A80EDA78A80EDAA8ACDB2A8
:1028A00094F91100A842D1DC0021B0EE680A06F1CB
:1028B000400204F59C7007F079FC04F112003946DF
:1028C00007F006FB84ED078A84ED068A002084ED7C
:1028D000058A05E0411C04EB800080EDA38AC8B2A4
:1028E00094F911108142F5DC002505E0E06800EB69
:1028F000C50006F093FE6D1C94F91100A842F5DCAA
:10290000002084E70000000070B504001ED0002500
:102910000AE000BF04EB8501086A18B191EDA30A33
:1029200006F0E4FE6D1CEDB294F91100A842F1DC52
:10293000002507E004EB8500006A08B106F0CEFD33
:102940006D1CEDB294F91100A842F3DC70BD0000DB
:102950002DE9F04104000E462DED028B07D0207CBE
:10296000B04207D10020BDEC028BBDE8F0816FF0D2
:102970000100F8E7042E11D104280FD01046FDF70E
:102980002DFEFDF775FDC00701D0701F00E001208E
:1029900000EE100AB8EEC00A84ED0D0A00259FED86
:1029A000108A16E0C5EB051004EB8000483007F0F4
:1029B0003DFC04EB4517B0EE480A07F5C67006F07B
:1029C00069FBB0EE480A07F5037006F063FB6D1C67
:1029D000EDB294F91100A842E4DC2674C2E70000CD
:1029E0000000000070B50024054617E0E86800EB21
:1029F000C40006F0D3FEE86800EBC40006F0F3FD67
:102A000005EB8401086278B1083005EB041606F581
:102A100027760FC8641C86E80F00E4B295F9110010
:102A2000A042E3DC002070BD6FF0010070BD90EDAE
:102A3000001AF5EEC00AF1EE10FA31EE000A0EDDD2
:102A4000B4EEE00AF1EE10FA02DB30EE600A06E0C6
:102A5000B5EEC00AF1EE10FA01D230EE200A80ED98
:102A6000000A7047B5EEC01AF1EE10FA30EE600AB7
:102A70000ADDF6EE000A61EE200AB4EEE00AF1EE9D
:102A800010FA02DD30EE410A7047F1EE600AB4EE52
:102A9000E00AF1EE10FAF7D230EE010A704790ED3D
:102AA000001AB4EEE01AF1EE10FA02DCF0EE410A80
:102AB00001E0C0ED000AF4EEC00AF1EE10FA01D216
:102AC00080ED000A7047000000487047D8000024DD
:102AD000014801F03DBA00003C070024014801F024
:102AE00037BA0000B4070024014801F031BA0000F1
:102AF00058090024294A016891423AD0274A1832DD
:102B0000914236D0254A3032914232D0234A48325F
:102B100091422ED0214A603291422AD01F4A783207
:102B2000914226D01D4A9032914222D01B4AA832AF
:102B300091421ED01A4A91421BD0194A1832914232
:102B400017D0174A3032914213D0154A4832914279
:102B50000FD0134A603291420BD0114A7832914221
:102B600007D00F4A9032914203D00D4AA8329142C9
:102B700011D1CAB21823103AB2FBF3F26FF3090174
:102B8000032A02F00703074AD25CC26500D9091D77
:102B900081650846704721F0FF01F9E71000024007
:102BA00010040240D4FF000830B5224A0123016816
:102BB0009142CAB21BD01F4C1434A14217D01D4CF5
:102BC0002834A14213D01B4C3C34A1420FD0194CE5
:102BD0005034A1420BD0174C6434A14207D0154C9D
:102BE0007834A14203D0134C8C34A1420CD114216F
:102BF000114C083AB2FBF1F10F4A803201F01F0587
:102C000004EB8101AB4010E00C4D1824103A0D4448
:102C1000B2FBF4F1A82D00D80831094A01F01F04D5
:102C200002EB8101064AA3408032603080E80E004A
:102C300030BD00000854025800580258F0FBFDBF98
:102C40000008024010B50279531E072B2DD8174CEF
:102C50000168A1421BD0154C1434A14217D0134C6B
:102C60002834A14213D0114C3C34A1420FD00F4C58
:102C70005034A1420BD00D4C6434A14207D00B4C10
:102C80007834A14203D0094C8C34A14203D10849C5
:102C9000074C443102E00749064C443104EB820200
:102CA000C0E91B2101219940416710BD0854025819
:102CB000FC580258FC08024010B583694FF0C074FC
:102CC000826A0146002053B1B3F5005F15D072B19E
:102CD000012A0CD0022A0AD0032A09D104E01AB131
:102CE000012A06D0022A03D1C96AC90100D50120F0
:102CF00010BDC96AA142FAD010BD002AF7D0012A3E
:102D0000F2D0022AF3D0032AF3D010BD2DE9F04F00
:102D1000804E804FDFF8FC911836DFF8F8A1483775
:102D20000468856D0AF1300ADFF8ECB14C45DFF834
:102D3000ECC1DFF8ECE16DD0B4426BD0544569D002
:102D4000BC4267D0DFF8D081A8F11808444561D0B3
:102D50005C455FD064455DD074455BD0DFF8C481CD
:102D6000444557D0DFF8BC8108F11808444551D0DC
:102D7000DFF8B08108F1300844454BD0DFF8A4817A
:102D800008F14808444545D0DFF8988108F160080B
:102D900044453FD0DFF88C8108F17808444539D0AC
:102DA000DFF8808108F19008444533D0DFF8748162
:102DB00008F1A80844452DD0DFF86C81444529D09E
:102DC000DFF8648108F11408444523D0DFF8588106
:102DD00008F1280844451DD0DFF84C8108F13C0873
:102DE000444517D0DFF8408108F15008444511D020
:102DF000DFF8348108F1640844450BD0DFF82881FE
:102E000008F17808444505D0DFF81C8108F18C08EA
:102E1000444509D1D0E91948C4F80480C46E1CB1F6
:102E2000D0E91C48C4F8048004684C452ED0B44254
:102E30002CD054452AD0BC4228D0374E183EB4423C
:102E400024D05C4522D0644520D074451ED0354E38
:102E5000B4421BD0334E1836B44217D0314E303600
:102E6000B44213D02F4E4836B4420FD02D4E6036A8
:102E7000B4420BD02B4E7836B44207D0294E903650
:102E8000B44203D0274EA836B44215D190F85C6006
:102E90003F2406F01F06B440AC600468256825F4A2
:102EA000802525602EE09A600068C160BDE8F08F43
:102EB00099600068C260F9E71B4EB4421BD01A4EFD
:102EC0001436B44217D0184E2836B44213D0164EDA
:102ED0003C36B4420FD0144E5036B4420BD0124E92
:102EE0006436B44207D0104E7836B44203D00E4E4A
:102EF0008C36B442DAD190F85C60012406F01F06EB
:102F0000B4406C60046863608368402B0368CFD171
:102F1000C9E700001000024088000240A000024003
:102F2000B8000240100402400854025870B56FF017
:102F3000010590B10A4C207810B16FF0020070BD0D
:102F40000AF05AFF606040B1064A03210020FEF7F4
:102F5000CFFF01202070002070BD284670BD00000A
:102F6000B40000242131000810B538B1002100F868
:102F7000241B3421FDF7F1FB002010BD6FF0010090
:102F800010BD000070B504007ED0218A01254FF4E9
:102F9000A560C1F30A01A1F5B671814275D8B4F8F4
:102FA0001110C1F3CA01A1F5B67181427FD8B4F8FE
:102FB0001310C1F30A01A1F5B671814277D8A18A35
:102FC000C1F3CA01A1F5B671814270D8A07D800716
:102FD0006DD0607D80096AD02570FEF74CFFC4E992
:102FE0000201342104F12400FDF7B7FB208A9FED94
:102FF0004A0AF0EE000A9FED491AC0F30A00A18ABE
:1030000001EE900AA27DC1F3CA00637DB8EE612A89
:1030100001EE900A667F02F003019A0932EE402A1F
:10302000F8EE612A002E62EE201A72EEC02A81EEBE
:10303000812A62EEA01A84ED0B2AB4F8110081EE09
:10304000812AC0F3CA0001EE900AF8EE611A71EE0F
:10305000C01A61EEA01AC1EE812AC4ED0C2AB4F8A0
:10306000130084ED0A2A84F83910C0F30A0084F8AA
:10307000382001EE900AF8EE611A71EEC01A61EE86
:10308000A01A81EE812A01E00EE010E084ED092A09
:10309000B4F817006087B4F81900A087B4F81B00D3
:1030A000E08707D0012006E06FF0010070BD4FF00F
:1030B000FF3070BD0020A17F84F8400009B10120DD
:1030C00000E0002084F84100B4F81F205FF0000009
:1030D00005FA00F1114000D001212318401C0F28EF
:1030E00083F84210F4DD94F8400094F8411084F81D
:1030F000520084F85310B4F8210001EE900A002029
:10310000F8EE611A31EEC00A20EE200AC0EE010A84
:10311000C4ED0D0A70BD0000000080440000A5440D
:103120000248012140680AF0E1BD0000B40000241B
:1031300010B504460020FEF7D3FE132204F110015F
:1031400005F094FE002801D04FF0FF3010BD0121A2
:103150000246084610B50AF003FE012800D0002000
:1031600010BD70474FF4806010B502F0B5FB4FF40E
:10317000805002F0B1FBBDE810404FF4004002F077
:10318000ABBB72B6FEE70000054805490839026886
:1031900042F00202026008688004FCD5704700001B
:1031A0000C480258014801F09BBF00004C04002469
:1031B000014801F095BF00004C040024014801F0D3
:1031C0008FBF0000EC040024014801F089BF00001B
:1031D000EC040024014801F083BF00008C050024AA
:1031E000014801F07DBF00008C050024F0B50368A4
:1031F0004FF6FC716D4C426BD3F884508D4345EA19
:103200008205C3F88450036853F8845F068F25F461
:103210007F0545EA06451D60836B654D9F18026872
:10322000D2F888308B4343EA8703C2F888300268BB
:1032300052F8883F868F23F4FE0343EA0643136067
:10324000066856F8A03FC26B8B4307EB420243EA85
:1032500082033360076857F8A03FB0F8406023F45A
:10326000FE0343EA06433B60D0E9103603FB062227
:103270000368D3F8B0608E4346EA8206C3F8B060B4
:103280000368B0F84860D3F8B07027F4FE0747EA47
:103290000646C3F8B060D0E91267036806FB072250
:1032A000D3F8AC608E4346EA8206C3F8AC60D0E93E
:1032B0001467036806FB0722D3F8F0608E4346EAE2
:1032C0008206C3F8F0600368B0F85860D3F8F07075
:1032D00027F47C1747EA0646C3F8F0600368876D59
:1032E00053F8C06F02EB47028E4346EA8201196031
:1032F0000168B0F85C20D1F8C03023F47C1343EAB5
:103300000242C1F8C020016890F86020D1F8C030B6
:1033100023F07C5343EA0262C1F8C020416B04EB06
:103320008101C166826B01EB82020267C36B02EB13
:10333000C3024267D0E91034634302EB8302826721
:10334000D0E91234634302EB8302C267D0E914343C
:10335000634302EB8302C0F88020836D02EBC3035A
:10336000C0F88430C46D826E544303EB8403C0F80C
:103370008830046E544303EB8402C0F89020AA42C4
:103380000AD9D0F89C20032142F02002C0F89C20EA
:1033900080F898100120F0BD002200E004C1D0F8B0
:1033A00090308B42FAD80020F0BD000000AC004005
:1033B000FCD30040F0B58E680C69D1E9005744EAAF
:1033C0000604DFB145F080452C43866ED1E906C581
:1033D0004F695E4391F8203045EA0C05B1F80CC006
:1033E000D0F884E0002047EA0363104F1D430EEB42
:1033F000860345EA0C45E3E8024511E044EA8544CA
:10340000E3E71418155CA67894F803C094F801E07B
:10341000360445EA0C6446EA0E252C43001D10C311
:10342000CC683C5D8442ECD8F0BD0000DCFF0008B5
:1034300078B100680849884201D1002070470749E7
:10344000884201D1012070470549884201D10220FC
:10345000704704207047000000A0004000A4004016
:1034600000D400402DE9F04104000D462DED068BFF
:1034700038D0B5B3FEF7FFFCD4E90023801A61EB26
:1034800003010CF01AFD00EE100ADFEDA00A80EE39
:10349000201A84ED021AFEF7EEFCC4E90001297837
:1034A000204600F0DDF995ED010AD4ED020A984EB0
:1034B000984F60EE200AB7EE081ADFED979A9FED5D
:1034C00097AAE06860EE818A90ED280AB5EEC00AFE
:1034D000F1EE10FA49DD207C012809D0022810D134
:1034E00009E0FFE74FF0FF30BDEC068BBDE8F0814F
:1034F000B0EE699A11E094ED600AD4ED5D0A30EE09
:10350000609A19EE100AB04201DD39EE4A9A19EEBE
:10351000100AB84201D939EE0A9A94ED050AB0EEC4
:103520004A1A70EE090A94ED440A70EEA80AFFF7F1
:1035300099FAB0EE408A94ED050AB0EE4A1A70EEA0
:10354000090A94ED450A70EEA80AFFF78BFAF4EE2B
:10355000C88AF1EE10FA01DDF0EE488AF4EEC08A76
:10356000F1EE10FA01D2F0EE408AB0EE4A9AB0EED7
:10357000680AF0EE490A04F11400FFF758FAE0680F
:10358000D5ED020A94ED021A90ED290A60EE818AC7
:10359000B5EEC00AF1EE10FA42DD207C012802D01F
:1035A000022809D102E0B0EE698A11E094ED640AC4
:1035B000D4ED5E0A30EE608A18EE100AB04201DDEA
:1035C00038EE498A18EE100AB84201D938EE098A55
:1035D00094ED060AB0EE491A70EE080A94ED460A18
:1035E00070EEA80AFFF73EFAB0EE40AA94ED060A84
:1035F000B0EE491A70EE080A94ED470A70EEA80A78
:10360000FFF730FAF4EECA8AF1EE10FA01DDF0EEBF
:103610004A8AF4EEC08AF1EE10FA01D2F0EE408A46
:10362000F0EE490AB0EE680A04F11800FFF7FFF95E
:10363000217C71B1012904F1200204F1980604F5FE
:10364000907804F5A07504F1D40707D002295AD167
:103650001FE0C4ED589AC4ED599A54E0D4ED021A13
:10366000D4ED600A94ED050AB0EE691A104606F032
:10367000E9FCD4ED021AD4ED5C0AB0EE691A3846C2
:1036800006F0E0FC84ED580AD4ED021AD4ED640A89
:1036900019E0D4ED021AD4ED5D0A94ED050AB0EEFE
:1036A000691A104606F0CEFCD4ED021AD4ED5C0A7D
:1036B000B0EE691A384606F0C5FC84ED580AD4ED20
:1036C000021AD4ED5E0A94ED060AB0EE691A30468D
:1036D00006F0B8FCD4ED021AD4ED5A0AB0EE691A1D
:1036E000384606F0AFFC84ED590A94ED580A40467E
:1036F00005F03CFC84ED580A94ED590A284605F083
:1037000035FC84ED590A0020EEE6000000247449DF
:10371000DB0F4940DB0F49C000000000DB0FC94050
:1037200010B504002DED028BB0EE408A65D0E1604B
:10373000002001F130020146B0EE480A207404F185
:10374000200006F033FDE2680121B0EE480A103295
:1037500004F15C0006F02AFDE2680021B0EE480AA0
:10376000703204F1980006F021FDE2680121B0EE0C
:10377000480A503204F1D40006F018FDE068B0EEBB
:10378000480AD0ED240A04F5907005F01DFCE068AD
:10379000B0EE480AD0ED240A04F5A07005F014FC40
:1037A000E06890ED260AD0ED280A30EE200A84ED7C
:1037B000440A90ED260A84ED450A90ED270AD0EDE3
:1037C000290A30EE200A84ED460A90ED270A84ED9E
:1037D000470AFDF775FFE06805F056FDE068083020
:1037E00005F052FDE06805F079FCE068083005F06E
:1037F00075FC0020BDEC028B10BD4FF0FF30F9E7E7
:1038000010B58AB0044614216846FCF7A6FF94ED73
:10381000590AF1EE040AB7EE001A20EE200A6946B2
:103820008DED000A8DED041AE06805F0AEFC142160
:1038300005A8FCF792FFD4ED580AB2EE001A9FEDEE
:10384000070A60EE810A05A9CDED050A8DED090A8A
:10385000E068083005F099FC0AB010BD9A99993ECD
:1038600070B504000D462DED028B06D0207CA842D9
:1038700006D10020BDEC028B70BD4FF0FF30F9E7A0
:1038800004F1200006F0D2FC04F15C0006F0CEFC4E
:1038900004F1980006F0CAFC04F1D40006F0C6FC5E
:1038A0009FED158A04F59070B0EE480A05F0F2FB22
:1038B000B0EE480A04F5A07005F0ECFBE0680830B3
:1038C00005F00CFCE06805F009FC04F11400FDF7BC
:1038D000AFF894ED640A012D84ED060A02D0022DA2
:1038E00003D006E094ED600A01E094ED5D0A84EDFA
:1038F000050A2574BDE700000000000010B50400B3
:103900001DD0E06805F09EFDE06805F01FFC28B1C1
:103910001C3004F5C87C0FC88CE80F00E068083044
:1039200005F090FDE068083005F010FC28B11C306F
:1039300004F5C0740FC884E80F00002010BD4FF0DC
:10394000FF3010BD30B558B100F5BA7238C900F576
:10395000B47080E838000BC982E80B00002030BD4D
:103960004FF0FF3030BD00002DE9F84F044602F063
:10397000D7F800903CB194F83500022806D0802199
:1039800061650020E4E00120BDE8F88FC74DC74E17
:10399000C649183520683036DFF81483DFF81493F1
:1039A0008842DFF814A3DFF814B32ED0A8422CD03D
:1039B000B0422AD0404528D0484526D0504524D092
:1039C000584522D0BD4A183290421ED0BC4A90427F
:1039D0001BD0BB4A1832904217D0B94A30329042BD
:1039E00013D0B74A483290420FD0B54A6032904265
:1039F0000BD0B34A7832904207D0B14A903290420D
:103A000003D0AF4AA832904209D1026822F01E02C8
:103A100002602068426922F08002426103E002688D
:103A200022F00E02026027688F4238464DD0A8422D
:103A30004BD0B04249D0404547D0484545D050458D
:103A400043D0584541D09D4A183290423DD09C4ABF
:103A500090423AD09A4A1832904236D0984A303240
:103A6000904232D0964A483290422ED0944A6032E8
:103A700090422AD0924A7832904226D0904A903290
:103A8000904222D08E4AA83290421ED08D4A904257
:103A90001BD08C4A1432904217D08A4A2832904266
:103AA00013D0884A3C3290420FD0864A503290421E
:103AB0000BD0844A6432904207D0824A78329042D6
:103AC00003D0804A8C32974204D1206E026822F4DF
:103AD0008072026075492068884228D0A84226D0AA
:103AE000B04224D0404522D0484520D050451ED079
:103AF00058451CD071491831884218D07049884205
:103B000015D06F491831884211D06D493031884243
:103B10000DD06B494831884209D0694960318842EB
:103B200005D067497831884201D0654990310168F4
:103B300021F0010101600EE001F0F2FF0099401A4E
:103B4000052808D9202262650321002084F8351059
:103B500084F8340017E73868C007EDD1534A0121D3
:103B6000206890422ED0A8422CD0B0422AD04045A6
:103B700028D0484526D0504524D0584522D04F4B18
:103B8000183398421ED04E4B98421BD04C4B1833E2
:103B9000984217D04A4B3033984213D0484B4833A1
:103BA00098420FD0464B603398420BD0444B783349
:103BB000984207D0424B9033984203D0404BA833F1
:103BC000984208D194F85C703F23A06D07F01F075E
:103BD000BB40836007E094F85C30A06D03F01F03E6
:103BE00001FA03F34360206890424DD0A8424BD0C5
:103BF000B04249D0404547D0484545D0504543D0D4
:103C0000584541D02D4A183290423DD02C4A90421E
:103C10003AD02B4A1832904236D0294A303290425C
:103C200032D0274A483290422ED0254A6032904204
:103C30002AD0234A7832904226D0214A90329042AC
:103C400022D01F4AA83290421ED01E4A90421BD05A
:103C50001C4A1432904217D01A4A2832904213D08C
:103C6000184A3C3290420FD0164A503290420BD044
:103C7000144A6432904207D0124A7832904203D0FC
:103C8000104A8C3290420BD1D4E919024260E06EA6
:103C900030B1026822F480720260D4E91C024260F2
:103CA000002084F8351084F834006DE610000240DE
:103CB000580002407000024088000240A00002400C
:103CC00010040240085402582DE9F05F28B190F822
:103CD0003510022904D0802141650120BDE8F09F04
:103CE000904C904B0168183C18338E4ADFF83C9298
:103CF000A1428D4CDFF838E28E4FDFF83CB2DFF89E
:103D00003CA28F4D8F4E31D091422FD099422DD071
:103D1000A1422BD0494529D0714527D0B94225D0A1
:103D2000DFF810C20CF1180C61451FD0DFF808C293
:103D3000ACF1600C614519D0DFF8FCC1ACF1480C66
:103D4000614513D0DFF8F0C1ACF1300C61450DD006
:103D5000DFF8E4C1ACF1180C614507D0594505D036
:103D6000514503D0A94201D0B1422CD1DFF8B4C1F2
:103D70004FF0040880F83580ACF1180C61451DD077
:103D800091421BD0994219D0A14217D0494515D074
:103D9000714513D0B94211D06648183081420DD018
:103DA00065486038814209D063484838814205D06F
:103DB00061483038814201D05F481838086820F0E7
:103DC00001000860ABE0D1F800C02CF00E08DFF86D
:103DD00054C1C1F80080ACF1180C0168614527D0CE
:103DE000914225D0994223D0A14221D049451FD0EC
:103DF00071451DD0B9421BD0DFF838C10CF1180C49
:103E0000614515D0DFF830C1ACF1600C61450FD0D1
:103E1000DFF824C1ACF1480C614509D0DFF818C1C6
:103E2000ACF1300C614503D0DFF80CC1ACF1180CDB
:103E3000D1F800C02CF0010CC1F800C0DFF8E4801C
:103E40004FF0010C0168A8F11808414546D0914295
:103E500044D0994242D0A14240D049453ED071451C
:103E60003CD0B9423AD0334A1832914236D0324A25
:103E7000603A914232D0304A483A91422ED02E4A8E
:103E8000303A91422AD02C4A183A914226D05945CC
:103E900024D0514522D0A94220D0B1421ED02A4A76
:103EA00091421BD0284A1432914217D0264A283218
:103EB000914213D0244A3C3291420FD0224A5032D0
:103EC00091420BD0204A6432914207D01E4A783288
:103ED000914203D01C4A8C32914218D1016E0A687B
:103EE00022F480720A6090F85C20816D02F01F025B
:103EF0000CFA02F24A60D0E919124A60C16E31B17F
:103F00000A6822F480720A60D0E91C124A6000221A
:103F1000016D80F835C080F8342001B18847002059
:103F2000DCE6000028000240580002407000024019
:103F300088000240A0000240700402408804024051
:103F4000A0040240B804024008540258406D704773
:103F50002DE9FC5F0446F74E0020DFF8D88300907F
:103F60004FF41652F44808F11808A56DDFF8C49311
:103F7000DFF8C0A3016809F1300920680AF1480A96
:103F8000B1FBF2F1B04201912F68D5F800C0DFF823
:103F9000ACB335D04146884232D0484530D0504548
:103FA0002ED058452CD0E5491831884228D0E34915
:103FB0003031884224D0E1494831884220D0E0495C
:103FC00088421DD0DE491831884219D0DC49303191
:103FD000884215D0DA494831884211D0DFF860E3D1
:103FE0000EF1600E70450BD0D54A7832904207D062
:103FF000D34B9033984203D0D149A83188427DD128
:1040000094F85C20082102F01F0201FA02F23A4201
:104010004AD0B04232D0404530D048452ED05045ED
:104020002CD058452AD0C54A1832904226D0C34ACF
:104030003032904222D0C14A483290421ED0C04A0B
:1040400090421BD0BE4A1832904217D0BC4A303240
:10405000904213D0BA4A483290420FD0B84A6032E8
:1040600090420BD0B64A7832904207D0B44A903290
:10407000904203D0B24AA832904203D1026802F0C3
:10408000040202E0026802F008026AB1026822F04B
:104090000402026094F85C0000F01F008140A960F7
:1040A000606D40F00100606594F85C00012100F053
:1040B0001F008140394240D02068B04234D0404592
:1040C00032D0484530D050452ED058452CD09B4A50
:1040D0001832904228D0994A3032904224D0974AE0
:1040E0004832904220D0964A90421DD0944A1832CD
:1040F000904219D0924A3032904200E0AFE113D0A2
:104100008F4A483290420FD08D4A603290420BD095
:104110008B4A7832904207D0894A9032904203D03D
:10412000874AA83290427DD1406910F0800F04D0B8
:10413000A960606D40F00200606594F85C000421A5
:1041400000F01F00814039423ED02068B04232D09A
:10415000404530D048452ED050452CD058452AD027
:10416000764A1832904226D0744A3032904222D099
:10417000724A483290421ED0714A90421BD0704A17
:104180001832904217D06E4A3032904213D06C4AA7
:10419000483290420FD06A4A603290420BD0684A4F
:1041A0007832904207D0664A9032904203D0644AF7
:1041B000A83290424ED1006810F0020F04D0A960DE
:1041C000606D40F00400606594F85C00102100F020
:1041D0001F008140394258D02068B04234D0404559
:1041E00032D0484530D050452ED058452CD0534A77
:1041F0001832904228D0514A3032904224D04F4A4F
:104200004832904220D04E4A90421DD04C4A18323B
:10421000904219D04A4A3032904215D0484A48322A
:10422000904200E014E00FD0454A603290420BD03B
:10423000434A7832904207D0414A9032904203D0AC
:104240003F4AA832904207D1006800F0080006E01B
:10425000006872E70068B7E7006800F00400A0B1EA
:10426000A96020680168490304D50068000308D5E7
:10427000A16C07E00168C90503D4016821F00801B9
:104280000160216C09B12046884794F85C00202128
:1042900000F01F008140394279D02068B04232D00E
:1042A000404530D048452ED050452CD058452AD0D6
:1042B000224A1832904226D0204A3032904222D0F0
:1042C0001E4A483290421ED01D4A90421BD01C4AC2
:1042D0001832904217D01A4A3032904213D0184AFE
:1042E000483290420FD0164A603290420BD0144AA6
:1042F0007832904207D0124A9032904203D0104A4E
:10430000A832904203D1006800F0100002E000687B
:1043100000F00200B0B3A96094F8350004282068CA
:1043200001680FD049037ED5006800032BD4616C6F
:104330002AE0000010000240140000247000024037
:104340001004024021F0160101602068416921F04B
:1043500080014161206C08B9A06C20B1206801681F
:1043600021F00801016094F85C303F21012003F046
:104370001F0300229940A96084F8350084F8342096
:10438000216D65E003E0E16B09B120468847606D6F
:1043900000287DD0606DC00759D02068042184F8C2
:1043A0003510B0422BD0404529D0484527D0504544
:1043B00025D0584523D09D49884220D09B491831AB
:1043C00088421CD099493031884218D09849884297
:1043D00015D097491831884211D09549303188421B
:1043E0000DD093494831884209D0914960318842C3
:1043F00005D08F497831884201D08D4990310168CC
:1044000021F00101016020680099019A491C009186
:10441000914202D80168C907F6D10068C00710D0E0
:1044200003200FE0FFE70168C905ACD40368012150
:10443000002223F01003036084F8351084F8342040
:10444000A1E7012084F83500002084F83400E16CF5
:1044500000291DD002B02046BDE8F05F084775492D
:1044600088421DD073491431884219D071492831CE
:10447000884215D06F493C31884211D06D49503186
:1044800088420DD06B496431884209D0694900E007
:1044900084E07831884203D066498C3188427DD1EE
:1044A00094F85C800427016808F01F0807FA08F7F1
:1044B00017EA0C0F009746D04F0744D500980F0419
:1044C000686003D5C8033CD4A16CC1E7880638D422
:1044D0002068B0422DD055496039884229D04845DE
:1044E00027D0504525D0584523D05049884220D068
:1044F0004E49183188421CD04C493031884218D07E
:104500004B49884215D04A491831884211D0484950
:10451000303188420DD046494831884209D0704533
:1045200007D0904205D0984203D04149A831884233
:1045300003D1016821F0080102E0016821F00401C3
:104540000160216C84E7022707FA08F717EA0C0FCD
:1045500000974ED08F074CD500980F04686003D5A4
:10456000C80344D4616C73E7880640D42068B04225
:104570002FD02E49603988422BD0484529D050454C
:1045800027D0584525D02949884222D027491831BB
:1045900088421ED025493031884200E044E018D0DE
:1045A0002349884215D022491831884211D0204928
:1045B000303188420DD01E494831884209D07045BB
:1045C00007D0904205D0984203D01949A8318842BB
:1045D00003D1016821F0140102E0016821F00A0111
:1045E0000160012184F83510002084F83400E16B6B
:1045F0002EE7082202FA08F212EA0C0F14D009077B
:1046000012D5016821F00E01016094F85C100120C0
:10461000002201F01F0100FA01F16960606584F871
:10462000350084F8342012E7BDE8FC9F8800024082
:1046300010040240085402582DE9F05F044601F0CE
:104640006FFA002C07467DD0E24E022120684FF021
:104650000308DFF884934FF00005DFF880A3B04231
:10466000DFF87CB334D0DB4A1832904230D0484572
:104670002ED050452CD058452AD0D94A18329042D5
:1046800026D0D74A3032904222D0D54A4832904282
:104690001ED0D44A90421BD0D24A1832904217D032
:1046A000D04A3032904213D0CE4A483290420FD096
:1046B000CC4A603290420BD0CA4A7832904207D03E
:1046C000C84A9032904203D0C64AA83290427DD167
:1046D00084F83510B04284F834502ED0BD491831DA
:1046E00088422AD0484528D0504526D0584524D065
:1046F000BB491831884220D0B949303188421CD09A
:10470000B7494831884218D0B649884215D0B549D2
:104710001831884211D0B349303188420DD0B149A7
:104720004831884209D0AF496031884205D0AD494F
:104730007831884201D0AB499031016821F0010104
:10474000016008E025E100BF01F0EAF9C01B05287F
:1047500001D920211AE120680068C007F4D1D4E90A
:1047600002032168103418438E4694E88410D4E97B
:10477000033809683A4310439B4A40EA0C006769D2
:1047800018431140103C40EA0800042F40EA0100A1
:1047900003D1D4E90B12114308436168A1F1290246
:1047A000052A0BD9163A032A08D9083A012A05D94D
:1047B000083A032A02D97439032901D840F4801039
:1047C000CEF800002068676A406900E020E0042F0E
:1047D00020F0070047EA00070DD1D4E90A0107439A
:1047E00049B12046FEF768FA28B1402060650121F2
:1047F00084F83510CDE0206847612046FEF77AF94D
:1048000094F85C203F2102F01F029140816055E046
:10481000764A90421BD0754B1433984217D0734B95
:104820002833984213D0714B3C3398420FD06F4BD2
:10483000503398420BD06D4B6433984207D06B4B8A
:104840007833984203D0694B8C3398427ED184F8F8
:10485000351084F83450664B0168A26801EA030EF3
:10486000402A74D0802A73D05FF00002D4E9037824
:10487000D4E9053142EAD70242EAD8085B4AD4E9D2
:10488000077C48EAD30848EAD10141EAD7015242FD
:1048900041EA1C11142341EA0E0101602068104412
:1048A000B0FBF3F08000E0652046FEF723F994F8B2
:1048B0005C20012102F01F02914041602068B0425B
:1048C00057D044491831884253D0484551D05045BB
:1048D0004FD058454DD042491831884249D04049BF
:1048E0003031884245D03E494831884241D03D4927
:1048F00088423ED03B49183188423AD0394930315C
:10490000884236D037494831884232D03549603103
:1049100088422ED03349783188422AD031499031AB
:10492000884226D02F49A831884222D02F49884278
:104930001FD02E49143188421BD02C49283188427F
:1049400017D02A493C31884213D002E01DE017E01D
:1049500018E02649503188420BD0244964318842FE
:1049600007D022497831884203D020498C318842CF
:1049700029D12046FEF718F9A06880280CD00CE059
:10498000102273E74FF4804270E74021616584F89C
:1049900035800120BDE8F09F6560216E20790860B8
:1049A000D4E9190141606068401E072808D82046F4
:1049B000FEF748F9E06E0560D4E91C01416002E0B1
:1049C000E566256765670120656584F83500002088
:1049D000E0E70000100002404000024058000240A2
:1049E00070000240100402403F8010FE085402583C
:1049F0000F00FEFF2DE9F84F04008C464FF0000039
:104A0000009014D094F83400012812D094F8355056
:104A10000120002184F83400012D0CD0C002606513
:104A20000120009084F834100098BDE8F88F012030
:104A3000FBE70220F9E78C4D0226206884F83560F8
:104A4000A8428A4D61658A4E8A4FDFF82C82DFF8D2
:104A50002C92DFF82CA2DFF82CB226D0A84224D06A
:104A6000B04222D0B84220D040451ED048451CD08C
:104A700050451AD0584518D08349884215D08249EC
:104A80001831884211D08049303188420DD07E499A
:104A90004831884209D07C496031884205D07A4942
:104AA0007831884201D078499031016821F00101C4
:104AB000016061462046FEF729F96B49206888426B
:104AC0002CD0A8422AD0B04228D0B84226D04045A7
:104AD00024D0484522D0504520D058451ED06A4A9F
:104AE00090421BD0684A1832904217D0664A303242
:104AF000904213D0644A483290420FD0624A6032EA
:104B000090420BD0604A7832904207D05E4A903291
:104B1000904203D05C4AA83290420CD1026822F045
:104B20001E0242F016020260206C88B12068026802
:104B300042F008020BE0026822F00E0242F00A0284
:104B40000260206C20B12068026842F0040202601A
:104B5000206888424BD0A84249D0B04247D0B842E2
:104B600045D0404543D0484541D050453FD05845B9
:104B70003DD0454A90423AD0434A1832904236D00E
:104B8000414A3032904232D03F4A483290422ED091
:104B90003D4A603290422AD03B4A7832904226D039
:104BA000394A9032904222D0374AA83290421ED0E1
:104BB000364A90421BD0354A1432904217D0334ABD
:104BC0002832904213D0314A3C3290420FD02F4AC3
:104BD000503290420BD02D4A6432904207D02B4A7B
:104BE0007832904203D0294A8C3290420DD1206E07
:104BF0000268D20303D5026842F480720260E06E5C
:104C000018B1026842F4807202602068884226D09F
:104C1000A84224D0B04222D0B84220D040451ED075
:104C200048451CD050451AD0584518D016498842DE
:104C300015D015491831884211D0134930318842B6
:104C40000DD011494831884209D00F49603188425E
:104C500005D00D497831884201D00B499031016867
:104C600041F001010160DFE610000240280002402F
:104C7000400002405800024070000240880002409C
:104C8000A0000240B800024010040240085402583C
:104C900070B5044600F044FF0546601C02D004488D
:104CA0000078044400F03CFF401BA042FAD370BDE2
:104CB0000800002410B590F89830012B09D0022B81
:104CC00007D0D0F89C1041F00201C0F89C100120E0
:104CD00010BD03689C6D0C4203D1DC6D44F00104EF
:104CE00004E09C6D31EA04041FD00324DC658B05CD
:104CF00005D50368D3F8E0401443C3F8E0404B0502
:104D000005D50368D3F8E4401443C3F8E4400068D1
:104D1000084A01EA0203446D074A1C4344651068CF
:104D200040EA91701060002010BDDC6D44F0020478
:104D3000DCE70000FFFFCF3F14A8004070B5044639
:104D400090F89800022804D0D4F89C0040F00800A5
:104D50000DE02068D0F8C03013F07C5F0BD0D0F8A5
:104D6000C4309B020CD5D4F89C0040F40070C4F809
:104D70009C00012070BDD4F89C0040F02000F6E7B4
:104D8000D0F8C400C0F3044520462B46FEF712FBC2
:104D900021680120A840C1F8D000C4F89400002088
:104DA00070BD704770B590F89820012A09D0022A8A
:104DB00007D0D0F89C1041F00201C0F89C100120EF
:104DC00070BD0B68CA6883B10B69072A43EA427356
:104DD00025D00C7A4A6942EA84724968006F00EB78
:104DE000C100C0E90032002070BD072A0DD00C7A46
:104DF000D6060D8A4B6943EA847246EA0543C06EC3
:104E000049681A4340F82120EDE70B8A4FF06055BE
:104E1000D1E9062442EA034245EA0423EFE78A691E
:104E2000DBE730B590F89850039C012D07D0D0F8FF
:104E30009C1041F00401C0F89C10012030BD0D0110
:104E4000016845EA820040EA43002043C1F880003F
:104E5000002030BD10B5FEF7EBFA042808D0054954
:104E600001EB4010C069002802D0BDE810400047A7
:104E700010BD0000F0960024704700000068402933
:104E800005D0D0F8B40000BF00F07F007047D0F824
:104E9000A400F9E7F0B590F898500024022D04D052
:104EA000D0F89C1041F0080129E0402905D04129A3
:104EB00029D0056D8D4219D942E00568D5F8A0606A
:104EC00016F4FE0F12D0D5F8A460760613D0D5F8EC
:104ED000A460F60105D5D5F8A06016F0004F00D506
:104EE0000124D5F8A470466F456C24E0D0F89C10DE
:104EF00041F0200103E0D0F89C1041F48071C0F82B
:104F00009C100120F0BD0568D5F8B06016F4FE0FC6
:104F1000ECD0D5F8B4607606EDD0D5F8B460F601E3
:104F200005D5D5F8B06016F0004F00D50124D5F8AE
:104F3000B470866FC56CC7F305273C44654302E037
:104F4000456DC66F4D4306EB85052E6816F080460D
:104F500056602E6836D026F060461660D5F800C040
:104F600000262E4F0CF0005CC2F808C0D5F800C037
:104F70000CF0004CC2F810C0B5F804C01FFA8CFC4D
:104F8000C2F81CC0D5F804C0CCF3034CC2F80CC066
:104F9000D5F804C00CF4801CC2F814C0D5F804C0C5
:104FA0000CF4001CC2F818C0D5F804C0CCF3066C91
:104FB000C2F820C0D5F804C008354FEADC7CC2F83E
:104FC00024C008E0C6F38A46C7E700BF15F806C04C
:104FD00003F806C0761CD2F80CC017F80CC0B44514
:104FE000F4D840290AD041290CD020294FF00102E1
:104FF0000CD200688A40C0F898200DE00068C0F824
:10500000A84009E00068C0F8B84005E0006801F079
:105010001F018A40C0F89C200020F0BDDCFF000882
:1050200010B590F89820022A04D0D0F89C1041F0D6
:10503000080146E00268D2F8F03013F47C1F37D044
:10504000D2F8F4309B0638D0D2F8F430D0F8802073
:10505000C3F3042302EBC302146814F080444C60D1
:10506000146832D024F060440C60146804F00054DA
:105070008C60146804F000440C619488A4B2CC6184
:105080005468C4F30344CC60546804F480144C6145
:10509000546804F400148C61546804F440044C62B5
:1050A0005268120E0A620068C0F8F830002010BD85
:1050B000D0F89C1041F0200103E0D0F89C1041F49E
:1050C0008071C0F89C10012010BDC4F38A44CBE766
:1050D0000068D0F8C40000F03F007047704700003F
:1050E0002DE9FF5FDFF80CB304460BF10401DBF898
:1050F000000025680F68AA468007D5F85090696DB2
:10510000D5F850806E6D2A6DD5F854C02B6D00EA2D
:105110008770009009F470496F6D286D01EA0901EC
:105120000191DAF85410DAF85490DAF8505008F097
:105130000F0806EA0806029602F0F00203F0715327
:105140006FEA09061F4000F060700CEA020CCDF80F
:105150000CC0F20501EA00090CD4E843C00509D4EB
:1051600000214FF48073CAF85030CBF8001020466D
:10517000FFF7B4FF700512D4E84340050FD4206850
:1051800000234FF48068D0F8DC20D0F8E410C0F899
:105190005080CBF800301140204600F04FFBDFF884
:1051A00058A2009850B12268830F00EA0A001065E7
:1051B000CBF8003020460099FFF7F3FD019850B17D
:1051C0002268830F00EA0A001065CBF80030204601
:1051D000019900F057FB029850B12268830F00EA52
:1051E0000A001065CBF800302046029900F0E2FA80
:1051F000039850B12268830F00EA0A001065CBF8CB
:1052000000302046039900F0E7FA30050CD4E8435B
:10521000000509D4236800204FF400621A65CBF81A
:105220000000204600F040FBB00512D4E8438005A2
:105230000FD4206800234FF40078D0F8D820D0F89D
:10524000E010C0F85080CBF800301140204600F04C
:1052500007FB30030CD4E843000309D42368002083
:105260004FF400221A65CBF80000204600F0A0FAA7
:10527000F0030CD4E843C00309D4236800204FF4A2
:1052800080321A65CBF80000204600F0D5FA700392
:105290000CD4E843400309D4226800204FF4802353
:1052A0001365CBF80000204600F0C5FAB0030FD418
:1052B000E84380030CD4236800204FF400321A65C1
:1052C000CBF80000D4F89C0040F08000C4F89C00AB
:1052D000B9F1000F0BD022684FEA997309EA0A006E
:1052E0001065CBF8003049462046FFF7C5FD5FB199
:1052F0002268BB0F07EA0A001065CBF80030D4F82B
:105300009C003843C4F89C003C492068884268D11E
:10531000606881468068800763D0D9F82060D9F83A
:105320002410D9F82080D9F82400D9F820C0D9F861
:105330002470D9F82030D9F82450D9F8202003F46B
:10534000FC4306F00F0AD9F824601D40D9F824B0B8
:1053500008F030080CF4C07C02F4F02211EA0A01D3
:1053600000EA080807EA0C0706EA0206D9F820A0B6
:1053700004D0C9F82010204600F05AFAB8F1000015
:1053800005D0616808624146204600F053FA6FEA92
:105390000B0040060ED46FEA0A0040060AD460688B
:1053A0004021C36BC26B01622046190C02F03F0220
:1053B00000F03FFA2FB1606807623946204600F0DE
:1053C00036FA35B160680562D4F89C002843C4F809
:1053D0009C0036B160680662D4F89C003043C4F883
:1053E0009C00D4F89C00002802D02046FFF732FD34
:1053F000BDE8FF9F10A80040FFFFCF3F00A0004086
:105400002DE9F04194B08D494C2204466846FBF7E3
:1054100048F964B18A4D2068A84202D100F5807035
:10542000606094F898004FF0000820B108E0012077
:1054300014B0BDE8F081204684F8998000F002F9AC
:105440002068816921F01001816100F069FB032768
:10545000064604E000F064FB801B0A2811D820688F
:1054600080690007F6D42068816941F001018161FB
:1054700000F056FB06460DE000F052FB801B0A28A8
:1054800008D9D4F89C0040F00100C4F89C0084F8CE
:105490009870CCE720688069C007EDD020688169EA
:1054A00041F002018161207C01282068816937D0A8
:1054B00041F040018161607C01282068816932D01F
:1054C00021F480418161A07C0128206881692DD070
:1054D00041F4805181612068A268816921F44071A2
:1054E000114381612068816921F0A40181612068F4
:1054F000016921F010010161E068012819D010B3A1
:1055000002281BD02068816941F0800181612068F8
:10551000016941F010010161E06803280ED012E03A
:1055200021F04001C6E741F48041CBE721F48051EE
:10553000D0E72068816941F0040103E020688169B7
:1055400041F020018161207E6FF0FF02D4E90773F2
:10555000A68A1102400602EB0727A0F1007038432B
:1055600027685B1E184301EB06463043F861A068CC
:10557000B0F5407F11D104F12800A68C6FF00F0C1C
:1055800089C801EB0641401E02EB0322104322684A
:105590000CEB071318430843D060206E30B120682D
:1055A000626ED0F8C0101143C0F8C010D4E91712D1
:1055B0006846D14209D02168A36E51F8C82F50F82F
:1055C000233022F007021A430A60216C49B1216896
:1055D000626C51F8BC3F50F8226023F0070232435E
:1055E0000A60A16C51B12168E36C51F8BC2F50F8EE
:1055F000233022F0700242EA03120A60216D51B199
:105600002168626D51F8BC3F50F8220023F4E0623B
:1056100042EA002008602068A84204D160688168DE
:1056200021F003018160C4F894800121C4F89C80BA
:1056300084F898102046FDF7D9FDF9E6ECFF000844
:1056400000A00040F0B587B0054614216846FBF77E
:1056500084F8514E00244F4B02272D684FF0090C5F
:10566000DFF838E10C3B31684A4A75454C4801F196
:1056700001012AD10129316007D1116841F48071FB
:105680001160116801F480710591196841F00801F9
:105690001960196801F00801059103210091CDE915
:1056A0000174CDE9034C694600F022F9002205217E
:1056B000132000F0E7FA132000F0D7FA00220521AA
:1056C000152000F0DFFA15202EE0DFF8D8E0754550
:1056D0002ED10129316007D1106840F4807010602C
:1056E000106800F480700590186840F0020018609F
:1056F0001868694600F00200059060200090CDE92E
:1057000001742948CDE9034C00F0F2F8002205218C
:10571000142000F0B7FA142000F0A7FA00220521A7
:10572000162000F0AFFA162000F09FFA07B0F0BD87
:10573000DFF878C06545F9D10129316007D11168DA
:1057400041F480711160116801F48071059119684C
:1057500041F0080119601968052201F0080105915E
:105760004FF440510091CDE90174CDE903426946FF
:1057700000F0BEF8002205219F2000F083FA9F2050
:1057800000F073FA00220521A02000F07BFAA0208F
:10579000CAE70000EC4402580400002400A00040C6
:1057A000000C025800A400400004025800D400403D
:1057B0007047000010B5FDF73BFE042808D00549EE
:1057C00001EB4010C068002802D0BDE8104000473F
:1057D00010BD0000F096002410B5FDF729FE042846
:1057E00008D0054901EB40104069002802D0BDE80F
:1057F0001040004710BD0000F096002490F898106B
:10580000012907D0D0F89C1041F00401C0F89C1089
:1058100001207047022180F89810002201688B69EE
:1058200023F001038B61C0F89C201046704770473D
:1058300070477047704770477047000010B5FDF71C
:10584000F7FD042808D0054901EB401080680028C6
:1058500002D0BDE81040004710BD0000F0960024C3
:1058600010B5FDF7E5FD042808D0054901EB40100F
:105870004068002802D0BDE81040004710BD00007D
:10588000F096002410B5FDF7D3FD042808D0054993
:1058900001EB40100068002802D0BDE8104000472E
:1058A00010BD0000F0960024704700002DE9F04183
:1058B000084F01250024064605FA04F0304203D0C3
:1058C00057F8240000B18047641CE4B2102CF3D3D5
:1058D000BDE8F081E8BC00244FF0B04110B5D1F82C
:1058E0008820024203D0C1F88800FFF7DFFF10BD17
:1058F0002DE9F84F03247A4D00234FF001094FF0B2
:10590000B04B4FF00F0AE4E009FA03F6324078D0CA
:105910000F7907F00307012F01D0022F1AD18768F2
:105920004FEA430ED1F80CC004FA0EF827EA080734
:105930000CFA0EFC4CEA070CC0F808C0476891F856
:1059400004C0B743CCF3001C0CFA03FC4CEA070C70
:10595000C0F804C00E79F643B6070BD0C6684FEA0C
:1059600043088F6804FA08FC26EA0C0607FA08F7D1
:105970003743C7600E7906F00306022E12D1DE0807
:105980000F694FEA437C00EB8606B646366A4FEA5B
:10599000DC6C0AFA0CF807FA0CF726EA080637431B
:1059A000CEF820700F7906684FEA430807F0030726
:1059B00004FA08FC07FA08F726EA0C0637430760E2
:1059C0004E6816F4403F1CD0464E376847F0020739
:1059D000376036689F0706F00206009623F003063C
:1059E00006F1B046B6463F0FD6F80864DFF8F880F7
:1059F0000AFA07FC404526EA0C0603D14FF0000CDA
:105A00003AE065E0DFF8E4C0604502D14FF0010CF8
:105A100032E0DFF8DCC0604502D14FF0020C2BE031
:105A2000DFF8D0C0604502D14FF0030C24E0DFF86E
:105A3000C8C0604502D14FF0040C1DE0DFF8BCC0C7
:105A4000604502D14FF0050C16E0DFF8B4C06045A8
:105A500002D14FF0060C0FE0DFF8A8C0604502D17C
:105A60004FF0070C08E0DFF8A0C0604502D14FF00E
:105A7000090C01E04FF00A0C0CFA07FC4CEA060C8A
:105A8000CEF808C44F68DBF80060FF0226EA020681
:105A900000D516435F46CBF80060D1F804C0DBF8B0
:105AA00004605FEA8C2C26EA020600D516437E606D
:105AB0006E684F6826EA0206BF0300D516436E6083
:105AC0002E684F6826EA0206FF0300D516432E60B3
:105AD0005B1C0A6832FA03F67FF416AFBDE8F88F54
:105AE00080000058F4440258000002580004025894
:105AF00000080258000C0258001002580014025806
:105B000000180258001C025800240258006908407E
:105B100000D0012070470AB1816170470904FBE79A
:105B2000014880687047000008000024024881682E
:105B3000027811448160704708000024032010B5EA
:105B400000F0C0F801F090F80F4A1049146813688B
:105B5000C4F3032203F00F038A5CC95C02F01F0246
:105B600001F01F01D0400A4A20FA01F111600949F1
:105B700008600F2000F010F808B1012010BD00F0FF
:105B800051F8002010BD00001844025860000108C0
:105B9000180000241400002410B5102804468AB010
:105BA0002DD2002201461C2000F06CF81C2000F0D1
:105BB0005CF8184804601848016841F00101016070
:105BC000006809A900F001000890684600F0D8FFBD
:105BD0000598B8B101F024F840001049002240F2C5
:105BE000E733B0FBF1F10E484FF080440460C0E9A8
:105BF0000332491EC0E9011202F0DAFA28B101208D
:105C00000AB010BD01F00CF8E7E7054802F022FBEE
:105C1000F6E700000C000024E844025840420F0060
:105C2000D0090024074882B0016841F002010160F8
:105C3000006800220F2100F002000090901E02B0C8
:105C400000F020B8F444025800280DDB410900F0B0
:105C50001F028900012001F1E0219040C1F880017C
:105C6000BFF34F8FBFF36F8F7047002809DB4109E7
:105C700000F01F028900012001F1E0219040C1F8ED
:105C8000000170470E4BF0B41B680D46C3F30223AE
:105C9000C3F10706042E00D90426191D072901D2D5
:105CA000002300E0DB1E012404FA06F19C40491E9B
:105CB0002940641E994014402143F0BC06F081BE87
:105CC0000CED00E0064900F0070210B54FF6FF04A6
:105CD0000868044B204040EA02201843086010BDC9
:105CE0000CED00E00000FA05134970B50A68D243D4
:105CF000520705D5096801F00701814213D118E068
:105D00000A6822F0070202430A60FFF709FF0A4D02
:105D10004FF47A760446083D07E000BFFFF700FF26
:105D2000001BB04201D9012070BD2868C043800427
:105D3000F4D4002070BD00000C48025810B500F0EB
:105D40004DFF05490968054AC1F30211515C01F094
:105D50001F01C84010BD0000204402586000010827
:105D6000494930B5484C0B1D0A68143409681D6850
:105D7000246802F00303C5F30012C1F30531C4F334
:105D8000CC04002914FB02F200EE102AF8EE400ABF
:105D900075D03F4A9FED3D1AB7EE000A6BB1DFEDBB
:105DA0003D1A012B01D0022B64D002EE101A1168AB
:105DB000F8EE422A81EEA22A21E0334C283C2368E7
:105DC0009B0612D5344B246801EE901A1168C4F377
:105DD000C104F8EE612AE34001EE903AC1F30801F4
:105DE000F8EE611A81EEA22A0BE001EE901ADFEDC7
:105DF0002B2A00BFF8EE611A116882EEA12AC1F3C6
:105E0000080101EE901A1168F8EE611A40EE811A4D
:105E100071EE800A62EE200AC1F3462101EE101AEB
:105E2000B8EE411A31EE001AC0EE811ABCEEE11A4A
:105E300080ED001A1168C1F3064101EE101AB8EEA8
:105E4000411A31EE001AC0EE811ABCEEE11A80ED63
:105E5000011A1168C1F3066101EE101AB8EE411A79
:105E600031EE000A80EE801ABCEEC10A80ED020A13
:105E700030BD04E001EE901ADFED092ABAE70021F7
:105E8000016041608160F3E7284402580000003956
:105E9000384402580024744A0090D0030024744C03
:105EA000001BB74B494930B5484C0B1D0A681C34E0
:105EB00009681D68246802F00303C5F30022C1F3DA
:105EC0000551C4F3CC04002914FB02F200EE102AA1
:105ED000F8EE400A75D03F4A9FED3D1AB7EE000A32
:105EE0006BB1DFED3D1A012B01D0022B64D002EE25
:105EF000101A1168F8EE422A81EEA22A21E0334CF2
:105F0000283C23689B0612D5344B246801EE901A76
:105F10001168C4F3C104F8EE612AE34001EE903A3F
:105F2000C1F30801F8EE611A81EEA22A0BE001EE3E
:105F3000901ADFED2B2A00BFF8EE611A116882EE8D
:105F4000A12AC1F3080101EE901A1168F8EE611A56
:105F500040EE811A71EE800A62EE200AC1F34621FA
:105F600001EE101AB8EE411A31EE001AC0EE811A95
:105F7000BCEEE11A80ED001A1168C1F3064101EE92
:105F8000101AB8EE411A31EE001AC0EE811ABCEEBA
:105F9000E11A80ED011A1168C1F3066101EE101AD1
:105FA000B8EE411A31EE000A80EE801ABCEEC10A4A
:105FB00080ED020A30BD04E001EE901ADFED092AFF
:105FC000BAE70021016041608160F3E7284402588C
:105FD00000000039404402580024744A0090D00365
:105FE0000024744C001BB74B2DE9FE4F0546DFF82B
:105FF00000A450F8081B0024FD4FC943019005F18F
:10600000280026460AF1240A009008011DD4686E73
:1060100050B1B0F5801F0CD0B0F5001F0ED0B0F518
:10602000401F1ED001240FE0386840F40030386073
:1060300017E00198022104F03DF903E000980221E5
:1060400004F0C8F904000CD026462888C043C005D7
:1060500023D4A86D05281ED2DFE800F00C11161B12
:106060001B006A6EDAF8001021F440111143CAF8DF
:106070000010EAE7386840F40030386009E0019821
:10608000002104F017F903E00098002104F0A2F9C0
:106090000446C4B100E0012426462888DFF8508376
:1060A000C04308F12C0840052FD4D5F8A400B0F562
:1060B000C00F28D010DCB8B1B0F5001F19D0B0F572
:1060C000800F0FD11AE0AA6DDAF8001021F0070155
:1060D0001143CAF80010E0E7B0F5000F13D0B0F597
:1060E000200F10D001240FE0386840F400303860F1
:1060F00009E00198002104F0DDF803E00098002198
:1061000004F068F9044694B126462888C043000587
:1061100030D4D5F8A800B0F1407F29D011DCC0B14F
:10612000B0F1807F1AD0B0F1007F10D11BE0D5F81C
:10613000A420D8F8001021F460011143C8F8001021
:10614000E3E7B0F1806F13D0B0F1A06F10D001245D
:106150000FE0386840F40030386009E00198002111
:1061600004F0A8F803E00098002104F033F9044695
:1061700094B126462868DFF878B2C0430BF1200BB3
:1061800080011FD4E86CD8B110280FD0202812D07D
:10619000302815D0012414E0D5F8A820D8F8001034
:1061A00021F0E0611143C8F80010E3E7386840F4DB
:1061B0000030386004E00198022104F07BF80446C6
:1061C00074B126462888C043C0042BD4E86DB0F5CE
:1061D000005F20D00DDCA0B1B0F5805F0FD115E0DD
:1061E000EA6CDBF8001021F030011143CBF800100D
:1061F000E8E7B0F5405F13D0B0F5804F10D0012430
:106200000FE0386840F40030386009E00198002160
:1062100004F050F803E00098002104F0DBF8044695
:106220008CB126462888C043800429D4286EB0F556
:10623000403F23D010DC08B3B0F5803F14D0B0F558
:10624000003F0FD115E0EA6DDAF8001021F4E041CB
:106250001143CAF80010E5E7B0F5802F0ED0B0F575
:10626000A02F0BD001240AE00198012104F022F8AC
:1062700003E00098012104F0ADF8044694B12646ED
:106280002888C04340042AD4D5F8AC00B0F1405F60
:1062900023D010DC08B3B0F1805F14D0B0F1005F00
:1062A0000FD115E02A6EDAF8001021F4E021114335
:1062B000CAF80010E4E7B0F1804F0ED0B0F1A04F63
:1062C0000BD001240AE00198012103F0F3FF03E061
:1062D0000098012104F07EF8044674B1264628880F
:1062E000C04300041FD4E86ED8B1B0F1805F0ED077
:1062F000B0F1005F10D0012414E0D5F8AC20D8F83C
:10630000001021F0E0411143C8F80010E7E73868B9
:1063100040F40030386004E00198012103F0CAFF26
:10632000044674B126462868C043C0011ED4A86C38
:10633000D0B101280ED0022811D0032814D0012496
:1063400013E0EA6EDAF8001021F040511143CAF868
:106350000010E8E7386840F40030386004E0019845
:10636000022103F0A7FF04466CB126462868C0430B
:10637000400255D41F48016841F480710160FFF765
:10638000CFFB81460EE0AA6CDBF8001021F0030180
:106390001143CBF80010E9E7FFF7C2FBA0EB0900BF
:1063A00064283BD813480068C005F5D5BCBBDFF8AE
:1063B0004090B5F8B01009F14409D9F8000001F493
:1063C000407100F44070884211D0D9F80010D9F81B
:1063D000002021F4407142F48032C9F80020D9F83D
:1063E000002022F48032C9F80020C9F8001003E030
:1063F0002C44025800480258D5F8B000B0F5807F10
:1064000019D1FFF78DFB029011E000BFFFF788FB69
:106410000299411A41F28830814208D90324264664
:106420002878DFF81494C043C00721D03CE0D9F8A5
:1064300000008007EAD5D5F8B010C1F30120032889
:10644000FE480DD0016821F47C510160B5F8B02000
:10645000D9F80010C2F30B021143C9F80010DFE7AE
:10646000F74A036802EA111223F47C511143ECE766
:10647000A86F182816D005DCA0B1082808D010286D
:1064800004D10AE020280DD028280BD001240AE0EE
:106490000198012103F00EFF03E00098012103F0B1
:1064A00099FF044664B126462878C04380071ED46D
:1064B000686F062819D2DFE800F0160C11161616C0
:1064C000AA6FD9F8001021F038011143C9F8001063
:1064D000EAE70198012103F0EDFE03E000980121B5
:1064E00003F078FF04467CB100E0012426462878BA
:1064F000C04340071FD4D5F89000062819D2DFE822
:1065000000F0160C111616166A6FD9F8001021F05B
:1065100007011143C9F80010E9E70198012103F0D0
:10652000C9FE03E00098012103F054FF0446A4B122
:1065300000E0012426462878C04380062BD4D5F8F5
:106540008C00B0F1405F24D011DC10B3B0F1805F5B
:1065500015D0B0F1005F10D116E0D5F89020D8F832
:10656000001021F007011143C8F80010E3E7B0F173
:10657000804F0ED0B0F1A04F0BD001240AE001985B
:10658000002103F097FE03E00098022103F022FFB0
:10659000044694B126462878C04340062BD4D5F84B
:1065A0009800B0F5406F24D011DC10B3B0F5806FC7
:1065B00015D0B0F5006F10D116E0D5F88C20D9F8C1
:1065C000001021F0E0411143C9F80010E3E7B0F5F5
:1065D000805F0ED0B0F5A05F0BD001240AE00198D7
:1065E000002103F067FE03E00098022103F0F2FEB1
:1065F000044694B126462878C04300062BD4D5F82B
:106600009C00B0F5C04F24D011DC10B3B0F5005F92
:1066100015D0B0F5804F10D116E0D5F89820D8F8F5
:10662000001021F4E0511143C8F80010E3E7B0F581
:10663000004F0ED0B0F5204F0BD001240AE0019896
:10664000002103F037FE03E00098022103F0C2FEB0
:10665000044654B126462878C04300071ED4D5F816
:106660008000B0F5805F0AD00FE0D5F89C20D8F804
:10667000001021F460411143C8F80010EBE70098C6
:10668000022103F0A7FE00B10126D5F88020D9F839
:10669000001021F440511143C9F800102878C0437C
:1066A000C00613D4D5F89400B0F5807F05D10098CA
:1066B000022103F08FFE00B10126D5F89420D8F80E
:1066C000001021F440711143C8F800102868C0433D
:1066D000000316D4D5F8A00038B1B0F5803F09D03A
:1066E000B0F5003F0BD001240AE00198002103F02F
:1066F000E1FD03E00098022103F06CFE04468CB13A
:1067000026462868C043400322D4D5F88400B0F55B
:10671000801F11D0B0F5001F13D0B0F5401F15D069
:10672000012414E0D5F8A020D8F8001021F440315D
:106730001143C8F80010E4E7386840F400303860CE
:1067400004E00098012103F045FE04465CB12646B2
:106750002868C043C0031CD4286D70B1B0F5803FD9
:1067600010D0012414E0D5F88420D9F8001021F4C9
:1067700040111143C9F80010EAE7386840F40030CE
:10678000386004E00198022103F094FD0446DCB176
:1067900026462868C043800005D40098022103F0F3
:1067A00019FE00B101262868C04380031BD4E86F9E
:1067B000B8B1B0F5807F10D0B0F5007F11D0B0F542
:1067C000407F0ED001240DE02A6DDBF8001021F48B
:1067D00080311143CBF80010DBE7386840F400301B
:1067E00038607CB326462868C043C00207D42A6FAD
:1067F000DAF8001021F000411143CAF800102868AF
:10680000C043800207D4AA6EDAF8001021F080712C
:106810001143CAF800102868C043400009D4074853
:10682000016821F4004101600168D5F8B4201143EA
:1068300001602868C04306E05444025810440258DE
:10684000CFFFFF001DE007D46A6DDBF8001021F0D8
:1068500040511143CBF800102868C043000208D40F
:10686000D5F88820D9F8001021F440011143C9F867
:10687000001028790024C04300F00100204309D013
:106880000EE0EA6FD9F8001021F440711143C9F805
:106890000010A8E70198002103F00CFD00B10646A6
:1068A0002879C04300F00200204305D1019801215E
:1068B00003F000FD00B106462879C04300F0040053
:1068C000204305D10198022103F0F4FC00B10646F3
:1068D0002879C04300F00800204305D1009800212A
:1068E00003F078FD00B106462879C04300F010009F
:1068F000204305D10098012103F06CFD00B106464C
:106900002879C04300F02000044304D100980221FC
:1069100003F060FD00B916B10120BDE8FE8F002034
:10692000FBE700002DE9F05F04000F467ED0DFF8A2
:106930003882D8F8000000F00F00B8420CD2D8F826
:10694000001021F00F013943C8F80010D8F80000FA
:1069500000F00F00B84269D12078844D40070AD575
:106960002069296801F07001884204D9296821F062
:1069700070010143296020787C4E361D00070AD53E
:106980006069316801F07001884204D9316821F0F2
:106990007001014331602078C0060AD5A0693168D2
:1069A00001F4E061884204D9316821F4E0610143D7
:1069B00031602078DFF8B4B180060BF1080B0CD5FC
:1069C000E1695846DBF8002002F07002914204D9D8
:1069D000026822F070020A430260207880070AD51C
:1069E000E068296801F00F01884204D9296821F084
:1069F0000F01014329602078C0073ED05B49A2689F
:106A00002868183920F470601043286060680228F4
:106A100018D0032819D00968012819D0490700297E
:106A20004ADADFF848A1AAF1080A00E044E0DAF8FF
:106A3000002022F007020243CAF80020FFF770F896
:106A4000814612E009688903E9E709688901E6E7F8
:106A5000C905E4E7FFF764F8A0EB090141F28830CB
:106A6000814202D90320BDE8F09F6168DAF8000096
:106A700000F03800B0EBC10FECD1207880070AD5C8
:106A8000E068296801F00F01884204D2296821F0EA
:106A90000F0101432960D8F80010404601F00F01B2
:106AA000B9420BD9016821F00F0139430160006838
:106AB00000F00F00B84201D00120D4E72078400751
:106AC0000AD52069296801F07001884204D229683A
:106AD00021F0700101432960207800070AD5606920
:106AE000316801F07001884204D2316821F07001F0
:106AF000014331602078C0060AD5A069316801F4ED
:106B0000E061884204D2316821F4E06101433160E0
:106B1000207880060CD5E1695846DBF8002002F0A9
:106B20007002914204D2026822F070020A430260AD
:106B300000F09AF80E492A682B68C2F3032203F08A
:106B40000F038A5CC95C02F01F0201F01F01D040F4
:106B5000084A20FA01F111600749086007480068F7
:106B6000BDE8F05FFFF718B8002000521844025843
:106B70006000010818000024140000240C00002408
:106B800070B5144C3F220260124A24680832131D6B
:106B9000114D04F00704446016681C1D06F470666D
:106BA0008660166806F00F06C660126802F0700272
:106BB00002611A6802F0700242611A6802F4E0622F
:106BC0008261226802F07002C261286800F00F0042
:106BD000086070BD104402580020005230B500F02B
:106BE00043F80B4A0B490C4B15681468C5F3032294
:106BF00004F00F048A5C095D02F01F0201F01F011E
:106C0000D040064A20FA01F119601060084630BDF4
:106C100018440258600001081800002414000024E1
:106C200000B5FFF7DBFF05490968054AC1F302110A
:106C3000515C01F01F01C84000BD00001C44025817
:106C40006000010800B5FFF7C9FF05490968054A5A
:106C5000C1F30221515C01F01F01C84000BD0000DA
:106C60001C44025860000108454970B54548096850
:106C7000434B103B11F0380208D00111082A03D011
:106C8000102A0BD0182A0BD0084670BD1968890647
:106C9000FBD51968C1F3C101C84070BD3A4870BD49
:106CA0003749374D18310C1D24350A6809682668A4
:106CB0002D6802F0030406F00102C1F30511C5F3CB
:106CC000CC0515FB02F200EE102AB8EE400AE9B33B
:106CD0002F4ADFED2E0AB7EE001A6CB1DFED2D1A48
:106CE000012C01D0022C43D002EE101A1068F8EEED
:106CF000422A81EEA22A1EE01C68A40611D51B6858
:106D000001EE901A1168C3F3C103F8EE612AD8406E
:106D100001EE900AC1F30800F8EE611A81EEA22A92
:106D20000BE001EE901ADFED1C2A00BFF8EE611AAD
:106D3000106882EEA12AC0F3080001EE900AF8EE76
:106D4000611A40EE201A31EE810A00E015E022EED1
:106D5000000A1068C0F34620401C00EE900AF8EECE
:106D6000600A80EE201ABCEEC10A10EE100A70BD57
:106D700001EE901ADFED092AD8E7002070BD00006F
:106D8000104402580090D00300366E010000003914
:106D9000304402580024744A0024744C001BB74B42
:106DA0002DE9F05F04007DD0FF4F2078FE4D1837AD
:106DB000DFF8F483103DC00748D0D8F800003968E8
:106DC00000F03800102815D0182803D101F0030076
:106DD00002280FD06068B0F5803F12D010B1B0F536
:106DE000A02F18D0286820F480302860286820F46C
:106DF000802009E02868800328D560680028D2D068
:106E000024E0286840F480302860606888B1FEF78C
:106E100087FE064609E0286840F480202860F0E7F5
:106E2000FEF77EFE801B64287ED828688003F7D595
:106E30000CE0FEF775FE064605E000BFFEF770FEAB
:106E4000801B6428F0D828688003F7D42078800756
:106E500056D5D8F80000DFF85093396810F03800A4
:106E6000A9F10C090ED0182801D188070AD0E068D2
:106E7000A8B3296821F0190101432960FEF750FEEB
:106E8000064628E02868400702D5E06800288AD036
:106E9000E168286820F0190008432860FEF740FEEA
:106EA000064606E0D2E000BFFEF73AFE801B02284D
:106EB000BAD828684007F7D5217CD9F8002022F0FD
:106EC000FE4242EA0161C9F8001019E0FEF728FE0F
:106ED000801B0228A8D828684007F7D5ECE7FFE711
:106EE000286820F001002860FEF71AFE064604E03C
:106EF000FEF716FE801B022896D828684007F7D4B4
:106F00002078C00646D5D8F80000DFF89C92396892
:106F100000F03800A9F10409082812D0182805D17A
:106F200001F00300012800E0CEE00AD0E06900286B
:106F3000286820D040F080002860FEF7F1FD06466A
:106F400015E02868C00502D5E06980287ED194F854
:106F50002010D9F8002022F07C5242EA0161C9F8E1
:106F6000001017E0FEF7DCFD801B0228A0D828687F
:106F7000C005F7D5EBE720F080002860FEF7D0FDD4
:106F8000064604E0FEF7CCFD801B022890D8286856
:106F9000C005F7D42078000729D58348616964309B
:106FA00000298146016811D041F001010160FEF71E
:106FB000B7FD064605E000BFFEF7B2FD801B0228C4
:106FC00088D8D9F800008007F6D510E021F001013B
:106FD0000160FEF7A5FD064605E000BFFEF7A0FD37
:106FE000801B022870D8D9F800008007F6D42078DA
:106FF000800623D5A0690028286810D040F480506E
:107000002860FEF78DFD064605E000BFFEF788FD0F
:10701000801B022858D828688004F7D50EE020F499
:1070200080502860FEF77CFD064604E0FEF778FD00
:10703000801B022848D828688004F7D420784007AD
:1070400051D5DFF86891D9F8001000E015E141F45E
:107050008071C9F80010FEF763FD064605E000BF29
:10706000FEF75EFD801B64282ED8D9F80000C0050D
:10707000F6D54D4EA068603601280AD008B1052823
:1070800013D0306820F001003060306820F0040038
:1070900002E0306840F001003060A06841F2883AB8
:1070A00098B1FEF73DFD81460AE0306840F00400EB
:1070B0003060EEE7FEF734FDA0EB0901514503D83F
:1070C00030688007F6D50EE072E0FEF729FD8146B4
:1070D00006E000BFFEF724FDA0EB0901514567D88B
:1070E00030688007F6D4606A00287CD0DFF8B8A04A
:1070F000D8F800100AF1200A4FF6F87B0AF10408CC
:10710000C1F3C2010329AAF104096DD0022828683D
:1071100020F08070286003D0FEF702FD044681E075
:10712000FEF7FEFC064604E0FEF7FAFC801B022890
:1071300075D828688001F7D4E26A40F2F3313868E4
:1071400054F8283F884340EA021018433860217BF6
:107150004FF4FE0C22894FF0FE47208A4902267D1B
:10716000521E401EA1F5007189B2C2F308021143FC
:10717000761E0CEA00400143484607EA06621143C6
:10718000CAF80010D9F8001021F00101C9F8001068
:10719000D8F80030266A23EA0B0343EAC601C8F890
:1071A0000010D9F8001004E01044025800480258BA
:1071B00035E0A26921F00C011143C9F80010016803
:1071C000E26921F0020111430160016841F480315C
:1071D0000160016841F400310160016841F48021DF
:1071E0000160016801E06CE020E041F00101016014
:1071F000286840F080702860FEF792FC044604E0A6
:10720000FEF78EFC001B022809D828688001F7D5FC
:1072100057E000BFFEF784FC001B022802D90320C0
:10722000BDE8F09F28688001F4D44AE0396801285D
:10723000DAF8000021D0A26A01F0030393421CD1C6
:10724000E26AC1F305118A4217D1216BC0F308022B
:10725000491E8A4211D1616BC0F34622491E9142F8
:107260000BD1A16BC0F30642491E914205D1E16BDF
:10727000C0F30660491E814201D00120D0E7A16C15
:107280004646D8F80000C0F3CC00814219D0D9F8A6
:1072900000004D4620F00100C9F80000FEF740FC58
:1072A0004FEA0007FEF73CFCB842FBD0A26C306806
:1072B00020EA0B0040EAC2003060286840F001007C
:1072C00028600020ACE7000070B5044603F0CCF95C
:1072D000032811D0204603F0C7F9084D05EB4010F4
:1072E0008069002808D0204603F0BEF905EB401065
:1072F0008069BDE87040004770BD000028BD0024D3
:107300002DE9F04704460068002103694269876857
:1073100094F8816000F130095FEA025C03EA02053B
:107320000AD51A0708D5816941F4006181612046B8
:1073300000F0AEFCBDE8F08715F0600F08D16807DB
:1073400006D5616F20468847216F20468847012176
:1073500005F04100012805D1680703D4216F2046BC
:107360008847012105F02200022806D1680704D4CD
:10737000616F2046BDE8F04708470029DAD12807A9
:107380004FF001085BD52068816941F008018161F7
:107390002068816941F0100181612068816941F4B0
:1073A000006181612068016921F0080101612068A4
:1073B000806810F4404F20D023E0E0680F2806D901
:1073C0002068616E006B0860606E001D0FE007288A
:1073D00006D9B9F80000616E0880606E801C06E076
:1073E0002068616E90F830000870606E401C606626
:1073F000B4F86A00401EA4F86A00B4F86A000028D5
:10740000DBD1204603F07CF884F88180D4F8840036
:1074100018B12046FFF758FF8CE7052E07D0042E41
:1074200009D0032E86D1204600F010FE82E72046C8
:1074300000F03AFE7EE7204600F0F2FB7AE715F412
:10744000587FE9D068060AD5D4F8840040F00400DB
:10745000C4F884002068816941F040018161A80579
:107460000AD5D4F8840040F00100C4F884002068F4
:10747000816941F400718161E8050AD5D4F884007E
:1074800040F00800C4F884002068816941F48071EC
:107490008161A8060AD5D4F8840040F08000C4F8C1
:1074A00084002068816941F020018161D4F8840062
:1074B0000028B1D0206840F26B32C7F381310368F5
:1074C000032923F0010101602068016921EA02011A
:1074D000016102D084F881809BE72068104D8168AB
:1074E00021F440418160E06F50B10565E06FFCF729
:1074F000EBFB28B1D4F8840040F04000C4F88400CD
:10750000A06F002888D00565A06FFCF7DDFB002880
:107510008CD0D4F8840040F04000C4F8840009E71F
:10752000BDA500082DE9F047040029D0594A4FF0C5
:1075300000092068584B594D9042C4F8289006D055
:10754000984204D0A84202D0E1680F2918D8E16817
:107550004FF0010AE76B0831C9080AEB571671436F
:10756000904205D0984203D0A84201D0082907D8FC
:10757000904203D0984201D0A84204D1102902D9E8
:107580000120BDE8F08794F8810020B9204684F8F6
:10759000809000F085F8022084F88100206801685E
:1075A00021F0010101602068A1698268B1F1806F5A
:1075B00002F4F81110D16268B2F5800F01D01AB14F
:1075C0000AE0A26B22B107E0A26BB2F1805F03D1A7
:1075D000026842F4805202606068400209D5E068A7
:1075E000072806D32068236D026822F480721A43AC
:1075F00003E02068026822F480720260A66AE069F3
:10760000E26B25683043E3680A4310431843A860DF
:10761000D4E90D02D4E90581636A25691843D4F8D9
:1076200020C00A43266810432843A56DD4E901729F
:10763000D4E9123140EA080040EA0C00384308431C
:10764000104318432843F060606868B92068816877
:1076500021F4C05141F4006181602068816821F407
:10766000C06141F4806181602068016D21F00101F9
:1076700001656068400206D52068626DC16821F02E
:1076800000411143C160C4F8849084F881A00020B7
:1076900077E700000030014000380040003C004027
:1076A0002DE9F041B4B0074614212EA8F9F755F89A
:1076B000B8216846F9F751F8534902263868002482
:1076C000524D884273D1811417940020CDE90010E7
:1076D0006846FEF789FC08B1FBF753FD4B480830BC
:1076E000016841F480410160006800F480403390FB
:1076F000286840F004002860286800F004003390F7
:10770000286840F0020028602868B046032500F091
:10771000020006210526CDE92E18CDE932603C484D
:107720002EA9CDE93045FEF7E3F84FF40051394872
:1077300030AACDE92E182EA982E87000FEF7D8F8FD
:10774000354E272235494FF48068304686E81600CA
:10775000C6E903487461B461F46134627462FCF791
:107760006BFF08B1FBF70DFD2B4D28222B49402361
:107770007835FE671831B763284685E81E016C61CD
:10778000AC61EC612C626C62FCF756FF08B1FBF750
:10779000F8FCBD6700220521AF632420FEF772FAD2
:1077A0002420FEF762FA34B0BDE8F081FFE71C49FF
:1077B0008842F8D100202B944FF48041CDE900108D
:1077C0006846FEF711FC08B1FBF7DBFC0F481430EC
:1077D000016841F020010160006800F02000339052
:1077E000286840F0010028602868082100F00100A6
:1077F0003390A0202E90CDE92F64CDE93141094886
:107800002EA9FEF775F8CEE700380040E044025894
:1078100000080258000402583C07002410000240EF
:1078200000140058000002582DE9F84F8946C16B3A
:10783000044600689A4616464909491C1FFA81F811
:1078400030300090FEF76CF9834694F881000128EF
:1078500038D1B9F1000F6FD0002EFCD094F8800021
:1078600001282FD0A1680025012784F8807004200A
:1078700084F88100C4F88450C4F86490E565A4F8E5
:107880006050256765672C34B1F5C02FA687E68761
:10789000E58654F82C0D18D0C16821F4C02141F4BC
:1078A0008021C160206841686FF30F01314341605E
:1078B0002068016841F0010101606068B0F5800F47
:1078C00008D00CE00220BDE8F88F016821F40061C7
:1078D0000160E7E72068016841F400710160E06839
:1078E0000F2824D829E0206841694269D20705D1D0
:1078F000B4F86A3043450DD209040BD5006B616EB4
:107900000860606E001D6066B4F86A00401EA4F84E
:107910006A000CE0FEF704F9A0EB0B01514503D31C
:10792000BAF1FF3F03D0AAE0BAF1000F40D0B4F89B
:107930006A000028D7D194E09FE007283CD88CE06B
:10794000216848694969C9070AD000980088616EB2
:107950000880606E801C6066B4F86A00401E15E006
:10796000B4F86A20424514D2010412D50098008868
:10797000616E0880606E801C6066009909880180D5
:10798000606E801C6066B4F86A00801EA4F86A000D
:1079900012E0B4F86A10012901D18004D5D4FEF7B1
:1079A000BFF8A0EB0B01514503D3BAF1FF3F03D061
:1079B00065E0BAF1000F62D0B4F86A000028BFD1C8
:1079C0004FE0206841694269D2070AD090F8300040
:1079D000616E0870606E401C6066B4F86A00401EFC
:1079E00024E0B4F86A30434523D20A0421D590F844
:1079F0003000616E0870606E401C6066216891F80E
:107A000030100170606E401C6066216891F8301083
:107A10000170606E401C6066216891F83010017042
:107A2000606E401C6066B4F86A00001FA4F86A002B
:107A300013E0B4F86A20042A02D211F4C04FC5D171
:107A4000FEF76EF8A0EB0B01514503D3BAF1FF3FEF
:107A500003D014E0BAF1000F11D0B4F86A00002886
:107A6000AFD1204602F04CFD84F88170D4F8840038
:107A700084F8805000283FF426AF012023E72046F9
:107A800002F03EFDD4F8840084F8805040F4807009
:107A9000C4F8840084F88170032014E72DE9F041D4
:107AA000044690F8810016460025012802D084F88B
:107AB00080502FE059B356B394F88000012829D0A4
:107AC000A268012784F88070042084F88100C4F83B
:107AD0008450256765676166A4F860502C34B2F560
:107AE000C02FA687E687E58654F82C0D15D0C1680F
:107AF00021F4C02141F48021C0F80C10E0684FF45B
:107B000080410F280ED9E26F92698A420AD084F828
:107B1000805055E00220BDE8F081016821F4006149
:107B20000160EBE707284FF4005205D9E06F806948
:107B3000904201D08842EAD12068836823F48043D0
:107B40008360E068072811D8E06F8369934205D10C
:107B5000B4F86A20521C5208A4F86A20806988424E
:107B600010D1B4F86A00C01C800809E00F2809D8B9
:107B7000E06F8069884205D1B4F86A00401C400873
:107B8000A4F86A00E06F23490164E16F2248C863EA
:107B9000E16F2248C864E06F0565B4F86A30216877
:107BA000626EE06F3031FCF725FF58B1D4F88400E5
:107BB00084F8805040F01000C4F8840084F881708C
:107BC0000120A8E7E06FC069B0F5807F20684168B8
:107BD0006FF30F0100D0314341602068816841F4A8
:107BE000804181602068016941F450710161206821
:107BF000016841F0010101606068B0F5800F04D1B7
:107C00002068016841F400710160002084F8805010
:107C100081E7000003A6000817A60008D7A5000802
:107C200070B5044602F020FD032811D0204602F072
:107C30001BFD084D05EB40104068002808D0204689
:107C400002F012FD05EB40104068BDE870400047AF
:107C500070BD000028BD002470B5044602F004FD8C
:107C6000032811D0204602F0FFFC084D05EB401020
:107C70000069002808D0204602F0F6FC05EB401011
:107C80000069BDE87040004770BD000028BD0024B9
:107C900070472DE9F84F044600689946174600F1F1
:107CA000200B8A46FDF73CFF064694F88100012828
:107CB00039D1BAF1000F7ED0002FFCD094F88000AB
:107CC000012830D0A26800254FF0010884F8808098
:107CD000032184F88110C4F88450C4F85CA0656660
:107CE000A4F86850656725672C34B2F5C02FA786C5
:107CF000E786E58754F82C0D18D0C16821F4C0211F
:107D000041F40031C160206841686FF30F013943CD
:107D100041602068016841F0010101606068B0F5D0
:107D2000800F08D00CE00220BDE8F88F016841F414
:107D300000610160E7E72068016841F400710160BB
:107D4000E0680F281CD820E02068416989070BD51E
:107D5000E16D09680162E06D001DE065B4F8620044
:107D6000401EA4F862000BE0FDF7DAFE811B4945D6
:107D700003D3B9F1FF3F03D09DE0B9F1000F32D03A
:107D8000B4F862000028DFD179E007282FD872E02C
:107D90002068416989071ED5B4F8621001290DD900
:107DA000E16B59B1E16D09680162E06D001DE065AC
:107DB000B4F8620000E07CE0801E09E0E06D01881C
:107DC000ABF80010E06D801CE065B4F86200401E66
:107DD000A4F862000BE0FDF7A3FE811B494503D325
:107DE000B9F1FF3F03D066E0B9F1000F63D0B4F8FA
:107DF00062000028CCD142E02068416989072ED575
:107E0000B4F8621003290CD9E16B402909D9E16D5E
:107E100009680162E06D001DE065B4F86200001FB2
:107E20001AE0B4F8621001290CD9E16B51B1E06D90
:107E30000188ABF80010E06D801CE065B4F86200CA
:107E4000801E09E0E16D097880F82010E06D401C8B
:107E5000E065B4F86200401EA4F862000BE0FDF794
:107E60005FFE811B494503D3B9F1FF3F03D022E0F8
:107E7000B9F1000F1FD0B4F862000028BCD1002275
:107E80004B4608212046009602F000FC28B1D4F8A9
:107E9000840040F02000C4F88400204602F030FB4B
:107EA00084F88180D4F8840084F8805000283FF45E
:107EB0003BAF012038E7204602F022FBD4F88410C3
:107EC00084F8805041F48071C4F8841084F8818073
:107ED000032029E72DE9F041044690F88100164679
:107EE00001283DD100293AD0002E7FD094F880009F
:107EF000012835D0A2680025012784F8807003206E
:107F000084F88100C4F88450656665672567E1657B
:107F1000A4F868502C34B2F5C02FA686E686E58713
:107F200054F82C0D1FD0C16821F4C02141F4003158
:107F3000C0F80C10E1684FF480420F2903D9A06FFC
:107F40008069904209D1A06F07294FF400530FD9DF
:107F5000806998421DD090421BD084F8805045E043
:107F60000220BDE8F081016841F400610160E1E7B1
:107F70008169994205D1B4F86210491C4908A4F8F6
:107F80006210806990420ED1B4F86200C01C800873
:107F900007E00F2907D8904205D1B4F86200401CD1
:107FA0004008A4F86200A06F25490164A16F25482C
:107FB000C863A16F2448C864A06F05652068816804
:107FC00021F400418160B4F862302268E16DA06F55
:107FD0002032FCF70FFD58B1D4F8840084F88050AB
:107FE00040F01000C4F8840084F881700120B8E7E4
:107FF000A06FC069B0F5807F206841686FF30F0102
:1080000000D0314341602068816841F400418160C3
:108010002068016941F4487101612068016841F0FC
:10802000010101606068B0F5800F04D1206801682B
:1080300041F400710160002084F8805091E7000055
:108040000DA600083FA60008D7A5000810B502F04D
:108050000BFB032808D0054901EB401000680028FD
:1080600002D0BDE81040004710BD000028BD00242C
:1080700070B5044602F0F8FA032811D0204602F049
:10808000F3FA084D05EB4010C068002808D02046E0
:1080900002F0EAFA05EB4010C068BDE87040004706
:1080A00070BD000028BD002470B5044602F0DCFA63
:1080B000032811D0204602F0D7FA084D05EB4010F6
:1080C0008068002808D0204602F0CEFA05EB401068
:1080D0008068BDE87040004770BD000028BD0024E6
:1080E000024A136883430B4313607047040400582B
:1080F0007047704770470000F0B590F83C20012AA7
:1081000041D0224E012480F83C40022280F83D20DC
:1081100002681F4D5368B242D2F808C001D0AA428B
:1081200003D14F6823F470033B430F6823F07003BF
:108130001F4357600268B24219D0B2F1804F16D087
:10814000144B9A4213D0144B9A4210D0134B9A42BC
:108150000DD0AA420BD0124B9A4208D0114B9A4232
:1081600005D0114B9A4202D0104B9A4204D1896833
:108170002CF0800319439160002180F83D4080F885
:108180003C100846F0BD0220F0BD00000000014098
:10819000000401400004004000080040000C0040C2
:1081A000001800400040014000E0004000E40040B2
:1081B00010B5040003D094F83D0010B107E0012091
:1081C00010BD002084F83C00204600F023F8022077
:1081D00084F83D002068211D03F01EF9012084F879
:1081E000480084F83E0084F83F0084F8400084F89A
:1081F000410084F8420084F8430084F8440084F885
:10820000450084F8460084F8470084F83D000020CB
:1082100010BD000008B50C4A01680C48914207D116
:10822000016841F002010160006800F0020009E00D
:10823000074A914207D1016841F04001016000689E
:1082400000F04000009008BD00040040E8440258DF
:108250000018004090F83D10012901D0012070471E
:108260001A4A022180F83D100168CB6843F00103EF
:10827000CB60006890421AD0B0F1804F17D01449FB
:10828000884214D01349884211D0134988420ED035
:10829000124988420BD01249884208D011498842BD
:1082A00005D01149884202D01049884207D181681F
:1082B0000F4A1140062906D0B1F5803F03D001686E
:1082C00041F0010101600020704700000000014002
:1082D0000004004000080040000C00400004014081
:1082E000001800400040014000E0004000E4004071
:1082F0000700010070B5044690F83C0000250128F5
:1083000014D03A4B012684F83C60022084F83D00EA
:1083100022689068184020F47F40906008687028B8
:108320002FD010DC10F00F0F03D022E04FF002002E
:1083300070BD4FEA2012072A1BD2DFE802F0535328
:1083400053534B394100B0F1101F4BD009DCB0F54D
:10835000805F0FD0B0F5005F1ED0B0F5801F08D150
:1083600040E0A0F5801120393CD010293AD02029D6
:1083700038D0012584F83D60002084F83C00284670
:1083800070BD4A682068D1E9021303F0C2F8206882
:10839000816841F0770109E04A682068D1E9021359
:1083A00003F0B7F82068816841F480418160E1E71B
:1083B000CA684968206803F059FA2068502106E02D
:1083C000CA684968206803F062FA2068602103F0F7
:1083D000A9F8CFE7CA684968206803F047FA20681F
:1083E0004021F4E7226801461046F0E788FFCEFFFF
:1083F00070472DE9F041044600680027C66805690A
:10840000A90713D5B10711D5FA1E02610121217701
:10841000206880698007204602D0FFF7E9FF04E06A
:1084200000F0C4F8204600F086F92777680716D5D3
:10843000700714D5226802206FF0040111612077C3
:108440002068806910F4407F204602D0FFF7D0FFFB
:1084500004E000F0ABF8204600F06DF9277728071C
:1084600015D5300713D5226804206FF0080111617B
:1084700020772068C0698007204602D0FFF7B8FF48
:1084800004E000F093F8204600F055F92777E8065D
:1084900016D5F00614D5226808206FF0100111617E
:1084A00020772068C06910F4407F204602D0FFF793
:1084B0009FFF04E000F07AF8204600F03CF92777AF
:1084C000E80708D0F00706D021686FF001000861C6
:1084D000204600F0C3F9280601D4A80408D53006C8
:1084E00006D521686FF4025008612046FFF701FEAF
:1084F000E80508D5300606D521686FF4807008615C
:108500002046FFF7F5FD680608D5700606D52168F8
:108510006FF040000861204600F0A7F9A8060AD5D0
:10852000B00608D521686FF0200008612046BDE83C
:10853000F041FFF7DFBDBDE8F081000030B587B046
:10854000044614216846F8F708F924680021144D00
:108550000223124A1348AC4209D1146844F00204C1
:1085600014601268009302F0020205920CE00E4DB6
:10857000AC4210D1146844F002041460126802F096
:1085800002020592EA130092CDE90131CDE903130D
:108590006946FDF7ADF907B030BD0000E044025870
:1085A000000400400004025800180040704770B5F5
:1085B000044690F83C0000260D4601280BD001200F
:1085C00084F83C000C2A4AD007DC82B1042A20D06F
:1085D000082A06D131E0022070BD102A53D0142A97
:1085E00063D00126002084F83C00304670BD20682E
:1085F00002F0A2FF2068816941F0080181612068D2
:10860000816921F00401816120682A69816911432F
:1086100011E0206802F0E2FF2068816941F4006106
:1086200081612068816921F4806181612068296904
:10863000826942EA01218161D4E7206803F01AF8D7
:108640002068C16941F00801C1612068C16921F059
:108650000401C16120682A69C169114311E02068E1
:1086600003F054F82068C16941F40061C1612068D9
:10867000C16921F48061C16120682969C26942EA47
:108680000121C161AEE7206803F07CF82068416DEC
:1086900041F0080141652068416D21F00401416508
:1086A00020682A69416D114311E0206803F0A4F8A5
:1086B0002068416D41F4006141652068416D21F4FD
:1086C0008061416520682969426D42EA0121416566
:1086D00088E710B5040003D094F83D0010B107E01E
:1086E000012010BD002084F83C00204600F022F854
:1086F000022084F83D002068211D02F08DFE01203B
:1087000084F8480084F83E0084F83F0084F8400074
:1087100084F8410084F8420084F8430084F844005F
:1087200084F8450084F8460084F8470084F83D004A
:10873000002010BD7047704730B504464FF002026C
:1087400069B1042912D0082917D00C291CD010298E
:1087500021D094F84300012824D0012030BD94F8A2
:108760003E000128F9D184F83E201DE094F83F0036
:108770000128F2D184F83F2016E094F84000012847
:10878000EBD184F840200FE094F841000128E4D1B7
:1087900084F8412008E094F842000128DDD184F8F3
:1087A000422001E084F843200122206802F0A4FE68
:1087B0001E4920681E4A1F4B884209D0904207D0AC
:1087C000984205D01C4DA84202D01C4DA84203D1AE
:1087D000456C45F4004545642068884218D0B0F1E6
:1087E000804F15D01649884212D0164988420FD0C2
:1087F000154988420CD090420AD01449884207D0CB
:10880000984205D01249884202D01249884207D1C5
:108810008168114A1140062906D0B1F5803F03D086
:10882000016841F001010160002030BD00000140FD
:108830000004014000400140004401400048014064
:108840000004004000080040000C004000180040F8
:1088500000E0004000E40040070001000068B0F1C3
:10886000804F01D1FDF762B97047704730B590F87D
:108870008410012918D0012280F884202421C0F816
:1088800088100022202401680B680D6823F0005333
:1088900025F001050D60426601680B60C0F8884054
:1088A00080F88420104630BD022030BD70477047EC
:1088B00070B5044690F8840001281DD0012284F888
:1088C00084202420C4F8880020680568026822F00B
:1088D000010202602068826822F060620A438260BE
:1088E000204603F007FC2268202100201560C4F810
:1088F000881084F8840070BD022070BD70B50446F5
:1089000090F8840001281DD0012284F884202420BE
:10891000C4F8880020680568026822F0010202603D
:108920002068826822F060420A438260204603F099
:10893000E1FB2268202100201560C4F8881084F82B
:10894000840070BD022070BD7047704710B503F001
:108950006FFD02280AD000EBC001054800EB810042
:108960000069002802D0BDE81040004710BD00009B
:1089700068BD00242DE9F04107680025044640F653
:108980000F030226F8693968BA6818420AD18306CB
:108990007ED501F0200302F0805C53EA0C0377D00F
:1089A000616F7EE1D44BDFF854C3134001EA0C0C35
:1089B00053EA0C0C6CD05FEAC07C0CD05FEAC15C5F
:1089C00009D54FF0010CC7F820C0D4F8907047F0DB
:1089D0000107C4F89070870709D5D70707D0276823
:1089E0003E62D4F8906046F00406C4F890604607F2
:1089F0000AD5D60708D0276804263E62D4F89060CE
:108A000046F00206C4F8906006070CD501F0200677
:108A10001E4308D0266808233362D4F8903043F010
:108A20000803C4F8903003050BD54B0109D526681F
:108A30004FF400633362D4F8903043F02003C4F85D
:108A40009030D4F89030002B3DD0800609D501F04D
:108A5000200002F08051084303D0616F09B1204625
:108A600088472168D4F890008968490602D410F03C
:108A7000280F2AD0204603F099FC20688068400621
:108A80001ED52068083050E8001F21F0400100E0AA
:108A900021E040E80012002AF3D1D4F8800078B138
:108AA00097490165D4F88000FBF70EF900280AD039
:108AB000D4F88000016D00E02046BDE8F041084791
:108AC0002046FFF743FFBDE8F0812046FFF73EFF59
:108AD000C4F89050F7E7D4F86CC02023BCF1010F24
:108AE0007ED15FEAC06C7BD55FEAC16C78D510207F
:108AF000386220688068400673D5D4F880208149A8
:108B00001068884234D07F491831884230D07D497E
:108B1000303188422CD07B494831884228D079496D
:108B20006031884224D077497831884220D0754915
:108B3000903188421CD07349A831884218D07249BC
:108B4000884215D070491831884211D06E493031B1
:108B500088420DD06C494831884209D06A49603159
:108B6000884205D068497831884201D06649903101
:108B700040684FF480770004000C40D0B4F85C10DB
:108B800081423CD9A4F85E00D069B8422FD0216858
:108B900051E8000F20F4807041E80002002AF6D16D
:108BA0002068083050E8001F21F0010140E8001261
:108BB000002AF5D12068083050E8001F21F040015C
:108BC00040E80012002AF5D1C4F88C30E566206830
:108BD00050E8001F21F0100140E80012002A01E0D7
:108BE0004AE019E0F3D1D4F88000FAF7BDFE266719
:108BF000B4F85C00B4F85E10401A81B208E0B4F832
:108C00005C1081427FF466AFD069B842FAD1266722
:108C10002046FFF74BFE56E7B4F85C00B4F85E1050
:108C2000B4F85E20401A81B2002AF4D00029F2D0B4
:108C3000226852E8000F20F4907042E80007002FED
:108C4000F6D1324F206800F1080050E8002F02EA08
:108C5000070240E8002CBCF1000FF3D1C4F88C30BF
:108C6000E5666567226852E8000F20F0100042E8D0
:108C70000003002BF6D1CAE7C60209D5560207D574
:108C80004FF4801038622046BDE8F041FFF75DBE2A
:108C900006060AD501F0800602F40002164304D04D
:108CA000A16F00297FF408AF0DE7420611D54A06EF
:108CB0000FD52046016851E8002F22F0400241E81C
:108CC0000024002CF6D1C0F88830856700F01AF92E
:108CD000F9E6020206D54A0004D52046BDE8F04177
:108CE000FFF732BEC00196D5002994DA2046BDE8D0
:108CF000F041FFF7DCBD000001000010200100047E
:108D0000ABC200081000024010040240FEFFFFEF5B
:108D100010B5040003D0D4F8880010B107E001209A
:108D200010BD002084F88400204600F027F824209D
:108D3000C4F888002068016821F001010160A06A80
:108D400010B1204603F0F8F9204603F07BFB012820
:108D5000E6D02068416821F4904141602068816834
:108D600021F02A0181602068016841F00101016061
:108D70002046BDE8104003F043BA0000F0B5B5B09E
:108D8000064614212EA8F7F7E8FCB8216846F7F745
:108D9000E4FC3049306888425AD100201D900221FD
:108DA0000546CDE900106846FDF71EF908B1FAF74F
:108DB000E8F92948016841F480110160006800F475
:108DC0008010339024480838016841F004010160A4
:108DD000016801F004013391016841F0080101606C
:108DE000006802242EA900F008003390E002082752
:108DF00081E831001948CDE93157FCF779FD2EA9FA
:108E0000042081E831001648CDE93157FCF770FDA8
:108E1000144C4121144802152060C4E90115D00109
:108E2000C4E903526561A561C4E907502046656243
:108E3000FBF702FC08B1FAF7A4F9C6F8804000225B
:108E40000521A6633520FCF71DFF3520FCF70DFF3B
:108E500035B0F0BD00500040E84402580008025808
:108E6000000C0258580900248804024030B4D0F89D
:108E70008C30202B02D0022030BC7047A9B1A2B1A7
:108E80000B4D00240368C466AB420BD05B681B0229
:108E900008D5046854E8003F43F0806344E8003597
:108EA000002DF6D130BC03F0BBBC0120E4E700008C
:108EB000000C005810B503F0BBFA02280AD000EBF2
:108EC000C001054800EB8100C068002802D0BDE861
:108ED0001040004710BD000068BD002410B503F02D
:108EE000A7FA02280AD000EBC001054800EB810078
:108EF0008068002802D0BDE81040004710BD000087
:108F000068BD002410B503F093FA02280AD000EBE4
:108F1000C001054800EB81004068002802D0BDE890
:108F20001040004710BD000068BD0024FEE70000AF
:108F300010EE100A0C49B6EE001AF7EE080A20EE01
:108F4000011AA1EB600000EE100AF0EE601A21EEAB
:108F5000002A42EE401A21EE800A21EE001A41EE6C
:108F6000400A20EE800A7047DF59375F38B390ED32
:108F7000061AD0ED012AF0EE400AD0ED071A41EEB4
:108F8000620A90ED022A4FF07F4241EEC20A10EED3
:108F9000901AB2EB410F01D1F0EE400A90ED040AB5
:108FA000D0ED032A90ED052A21EE000A80ED071A84
:108FB000C0ED060A00EEA20A01EE820A70479FED9C
:108FC000010A70470000000010B504002DED068B6B
:108FD00018D0F5EEC00A9FED2C1AC4ED000AF1EE90
:108FE00010FA84ED061AF7EE008A84ED071A0CD801
:108FF000C4ED038A84ED041A84ED051A84ED011A88
:1090000080ED021ABDEC068B10BD80EE201ADFED5C
:109010001F0A80EE810A04F057FA9FED1DAAB0EEF8
:10902000408AB0EE4A0A04F0B9F8F0EE009AB0EEC9
:10903000689A20EE291AB0EE680A68EE080A18EE5F
:10904000080A01EE089A20EE291A08EE089A80EE26
:10905000890AC1EE090A84ED030A20EE291A84ED7B
:10906000050AB0EE4A0AC4ED010A84ED041A04F0C0
:1090700095F820EE290A40EE488A48EE088A88EEE4
:10908000890A84ED020ABDE700000000DB0F4940B9
:10909000DB0F493FB8B190ED031AD0ED041AD0EDC3
:1090A000050A31EE211A31EE201AC0EE010A10EE47
:1090B000901A6FEAD15111F0FF0F07D0C0ED060AE8
:1090C000C0ED070A06E09FED040A704780ED060A2E
:1090D00080ED070AFFF74ABF0000000000B593B01B
:1090E00018B300F033F818B38388FF2108228DF8F5
:1090F00004208DF808108DF805108DF809100093E4
:10910000FC238DF806108DF80A108DF807108DF8E5
:109110000B1069468DF80C300078F8F761FD0028D7
:1091200001D04FF0FF3013B000BD6FF00100FAE73F
:109130006FF00300F7E70000032801D30020704719
:10914000014951F820007047A0BD002470B504000B
:1091500019D02078FFF7F0FF010014D091F8843087
:1091600000200EE001EB800252684AB115782678A3
:10917000B54205D155886688B54201D1104670BD0B
:10918000401C8342EEDC002070BD10B50C4640B19F
:109190003CB1FFF7DBFF38B12146BDE8104000F0DD
:1091A000D3B86FF0010010BD6FF0030010BD0000D8
:1091B00070B504000D4636D0A5B3B5F801001021F6
:1091C000DFED2D0A9FED2D0A40BA05F033FB84ED4B
:1091D000070AE8782979F3EE0E0A000140EA111037
:1091E0000C21BBEE0E0A05F025FB84ED080A287958
:1091F000697900F00F00F2EE080A41EA00200C2124
:10920000BAEE080A05F016FB84ED090AA879DFED2D
:109210001C0A01EE100AB8EE411A84ED0A1A94ED08
:10922000071A07E0FFE76FF0010070BD31EE201A6A
:1092300084ED071AB5EEC01AF1EE10FAF6D3114913
:1092400011EE100A884204DB31EE601A84ED071A31
:10925000F6E7E07968B1D4ED081A70EEC10AB1EE14
:10926000400A84ED090AB1EE611AC4ED070A84EDE3
:10927000081A002070BD0000DA0F4941DA0F49C119
:10928000DB0FC940DB0FC9402DE9F04105000AD0D2
:109290002C784FF0FF38032C46D22A4E002756F880
:1092A000240080B903E06FF00100BDE8F081882060
:1092B000F8F75AFD46F82400B0B38821F7F74DFAC5
:1092C00056F8240004702878FFF736FF04002BD0EE
:1092D00094F8841000200BE004EB8002526832B155
:1092E00052886B889A4202D16FF00200DDE7401C81
:1092F0008142F1DC202917D23020F8F735FD060035
:1093000012D03021F7F729FA286803223060686804
:1093100070603772E879307669882878F8F7E2FA71
:1093200020B13046F8F7BAFC4046BEE794F8840016
:1093300004EB8000466094F88400401C84F88400AC
:109340000020B2E7A0BD00242DE9F04F5FEA000B3A
:1093500089462DED028B93B068D0B9F1000F65D02E
:10936000102099ED020A9FED331ADFED330A04F065
:10937000C5FA99ED010AB3EE0E1AFBEE0E0A82460B
:109380000C2004F0BBFA9FED2E8A99ED030A9FEDA5
:109390002B1AF0EE480A07460C2004F0AFFA99EDBC
:1093A000040AB1EE041AF0EE480A06460C2004F056
:1093B000A5FA99ED000AB2EE081AFAEE080A054677
:1093C0000C2004F09BFA01464FEA1A202A0966F3A2
:1093D000070860F307042B0162F30F28380943EAFA
:1093E00011226AF30F243B0160F31744BBF8040019
:1093F00062F31748009043EA162308228DF80420F0
:1094000063F31F64CDF8054061F31F68CDF8098050
:109410009BF800006946F8F7E3FB002801D04FF005
:10942000FF3013B0BDEC028BBDE8F08F6FF0010090
:10943000F7E70000DA0F4941DA0F49C10000FA43AB
:109440000000000070B5040096B00AD02078FFF745
:1094500073FE01006FF003052ED091F884200020E8
:1094600028E06FF0010016B070BD00BF01EB800373
:109470005B68F3B15B886688B3421AD101EB800068
:109480006A46B1B2002345682078F8F7E7F8A8B13A
:10949000F8F7F1FCD5E904340F4E0022C01A61EB55
:1094A0000401301A8A4101D2002028724FF0FF30A7
:1094B000D9E7401C8242D9DC2846D4E70120287233
:1094C000F8F7D9FCC5E904010DF10D012846FFF7B5
:1094D0006FFE0020C7E70000A086010070B5040001
:1094E00092B015D0207800F063F8A8B16388082105
:1094F000801C4FF0FF35A3F201236A460B2B55D297
:10950000DFE803F00D0D0D0D212121213636360047
:109510006FF0010012B070BD6FF00300FAE74FF476
:10952000007300938DF804105FF0000130F81130E3
:109530001E0A02EB41035E7110F81160491C0429F8
:109540009E71F3DB2CE040F2FF1300938DF80410C2
:109550005FF0040130F811301E0A02EB410303F8FA
:10956000036D10F81160491C08295E70F2DB17E0EA
:1095700040F2FF2300938DF80410082130F81130D9
:109580001E0A02EB410303F80B6D10F81160491C31
:109590000B295E70F2DB00208DF80B008DF80C00BB
:1095A00011462078F8F71CFB0028B3D02846B1E715
:1095B000032801D300207047014951F8200070476B
:1095C000ACBD002430B1012807D0022808D04FF0EC
:1095D000FF30704742F2107070474FF48040704780
:1095E00047F23050704770B5040015D02078FFF76F
:1095F000DFFF00280CD090F8443000210AE000EB97
:10960000810292692AB155886688B54201D1104617
:1096100070BD491C8B42F2DC002070BD2DE9F04189
:10962000050009D02C784FF0FF37032C48D22B4E81
:1096300056F8240080B903E06FF00100BDE8F08126
:109640004820F8F791FB46F82400C8B34821F7F703
:1096500084F856F8240004702878FFF7A9FF040066
:109660002ED094F8441000200CE000BF04EB8002E0
:10967000926932B152886B889A4202D16FF002002F
:10968000DCE7401C8142F1DC0B2919D25020F8F7AD
:109690006BFB060014D02868282130606868706071
:1096A00006F11800F7F759F86879032286F82800C0
:1096B00069882878F8F716F920B13046F8F7EEFAFD
:1096C0003846BBE794F8440004EB8000866194F8C8
:1096D0004400401C84F844000020AFE7ACBD0024E7
:1096E0009FED010A00F002B80000000070B5040010
:1096F0002DED028BB0EE408A0ED02078FFF758FF98
:1097000005006FF0030625D018EE100AB0F17E5F59
:1097100007DDB7EE008A0BE06FF00100BDEC028BB5
:1097200070BD18EE100A10F1814F01D9BFEE008A0A
:10973000607908B1B1EE488A2046FFF754FF48B17E
:1097400021794FF0FF32608831B1012904D002291C
:1097500010D109E03046E1E7A0F20120072809D83E
:1097600044B2002C06DB07E0A0F20523062B01D84B
:10977000401EF5E71046D1E7AD1C0846FFF722FF73
:1097800000EE100AB8EEC00A20EE080ABDEEC00ACC
:1097900010EE100A25F814000020BFE7F0B5050010
:1097A00095B00AD02878FFF703FF01006FF0030699
:1097B00040D091F8442000203AE06FF0010015B04D
:1097C000F0BD00BF01EB80039C697CB363886F88A8
:1097D000BB422CD1B9B2287800236A46F7F73EFF86
:1097E00090B1F8F748FBD4E908354FF47A77C01AFE
:1097F00061EB05010022381A8A4102D2002020764E
:1098000018E04FF0FF30DAE701202076F8F733FB5D
:10981000C4E908016946204600F062FB04F1080033
:109820002C340FC884E80F000020C8E7FFE7401C75
:109830008242C7DC3046C2E7154808B5016841F0EE
:1098400001010160016801F001010091016841F02E
:109850000201016000680022052100F00200009072
:109860000B20FCF70FFA0B20FCF7FFF90022052173
:109870000C20FCF707FA0C20FCF7F7F90022052171
:109880004420FCF7FFF9BDE808404420FCF7EDB99F
:10989000D8440258184800212DE9F041154F012401
:1098A00081600E2507600522C16004230474102620
:1098B000417484744261C0E9062502624262C0E9D3
:1098C0000A250263C0E90D14C0E91131C0E9133162
:1098D000C0E91531C0E90F46C0E91716C0E91913F0
:1098E000FBF78EFD002803D0BDE8F041F9F749BC35
:1098F000BDE8F08100A000404C0400241A4800217B
:109900002DE9F041174F012481600E2507600522E3
:10991000C16040F23F3704740423417410268474FC
:109920004261C0E9062502624262C0E90A2500F1EF
:1099300040050263C0E90D74C46385E84A00C0E9CC
:109940001331C0E91531C0E91716C0E91913FBF747
:1099500057FD002803D0BDE8F041F9F712BCBDE87F
:10996000F081000000A40040EC0400241A4800210B
:109970002DE9F041174E0122816005230660102574
:10998000C1600E27027440F27E6641740424827422
:109990004561C0E90632C0E90823C0E90A3703631C
:1099A000C0E90D6200F14006C26386E83200C0E9FA
:1099B0001341C0E91541C0E91715C0E91914FBF7B7
:1099C0001FFD002803D0BDE8F041F9F7DABBBDE880
:1099D000F081000000D400408C050024074A0021DB
:1099E000074810B504F00AFA0649074A0860002142
:1099F000BDE81040054804F001BA0000B0FF0008BF
:109A000015B2000800000024A0010108B5B8000844
:109A1000F0B587B014216846F6F79FFE3848016814
:109A200041F004010160016801F004010591016841
:109A300041F080010160016801F080010591016839
:109A400041F001010160016801F001010591016827
:109A500041F002010160016801F002010591016815
:109A600041F010010160016801F0100105910168E9
:109A700041F00801016000684FF46047214E002268
:109A800000F00800394605903046FCF744F8012202
:109A900030460921FCF73FF800250097012469466C
:109AA0003046CDE901450395FBF722FF09206946C1
:109AB000CDE90004304602940394FBF719FF4FF4FC
:109AC000A0504FF404118DE813000F486946FBF7CE
:109AD0000FFFE0034FF488118DE823000B4869461F
:109AE000FBF706FF0021E006FEF7FAFA0022052147
:109AF0002820FCF7C7F82820FCF7B7F807B0F0BD1E
:109B0000E0440258000802580010025800000258B1
:109B10002DE9F04117484FF48007DFF854C00021C9
:109B2000FA000726C0F800C04FF04053C0E90362B6
:109B3000C0E90171C0E907314162551054008162EA
:109B40005201C162C0E90D21C163016441648164B5
:109B5000C164016541658165C0E90554FDF7E2FC1A
:109B6000002803D0BDE8F041F9F70BBBBDE8F08158
:109B7000003800402C06002470B514484FF48005CE
:109B80000021114C2B010322C0E90321C0E9051378
:109B9000C1611A0101626E1141628162C162C0E954
:109BA0000D21C163016441648164C1640165416543
:109BB000816580E87000FDF7B5FC002803D0BDE8A2
:109BC0007040F9F7DEBA70BD00140058B4060024E6
:109BD00010B58EB000241C21009407A801940294B3
:109BE0000394049405940694F6F7B7FD1E4840F6D6
:109BF000C31117221B4BC0E9024104618461C0E913
:109C00000032FEF7D5FA08B1F9F7BBFA4FF48050ED
:109C1000009015486946FEF76DFB08B1F9F7B1FAF7
:109C20001148FEF756FD08B1F9F7ABFA0E4804A942
:109C300004940694FEF760FA08B1F9F7A2FA6020DE
:109C4000CDE907040848042207A909940B94FEF7FC
:109C5000AEFC08B1F9F795FA0348FEF76FFC0EB0B9
:109C600010BD0000001800407808002410B58EB028
:109C700000241C21009407A80194029403940494E6
:109C800005940694F6F769FD1E4842F20F711722FB
:109C90001B4BC0E9024104618461C0E90032FEF758
:109CA00087FA08B1F9F76DFA4FF480500090154823
:109CB0006946FEF71FFB08B1F9F763FA1148FEF792
:109CC00008FD08B1F9F75DFA0E4804A9049406945A
:109CD000FEF712FA08B1F9F754FA6020CDE907044B
:109CE00008480C2207A909940B94FEF760FC08B100
:109CF000F9F747FA0348FEF721FC0EB010BD00004B
:109D0000000400402C080024184800212DE9F041EF
:109D1000154A0C24C0E90541C16101629514144B38
:109D2000561441621715816280E8EC00FEF7F0FFDF
:109D300008B1F9F726FA0D480021FEF7DFFD08B15A
:109D4000F9F71FFA09480021FEF7B2FD08B1F9F74B
:109D500018FA0648FEF78AFD002803D0BDE8F04156
:109D6000F9F70FBABDE8F08100500040C4080024A4
:109D7000A0860100FEE7000030B500284FF0FF3458
:109D80007DD00078DFED510A062834D2DFE800F0FC
:109D900003354C5B5B59042B55D191EC031A31EE22
:109DA000611A31EE021A82ED001A91ED001A91ED5E
:109DB000012AD1ED021A31EE021A31EE211A82ED9A
:109DC000011A91ED011AD1ED001A91ED022A31EE3E
:109DD000611A31EE021A82ED021A91ED002AD1EDDC
:109DE000011A91ED021AB1EE422A72EE611A31EEB9
:109DF000811A82ED031A002038E0042B23D191ED63
:109E0000000AB1EE400A82ED000A91ED000A82EDEF
:109E1000010A91ED000A82ED020A91ED000AB1EE0D
:109E2000400A82ED030A0EE0022B0CD191ED000AEC
:109E3000B1EE400A82ED000A91ED000A82ED010ABE
:109E400007E0012B01D000203CE091ED000A82EDFB
:109E5000000A002030E000BF02EB8001401C91EDC1
:109E6000001A40B2B0EEC11AC1FE200A9842F3DBDC
:109E700010EE900AB0F17E5F0EDD00200AE023E0D4
:109E800002EB8001401C91ED001A40B2C1EE201A95
:109E9000C1ED001A9842F3DB002009E002EB8001DB
:109EA000401CD1ED000A40B260EE800AC1ED000A0C
:109EB0009842F3DB002030BD411C02EB8000C0ED76
:109EC000000AC8B29842F7DB204630BD000000000F
:109ED00010B10170002070474FF0FF307047000054
:109EE0002DE9F0410E460446B1F80D00B1F80F100F
:109EF000B6F8112045BA49BA50BA0FB20FFA80F835
:109F00002079FFF75FFB217949B301292AD0B7EE09
:109F1000001A00BF18FB00F000EE905A9FED413A86
:109F200001EE907AF8EE600A9FED3F0AB8EEE12A62
:109F3000DFED3E2A20EE833A00EE900AA179F8EE9A
:109F4000E01A63EE000A61EEA21A59B3B4F84000B9
:109F5000281AB0F5805F08DD606C401E0AE09FEDB6
:109F6000341AD7E79FED331AD4E710F5805F02DA91
:109F7000606C401C606482EE013AD4ED112A21EE3F
:109F8000812AA4F84050F8EEE21A84ED042A41EE4A
:109F9000800AC0EE811AC4ED121AC4ED021A84EDD3
:109FA000033A0DE0A4F840500020C4ED020A84ED0D
:109FB000032A9FED211AC4ED041A606484ED121A7D
:109FC000D4ED020AF5EEC00AF1EE10FA09D270EEF5
:109FD000800AC4ED020AF5E770EEC00AC4ED020A79
:109FE00000E0164910EE900A8842F5DA94F828004D
:109FF00078B1F0EE601AD4ED030A94ED041A30EE55
:10A00000610A04F10800F1EE600AB1EE411A80EC39
:10A01000030AF07C00EE100AB8EE400A84ED050A4F
:10A02000BDE8F08100000039DB0FC9400000803836
:10A03000000010422CA0994100000000DB0FC94035
:10A04000FEE7000010B504462DED068BF0EE409AB9
:10A05000F0EE618AB0EE418AB0EE609A19EE900A95
:10A0600002F0A8FC002850D019EE100A02F0A2FC61
:10A0700000284AD0B0EE480A10EE100A02F09AFC0E
:10A08000002842D018EE900A02F094FCE8B3606811
:10A09000F0EE490AB0EE690A90ED071AF8F7E2FC13
:10A0A0006068F0EE409AD0ED000A04F11C0020EE4A
:10A0B000891A20EEA99AB0EE410AFEF757FF2078E0
:10A0C000DFED38AAB0EE40AA70B101280ED1D4ED70
:10A0D000020AB0EE680A03F009F9D4ED050A7AEE37
:10A0E000600A80EE808A01E0B0EE6A8A18EE100AFB
:10A0F000C4ED049A84ED05AA6FEAD05010F0FF0F6A
:10A1000001D1B0EE6A8A606800E047E0D4ED030A4E
:10A1100090ED010AD0ED031A49EE280A20EE090A53
:10A1200090ED021A204A11EE101A08EE610A21EE93
:10A13000201A91421CDD10EE901A6FEAD15111F0F5
:10A14000FF0F15D070EE011A90ED052AF0EEE11A1E
:10A15000F4EEC21AF1EE10FA0AD890ED042AF0EEED
:10A16000E01AF4EEC21AF1EE10FA01D8C4ED030AB7
:10A1700030EE010A10EE101A6FEAD15111F0FF0F04
:10A180000CD0D0ED050A10EE900A904201DDF6F7F2
:10A19000B1FF84ED060ABDEC068B10BD94ED060AF6
:10A1A000F9E7000000000000BD37863570B50400F7
:10A1B0000D464FF0FF3137D050686FEAD05010F0A5
:10A1C000FF0F31D090686FEAD05010F0FF0F2BD006
:10A1D000D0686FEAD05010F0FF0F25D010696FEAF9
:10A1E000D05010F0FF0F1FD050696FEAD05010F020
:10A1F000FF0F19D0B7EE001A6260C1EE000A10EE30
:10A20000900A6FEAD05010F0FF0F0DD0C4ED020A93
:10A21000D2ED060A04F11C00FEF7D6FE204625709A
:10A2200000F004F8002070BD084670BD10B570B194
:10A230009FED080A80ED030A80ED040A80ED050A0F
:10A2400080ED060A1C30FEF725FF002010BD4FF000
:10A25000FF3010BD0000000028B19FED040A80ED22
:10A26000030A002070474FF0FF30704700000000E5
:10A2700070B5AEB0B8216846F6F76FFA002318241F
:10A2800019464FF4004202208DE81C00C82506AB99
:10A29000CDE903502026059083E843000207684675
:10A2A0001B920991FBF7A0FE002801D072B6FEE7D1
:10A2B0002EB070BD2DE9F047454D044689464FF05C
:10A2C000000A2868C04380070AD0414E283E306803
:10A2D00020F080603060FBF723FC0746B04608E0C2
:10A2E0000120BDE8F08700BFFBF71AFCC01B022865
:10A2F00067D8D8F800000001F6D4206829684FF428
:10A30000FE0721F47C313E0241EA00302860207AC9
:10A31000A389B4F804C040022D4D2D495B1E227C58
:10A32000ACF1010C1035091DA0F5007080B2521E71
:10A33000CCF3080C07EA034340EA0C00184306EA92
:10A340000262104328600868626920F0C000104370
:10A3500008600A68A06922F0200202430A60281DF2
:10A360000A6822F010020A6002684FF6F873E46986
:10A370009A4342EAC40202600868B9F1000F40F053
:10A3800010020A6011D00868B9F1010F11D040F431
:10A3900000100860D8F80000444640F08060C8F81B
:10A3A0000000FBF7BDFB05460DE0086840F4002007
:10A3B000EFE740F48010ECE7FBF7B2FB401B02280C
:10A3C00001D903208DE720680001F5D5504688E7C4
:10A3D000284402582DE9F047454D044689464FF080
:10A3E000000A2868C04380070AD0414E283E3068E2
:10A3F00020F080503060FBF793FB0746B04608E042
:10A400000120BDE8F08700BFFBF78AFBC01B0228D4
:10A4100067D8D8F800008000F6D4208829684FF467
:10A42000FE0721F07C713E0241EA00502860207A4C
:10A43000A389B4F804C040022D4D2D495B1E227C37
:10A44000ACF1010C1835091DA0F5007080B2521E48
:10A45000CCF3080C07EA034340EA0C00184306EA71
:10A460000262104328600868626920F4406010436B
:10A4700008600A68A06922F4007202430A60281D7D
:10A480000A6822F480720A6002684FF6F873E46981
:10A490009A4342EAC40202600868B9F1000F40F42E
:10A4A00080720A6011D00868B9F1010F11D040F034
:10A4B00080700860D8F80000444640F08050C8F82A
:10A4C0000000FBF72DFB05460DE0086840F4800016
:10A4D000EFE740F40000ECE7FBF722FB401B02280B
:10A4E00001D903208DE720688000F5D5504688E724
:10A4F000284402580148FCF703BF00002C06002442
:10A5000010B5026840F26F335169946944F0080451
:10A5100094610268946944F01004946102681468BC
:10A5200024F001041460026814699C4314610268F9
:10A53000936823F44043936090F88120042A0CD060
:10A540008A060AD5D0F8842042F08002C0F8842020
:10A550000268936943F02003936190F88120032AF5
:10A560000CD04A060AD5D0F8842042F00402C0F884
:10A5700084200268936943F0400393618A050AD5F9
:10A58000D0F8842042F00102C0F884200268936968
:10A5900043F400739361C9050AD5D0F8841041F0E3
:10A5A0000801C0F8841001688A6942F480728A61E7
:10A5B0000021A0F86210A0F86A1010BD10B5806BE1
:10A5C00000210122A0F86A10A0F8621080F8812012
:10A5D000FCF77AFE10BD10B5846BF9F7B7FC0228C2
:10A5E0000ED02046FFF78CFFD4F88410012041F0F4
:10A5F0001001C4F8841084F881002046FCF764FE42
:10A6000010BD10B5806BFDF727FB10BD10B5806B3A
:10A61000FDF72EFD10BD10B5806B90F88110072955
:10A6200009D0C16FC969B1F5807F05D000680169A3
:10A6300041F00801016110BDFDF7F2FA10BD10B53F
:10A64000806B90F88110072909D0816FC969B1F535
:10A65000807F05D00068016941F00801016110BDEB
:10A66000FDF7F4FC10BD000000680649884201D1E6
:10A67000002070470449884201D10120704703201F
:10A680007047000000380040001400582DE9F041E8
:10A690001C4616460D460746DDF818800AE000BF46
:10A6A000FBF73EFAA0EB0800A04202D3601C01D0E9
:10A6B0000BE054B13868406935EA000007D000204B
:10A6C000B042EDD00020BDE8F0810320FBE701207F
:10A6D000F6E791ED000A90ED001A31EE000A10EE57
:10A6E000102AB2F17E5F0DDDF7EE001AC1EE800A8E
:10A6F00021EE200A80ED000A91ED000A20EE200AEA
:10A7000081ED000A7047000010B550B382699FEDDB
:10A71000180A137843B3012B22D1DFED160A08245F
:10A7200000EB011304EB8101114490ED672A93EDD6
:10A73000091AD1ED001A11EE821AB0EEC11AB4EE68
:10A74000E01AF1EE10FA09D221EE010A60EEA00A39
:10A75000F7EE001A80EE201A31EEC10A80ED460AAB
:10A7600010BDBFEE000A10BDDFED030AD7E7000001
:10A77000000000000000C8430000484270B504001B
:10A780000D462DED028B3FD0B4F82001D8B394EDE7
:10A79000000AD4ED470ADFED1E8A30EE608AD4ED60
:10A7A000490A94ED680AB0EE681AF8F75BF9A069F7
:10A7B000F7EE001A90ED061AC1EE810AF4EEC80A0F
:10A7C000F1EE10FA1BD8A978C9B110EE101AB1F148
:10A7D0007E5F14DC94ED000AF0EE680A84ED470A0F
:10A7E00090ED050A04F5D070B8EE401A80EE810AAB
:10A7F000F8F71DF9B4F82001401EA4F8200100204C
:10A80000BDEC028B70BDFFE74FF0FF30F8E70000B2
:10A81000DB0FC94028B18169097829B101290AD122
:10A8200005E04FF0FF3070479FED040A01E09FED17
:10A83000040A80ED670A00207047000000409C4534
:10A8400000007A4570B504000D462DED028B2CD02A
:10A850005DB3F7F710FB05F030FB00EE100A9FED3B
:10A86000148AC0EE080AC4ED000AF7F704FBD4E925
:10A870000223801A61EB030105F01FFB00EE100AB2
:10A88000C0EE080AC4ED040AF7F7F5FAC4E90201BC
:10A890009FED080A2046FFF7BDFF2946204600F03D
:10A8A000A1F80020BDEC028B70BD4FF0FF30F9E73E
:10A8B00000247449000069432DE9F04104000D466D
:10A8C0002DED028BB0EE408A05D025B1B5EEC08AE1
:10A8D000F1EE10FA05D84FF0FF30BDEC028BBDE869
:10A8E000F0812879A561C7B2F6F7EAFE002631E0CB
:10A8F00006EB860005EB40002C30FEF78FFEC6EB22
:10A900000610012104EB8008B0EE480A08F5D27069
:10A9100005F17002FFF74AFC0121B0EE480A08F584
:10A92000437005F19002FFF741FCA16904EB461862
:10A93000B0EE480A08F2EC40D1ED4C0AFEF744FBB9
:10A94000A069B0EE480AD0ED4D0A08F2AC50FEF70F
:10A950003BFB761CBE42CBDB05F16800FEF75EFEDA
:10A96000A16904F2744304F5966691F86C0078B11D
:10A97000012802D06FF00300AFE701211846B0EEC6
:10A98000480A05F1F002FFF711FC05F5887209E0AD
:10A9900001211846B0EE480A05F1B002FFF706FCA7
:10A9A00005F1D00230460121B0EE480AFFF7FEFB68
:10A9B000A069B0EE480AD0ED4E0A04F26C60FEF7D2
:10A9C00003FBA069B0EE480AD0ED4F0A04F28C6098
:10A9D000FEF7FAFA142104F58E70F5F7BEFE00209A
:10A9E0007BE7000070B504002DED028B11D0A0694B
:10A9F000002590F82020EAB394F8DC3001229FED86
:10AA00003E8A5BB1012B1BD0022B3DD0032B69D1B9
:10AA100051E04FF0FF30BDEC028B70BD94ED240A85
:10AA200090ED091AC0EE080AF4EEC10AF1EE10FA30
:10AA300026DD94ED000A84F8DC2084ED360A1FE060
:10AA400094ED240A90ED091AC0EE080AF4EEC10A4A
:10AA5000F1EE10FA46D3D4ED000A94ED361A90EDDB
:10AA60000A0A70EEC10AF4EEC00AF1EE10FA07DB32
:10AA7000022000E03AE084F8D42084F8DC0033E0DF
:10AA8000204600F0D1F82FE0A4F82051032290EDE9
:10AA9000050ADFED1A0A94ED491AB8EE400AC0EE35
:10AAA000801A31EE610A84ED680A84F8DC2094EDA6
:10AAB000000A84ED360A204600F0B6F894ED000A4C
:10AAC000D4ED360A0E4930EE600A10EE100A8842C4
:10AAD0000ADBD4ED240A0B4980EE880A10EE100A36
:10AAE000884201DA84F8DC50002094E784F8DC50D6
:10AAF00084F8D450C4E7000000007A44DB0FC9405A
:10AB00009A99993E0000A0412DE9F04104002DEDF5
:10AB1000028B05D0A06900259FED1E8A067920E0F2
:10AB20004FF0FF30BDEC028BBDE8F081C5EB0510A6
:10AB300004EB800707F5D270FFF778FB07F5437049
:10AB4000FFF774FB04EB4517B0EE480A07F2EC4040
:10AB5000FEF7A0FAB0EE480A07F2AC50FEF79AFAF8
:10AB60006D1CB542E2DB04F27440FFF75FFB04F5B5
:10AB70009660FFF75BFBB0EE480A04F26C60FEF7EC
:10AB800089FAB0EE480A04F28C60FEF783FA0020DE
:10AB9000C8E70000000000002DE9F041040003D0E8
:10ABA000A0690025067910E04FF0FF30BDE8F08184
:10ABB000C5EB051004EB800707F5D270FFF74CFBDF
:10ABC00007F54370FFF748FB6D1CB542F0DB04F25C
:10ABD0007440FFF741FB04F59660FFF73DFB002052
:10ABE000E4E7000028B181699FED0E0A0B7900218E
:10ABF0000DE04FF0FF30704700EB8102491C82ED01
:10AC00004C0A82ED520A82ED580A82ED5E0A9942A0
:10AC1000F2DB80ED640A80ED650A80ED660A0020B3
:10AC200070470000000000002DE9F04F0400884646
:10AC30002DED048B87B020D0B8F1000F1DD0A16995
:10AC40004FF02C0A207FDFF808940E79E0B194F8D9
:10AC5000D01004F2744002903C30019004F28C60F9
:10AC60009FEDFC8A009041B34FF0000B9FEDFA9AE4
:10AC700001297CD002297BD14DE14FF0FF3007B094
:10AC8000BDEC048BBDE8F08F0025574608E000BFFF
:10AC900005EB850107EB41010844FEF721FD6D1C22
:10ACA000A069B542F4DB6830FEF71AFD94ED490A5D
:10ACB00084ED680A89ED020AFEE000252BE000BF62
:10ACC000C5EB051004EB800000F5D2708346FFF75A
:10ACD000C3FAB0EE480A04EB85075846D4ED041ACF
:10ACE000D7ED3E0AB0EE401AFFF7ACF987ED4C0AFB
:10ACF00004EB451087ED580A00F2AC50FEF736F928
:10AD000005EB850187ED5E0A0AEB4100A169084465
:10AD1000FEF7ECFC6D1CB542D2DB0298D4ED041AB0
:10AD2000D4ED490AB0EE481A99ED020AFFF78AF904
:10AD300084ED640A0198D4ED041AD4ED4B0AB0EE08
:10AD4000481AFFF77FF984ED650A0098FEF70EF9BF
:10AD500084ED660AA0696830FEF7C8FC98F8010027
:10AD600000280ED02046FFF7CFFE204601E009E084
:10AD7000A0E0FFF711FF2046FFF734FF012084F821
:10AD8000D00099E0002765E007EB87000590A169F6
:10AD9000342202EB4002D4ED670A04920823885C57
:10ADA000401EC0B203EB80000844F9B290ED000AE7
:10ADB000204620EE200AC0EE099AFFF7A5FCC7EB5B
:10ADC000071004EB8705F0EE408AD4ED041AD5EDA8
:10ADD0003E0A04EB80000390B0EE481AB0EE690A18
:10ADE00000F5D270FFF72EF985ED4C0AA169049A9F
:10ADF0000398D4ED041AD5ED3E0A895C00F5437042
:10AE0000B0EE481A04EB810191ED430AFFF71AF9FD
:10AE100020EE280A05F5A47105F5987085ED520A13
:10AE2000FFF757FC95ED4C0AD5ED520A04EB47109D
:10AE300000F2AC5030EE200A85ED580AFEF796F885
:10AE400085ED5E0A0598A2690AEB40001044FEF702
:10AE50004DFC7F1CB74297DB02984D46D4ED041A97
:10AE6000D4ED490AB0EE481A99ED020AFFF7EAF864
:10AE700084ED640A0198D4ED041AD4ED4B0AB0EEC7
:10AE8000481AFFF7DFF884ED650A0098FEF76EF8C0
:10AE900084ED660AA0696830FEF728FC98F8010086
:10AEA00010B12878E8B107E02046FFF72DFE2046D4
:10AEB000FFF798FE84F8D0B0A0692C30FEF70EFBA7
:10AEC000A0694168042902D95430FEF707FBA06944
:10AED0006830FEF703FB98F80210002089F8001094
:10AEE000CDE698F802000128E6D1207F022184F8FF
:10AEF000D010012806D0022802D0032808D104E08F
:10AF0000A069808BA4F82001D6E741F60A20F9E772
:10AF1000A4F820B1D0E741462046FFF72FFC0027D8
:10AF200065E007EB87010591A269342000EB410140
:10AF3000D4ED670A04910823505CF9B2401EC0B2F8
:10AF400003EB8000104490ED000A204620EE200A1A
:10AF5000C0EE099AFFF7D8FBC7EB071004EB870593
:10AF6000F0EE408AD4ED041AD5ED3E0A04EB8000E1
:10AF70000390B0EE481AB0EE690A00F5D270FFF700
:10AF800061F885ED4C0AA26904990398D4ED041A7E
:10AF9000D5ED3E0A515C00F54370B0EE481A04EB63
:10AFA000810191ED430AFFF74DF820EE280A05F5DF
:10AFB000A47105F5987085ED520AFFF78AFB95EDAF
:10AFC0004C0AD5ED520A04EB471000F2AC5030EEBB
:10AFD000200A85ED580AFDF7C9FF85ED5E0A05993F
:10AFE000A2690AEB41001044FEF780FB7F1CB742C8
:10AFF00097DB0298D4ED041AD4ED490A94ED680A5F
:10B00000B0EE481AFFF71EF884ED640A0198D4EDFB
:10B01000041AD4ED4B0AB0EE481AFFF713F884ED8A
:10B02000650A0098FDF7A2FF84ED660AA069683002
:10B03000FEF75CFB98F8020000287FF43DAE01208B
:10B0400084F8D00094ED490A89ED020A60E7000017
:10B05000AC0300240000000000C0DA4510B1017705
:10B06000002070474FF0FF30704700002DE9F04797
:10B0700004002DED028B0BD0A0690025DFF880A124
:10B080004FF07E59B7EE008AFFEE008A06794AE05B
:10B090004FF0FF30BDEC028BBDE8F08705EB850873
:10B0A000A2692C2101EB4807D019FEF777FBA069B4
:10B0B0003844FEF798FA30B12C3004EB05172037EE
:10B0C0000FC887E80F0004EB051104EB451091ED64
:10B0D000090A00F2EC40FDF749FF9FED4A1A04EB24
:10B0E0008500C0EE010A80ED380A10EE901AC0ED1E
:10B0F0003E0A494501DD80ED3E8AD0F8F810514501
:10B1000001D9C0ED3E8AA2693421D0ED3E0A01EB9F
:10B1100048006D1C105C04EB800090ED430A30EE9B
:10B12000200A80ED430AB542B8DB00EE106A94EDC8
:10B13000451AF6EE000AB8EE400AC1EE001A21EEFA
:10B14000A00A84ED450AA0696830FEF727FBA069D4
:10B150006830FEF748FA5022014604F18000F5F706
:10B16000A0FAA06994ED321A9FED270AD0ED040AE7
:10B1700060EE810A02E000BF70EE800AC4ED490A69
:10B18000F5EEC00AF1EE10FAF6D3204910EE900A5F
:10B19000884204DB70EEC00AC4ED490AF6E794F871
:10B1A000A80018B130EE600A84ED490A94ED230A34
:10B1B00004F26C60FDF7DAFE154884ED4A0AD4ED1E
:10B1C000230A90ED011A80EE810A10EE100A84ED38
:10B1D0004B0A484501DD84ED4B8AD4F82C015045DB
:10B1E00001D9C4ED4B8A94ED090AD4ED0D0A04F59A
:10B1F0008064002030EE600A84EDAB0A4AE700006C
:10B20000000080BF00C0DA45DB0FC940DB0FC9403A
:10B21000AC03002410B502F0EFFDBDE8104002F0D1
:10B2200035BE000010B5094C607808B1002010BD93
:10B23000032200204FF48071F6F754FB10B14FF059
:10B24000FF3010BD01206070F0E70000BC0000245A
:10B250000B4810B596B04FF0FF34407838B100235A
:10B260006A464FF480711846F6F7F8F910B1204697
:10B2700016B010BD0DF10D0003F0C4FA0020F7E781
:10B28000BC0000244FF0E02010B5006904F0A0FBE2
:10B29000012803D0BDE8104003F04CBE10BD0000F3
:10B2A00030B59DB04C216846F5F757FA202113A818
:10B2B000F5F753FA0220FAF717FD1D48016821F44B
:10B2C000404101600168002401F440411B91016884
:10B2D0008904FCD502200A9014230990C20301219D
:10B2E0000C25CDE90012CDE90B03CDE90D10CDE918
:10B2F00010540F9068461294FBF752FD08B172B6D5
:10B30000FEE713AD40203F21032285E8160003012C
:10B310001146CDE916401A90CDE9180313A8FBF7A2
:10B3200001FB002801D072B6FEE71DB030BD000061
:10B33000184802582D48F0B52D4A016841F47001B3
:10B340000160106800F00F00072804D2106820F098
:10B350000F00C01D106027490020264C10340B68D8
:10B36000254D43F001030B6020600B682B400B6000
:10B37000136803F00F03072B04D9136823F00F039E
:10B38000DB1D13601B4C1D4A18341D4B261D371D39
:10B390002060184C1B4D28343060261D3860371D46
:10B3A00023603B1D35601C1D3A60251D2E1D186055
:10B3B000331D22602860326018600B680D4A0D4C06
:10B3C00023F48023D4320B60603420601068C00402
:10B3D0000BD4136843F2D2000B4943F4805313603B
:10B3E0000860106820F480501060F0BD88ED00E027
:10B3F00000200052004402587FEDF6EA800201016D
:10B40000000202020000FF01004000520148FCF768
:10B41000F0BF0000D00900242DE9F0472C4B4FF07D
:10B42000804A2C4D026898422B4E2C4F2C4C09D050
:10B43000504507D0A84205D0B04203D0B84201D051
:10B44000A04205D1D1F804C022F070024CEA0202F9
:10B45000DFF890C0DFF890809842DFF8909015D028
:10B46000504513D0A84211D0B0420FD0B8420DD0F1
:10B47000A0420BD0604509D0404507D0484505D0D3
:10B480001B4DA84202D01B4DA84203D1CD6822F427
:10B4900040722A438E684D6922F08002C6620E68AF
:10B4A0002A439842866207D0A04205D0604503D067
:10B4B000404501D0484501D1096901630368012174
:10B4C00043F00403036041610260BDE8F0870000BF
:10B4D000000001400004004000080040000C004053
:10B4E0000004014000400140004401400048014088
:10B4F00000E0004000E4004010B5046A012301F0C0
:10B500001F018B409C4304628A40016A114301621F
:10B5100010BD42EA032283680A4323F47F410A43B1
:10B5200082607047034B82681A400A4342F0070169
:10B53000816070478FFFCFFF2DE9F04FDFF88480E7
:10B54000214EDFF88890DFF888B0026A036AB042C3
:10B55000DFF880A022F0020C1F4F23F001020262EC
:10B56000426885698B680C6805EA080525F00305C3
:10B5700043EA0C0344EA050407D0484505D0584582
:10B5800003D0504501D0B84205D1CD6823F008035F
:10B590001D4325F00403B04207D0484505D0584567
:10B5A00003D0504501D0B84205D122F44076D1E90C
:10B5B000055235432A43426084614968416303620E
:10B5C000BDE8F08F8FFFFEFF000001400004014046
:10B5D000004001400044014000480140F0B5DFF860
:10B5E0007CE01F4C1F4D026A036AA04222F0200635
:10B5F00023F01003036242688369D1F808C00F6822
:10B6000003EA0E0323F4407E46EA0C134EEA0726B3
:10B6100001D0A84206D1CF6823F0800343EA071384
:10B6200023F04003A0420AD0A84208D00E4CA0420A
:10B6300005D00E4CA04202D00D4CA04207D1D1E95A
:10B64000054522F4406242EA840242EA85024260F1
:10B650008661496881630362F0BD0000FF8FFFFED1
:10B66000000001400004014000400140004401404E
:10B6700000480140F0B5DFF87CE01F4D1F4E026A24
:10B68000036AA84222F4007723F4807303624368BC
:10B69000C269D1F808C002EA0E020C6822F0030E5B
:10B6A00047EA0C2244EA0E0401D0B04206D1CF682A
:10B6B00022F4006242EA072222F48062A8420AD001
:10B6C000B04208D00E4DA84205D00E4DA84202D07F
:10B6D0000D4DA84207D1D1E9055623F4405343EA62
:10B6E000051343EA06134360C4614968C1630262FB
:10B6F000F0BD00008FFFFEFF00000140000401408C
:10B70000004001400044014000480140F0B5046A97
:10B71000026A22F4805202624268C36924F400542F
:10B72000DFF848C08E680D6803EA0C03104F23F45D
:10B73000407344EA0634B84243EA05230BD00D4D6A
:10B74000A84208D00C4DA84205D00C4DA84202D00A
:10B750000B4DA84204D14D6922F4804242EA851281
:10B760004260C361496801640462F0BDFF8FFFFE5F
:10B77000000001400004014000400140004401403D
:10B7800000480140F0B5164F164B026A046A984211
:10B7900022F4003524F4803303624268436D0E893D
:10B7A0000C6803EA070344EA030445EA06430BD0A6
:10B7B0000D4DA84208D00D4DA84205D00C4DA84211
:10B7C00002D00C4DA84204D14D6922F4803242EAE5
:10B7D000052242604465496881650362F0BD00004E
:10B7E0008FFFFEFF000001400004014000400140C7
:10B7F0000044014000480140F0B5164F164B026A64
:10B80000046A984224F48013036222F4001442680C
:10B81000436D0E890D6803EA070344EA065443EAC0
:10B8200005230BD00D4DA84208D00D4DA84205D0E0
:10B830000C4DA84202D00C4DA84204D14D6922F40F
:10B84000802242EA8522426043654968C1650462FC
:10B85000F0BD0000FF8FFFFE00000140000401402A
:10B8600000400140004401400048014010B5036A17
:10B87000046A23F00A0324F00104046284690B4380
:10B8800024F0F00141EA02118161036210BD10B59C
:10B89000036A046A23F0A00324F01004046284699C
:10B8A00043EA011124F4704343EA023282610162E7
:10B8B00010BD000010B502F0A7F8314A0021314850
:10B8C00002F09CFA304C0021304A2060304802F0EF
:10B8D00095FA606000212F4A2F4802F08FFAA0608D
:10B8E00000212E4A2E4802F089FAE06000212D4AFC
:10B8F0002D4802F083FA206100212C4A2C4802F0E6
:10B900007DFA606100212B4A2B4802F077FAA06192
:10B9100000212A4A2A4802F071FA0022E0610A2135
:10B92000022002F0F3F8002220625821032002F0E6
:10B93000EDF80022E0630421022002F0E7F8002283
:10B94000E0621021032002F0E1F80022A062182139
:10B95000022002F0DBF8002220630C21022002F01A
:10B96000D5F8002260630321022002F0CFF8A06323
:10B9700002F07CF802F040FABDE8104002F086BA0E
:10B98000C401010871BE000888CC0024E801010848
:10B99000C5B900080C0201087DBB0008300201088F
:10B9A00071BC00085402010845BD00087802010876
:10B9B000F1BD00089C020108B9BB0008C0020108E3
:10B9C000F1BE000802F00BF800EE100A9FED631BB9
:10B9D0000020B8EE400B80EE012BBCEEC20B10EE47
:10B9E000106A01F0C0FF01F0F3FF5E4905465E48B2
:10B9F000F5F7CCFB5C48F5F7A9FB5B494431A1F1B5
:10BA00001400F4F785FF5848F5F7A0FBF0EE400A64
:10BA1000B7EE001A5448002181EE200A534A5C30E8
:10BA2000FEF7C4FB0020F6F7A1F951490020F6F714
:10BA300065F90020F6F742F9DFF82CA1494C4D4F8B
:10BA4000AAF1100A241FD1460AF180083544F5F7FF
:10BA5000F9FCF5F769FBF5F773FBF5F785FBF5F7EF
:10BA60008FFB01F0D1FF4048F5F726FC3E48F5F783
:10BA700073FC2078012841D13B499AED000AD1EDB1
:10BA8000070A70EE201ACAED001A9AED010AD1EDEC
:10BA9000080A70EE200ACAED010A91ED090A9AED32
:10BAA000021A41F2883131EE001A8AED021A6088DA
:10BAB000401C80B26080884230D32A4800219FED2C
:10BAC0002E0A81EE802AC0EE801A80ED002AC1EE97
:10BAD000000AC0ED011AC0ED020A21700146224899
:10BAE000F5F754FB2048F5F731FB1F494431A1F12C
:10BAF0001400F4F70DFF207801280FD01A4B4433BF
:10BB0000A3F12802A2F10C0101F12000F4F796FF45
:10BB10001549303101F12000F4F792FE01F0A6FF43
:10BB200009F1600208F1340092E80C1080E80C1072
:10BB3000D9E90B23D9F8341040E90323C8F83010B1
:10BB4000386B02F043F808490023386B1A469831E5
:10BB500002F008F8284601F014FF77E70000000023
:10BB600000408F402C040024D8BD0024800101082F
:10BB7000D5E7000888CC002400409C4501F02FFF49
:10BB800000EE100A9FED0A1B0020B8EE400B80EE7D
:10BB9000012BBCEEC20B10EE105A01F0E4FE01F0D6
:10BBA00017FF04462C44204601F0EBFEFAE70000A4
:10BBB000000000000000594001F011FF00EE100AE3
:10BBC0009FED261B0020B8EE400B80EE012BBCEE53
:10BBD000C20B10EE10AA01F0C6FE01F0F9FE0746F6
:10BBE000F6F772FF00F52E711E48F6F7CBFB1D4CE1
:10BBF0001D4D1E4E04F1800904F19408A134194929
:10BC00000023E86B58391A46574401F04DFF154898
:10BC1000F6F787FCC6F80880C6E90049686B01F0B2
:10BC2000D5FF0023686BB1681A4601F09BFFA86B33
:10BC300001F0CCFF0023A86B31681A4601F092FF97
:10BC4000A86A01F0C3FF0023A86A71681A4601F0D0
:10BC500089FF384601F095FED1E7000000000000A2
:10BC600000407F40E0BE002488CC0024380400243B
:10BC70002DED028B01F0B3FE00EE100A9FED2A1BA2
:10BC80000020B8EE400B80EE012BBCEEC20B10EE94
:10BC9000106A01F068FE01F09BFE0446F6F714FFFF
:10BCA0009FED238A00F5F47105462248B0EE480A5C
:10BCB000F6F792FD204805F51A71B0EE480A00F03B
:10BCC000B9F91C481C4F9FED1D0A1D4D143F80ED16
:10BCD0000C0A0023394634441A46E86A01F0E4FEAF
:10BCE00015490023A86A1A46103901F0DDFE1148F3
:10BCF000F6F778FE01F06CFE0F4902460D48103948
:10BD0000F6F734FC0B48F6F7FFFD0B4800F0CDF9D1
:10BD10000849094800F01AF9074800F0ADF9204633
:10BD200001F02FFED5E700000000000000407F403A
:10BD30000000FA4388BF002478C2002485EB113F3D
:10BD400088CC002401F04BFE00EE100A9FED221B70
:10BD50000020B8EE400B80EE012BBCEEC20B10EEC3
:10BD6000106A01F000FE01F033FE0546F6F7ACFE66
:10BD70009FED1B0A00F5A0711A48F7F7D1FC1A4C89
:10BD80001A4F0023194935441A46206B203101F01F
:10BD90008BFE20B9154913482031F7F7D3FD13491D
:10BDA0000023606B1A46383101F07EFE0D48F7F72C
:10BDB000A5FD0023E06A1A46394601F0D3FE0B497F
:10BDC00008483831F7F74EFB0648F7F719FD2846C3
:10BDD00001F0D7FDD5E700000000000000407F40E3
:10BDE0000000FA43B8C3002488CC002438C50024DE
:10BDF00001F0F5FD00EE100A9FED171B0020B8EED4
:10BE0000400B80EE012BBCEEC20B10EE105A01F07D
:10BE1000AAFD01F0DDFD0446F6F756FE9FED100A7F
:10BE200001461048FEF748FD0F4E104F00230F4902
:10BE30002C441A46B06B01F037FE0A48FFF716F99A
:10BE400039780848FFF70AF908490648FEF7FAFC6E
:10BE5000204601F096FDE9E70000000000407F4029
:10BE60000000FA4380C5002488CC00244404002448
:10BE700001F0B5FD00EE100A9FED191B0020B8EE91
:10BE8000400B80EE012BBCEEC20B10EE105A01F0FD
:10BE90006AFD01F09DFD04461348F7F747F8124884
:10BEA000F7F746F9114E14202C44F7F750F9002803
:10BEB0000D4802D0F7F766F801E0F7F755F8F06B98
:10BEC00001F084FE00230849F06B1A4601F04AFE97
:10BED0000548F7F72DF9204601F053FDE3E7000090
:10BEE0000000000000407F4030CC002488CC0024BB
:10BEF00001F075FD00EE100A9FED111B0020B8EE59
:10BF0000400B80EE012BBCEEC20B10EE105A01F07C
:10BF10002AFD01F05DFD0446FFF784F90A4801217E
:10BF20007822017041708270C1702C44FFF790F943
:10BF30000548F5F7F1FF204601F023FDF5E7000085
:10BF40000000000000407F4047040024F0B50400DA
:10BF50000E462DED048B83B034D0F5F78CFF03F043
:10BF6000ACFF00EE100ADFED308A80EE288A84ED07
:10BF7000028AD4E9040103F0A0FF00EE100AC0EE2B
:10BF8000280A38EE600A84ED060AF5F774FFC4E962
:10BF90000401307C9FED258A022815D0032813D098
:10BFA0005FF0000004EB8001401C022881ED4E8A06
:10BFB000F8DB04F12000FEF739F9002003B0BDECF6
:10BFC000048BF0BDFF20F9E79FED199A00256F461D
:10BFD000F6EE008A06EB051007EB850190EDA80A46
:10BFE000D0EDAC0A05EB8500B0EE481A30EE200A21
:10BFF00004EB001020EE280A20EE090A81ED000A69
:10C00000C5EB0511D0ED290A04EB81002030D4EDF9
:10C01000061AFEF717F804EB85006D1C022D80ED63
:10C020004E0AD7DBC9E70000002474490000000075
:10C030008FC2F53C70B506000D462DED028BB0EEBB
:10C04000408A17D0B5B10024C6F800500121C4EBD6
:10C05000041005EB441206EB800020301032B0EEE5
:10C06000480AFEF7A3F8641C022CEFDB0020BDECAD
:10C07000028B70BDFF20FAE770B5050013D00024D5
:10C08000286805EB840100EBC40091ED4E0AFDF732
:10C090002DFB286800EBC400FDF720FA641C022C7D
:10C0A000EEDB002070BDFF2070BD70B5050018D01C
:10C0B0000024286800EBC400FDF770FB286800EB43
:10C0C000C400FDF790FA014604EB8400502205EB12
:10C0D00000109830F4F7E5FA641C022CE9DB00202C
:10C0E00070BDFF2070BD00000148FCF743BC00009C
:10C0F000C408002430B5416EB9B101680D4B03F19D
:10C1000008048A688968C2F34262490F5D5C615C19
:10C110002D01B5FBF1F1A0F86A10995CA25C090150
:10C12000B1FBF2F1A0F8681030BD0121A0F86A104F
:10C13000F8E700005000010890F82810090706D51C
:10C140000168836B4A6822F400421A434A6090F8FF
:10C150002810C90706D00168C36A4A6822F4003271
:10C160001A434A6090F82810890706D50168036BC6
:10C170004A6822F480321A434A6090F8281049072E
:10C1800006D50168436B4A6822F480221A434A604C
:10C1900090F82810C90606D50168C36B8A6822F496
:10C1A00080521A438A6090F82810890606D50168E3
:10C1B000036C8A6822F400521A438A6090F82810AF
:10C1C000490611D50168436C4A6822F480121A436B
:10C1D0004A60416CB1F5801F06D10168836C4A68E2
:10C1E00022F4C0021A434A6090F82810090606D5C6
:10C1F0000168C26C486820F4002010434860704712
:10C200002DE9F84300250446C0F89050F9F788FC62
:10C210008046206820266FF07E470068000713D50F
:10C220000022434631042046009700F04DFB58B1F0
:10C23000216851E8000F20F0800041E80002002A48
:10C24000F6D1C4F8886021E020680068400722D554
:10C25000002243464FF480012046009700F034FB53
:10C26000C8B1206850E8001F21F4907140E8001226
:10C27000002AF6D12068083050E8001F21F00101A3
:10C2800040E80012002AF5D1C4F88C60032084F83D
:10C290008450BDE8F883C4F88860C4F88C60E56613
:10C2A0002567002084F88450F3E710B5806B0021E7
:10C2B000A0F85E10FCF74AFB10BD70B5846B00253A
:10C2C0002168D4F88800D4F88C608968090606D5FE
:10C2D000212804D1A4F85650204600F091F8206897
:10C2E0008068400606D5222E04D1A4F85E50204670
:10C2F00000F05CF8D4F8900040F01000C4F8900012
:10C300002046FCF723FB70BD10B5C1690022806B8D
:10C31000B1F5807F2DD0A0F85E20036853E8001FA0
:10C3200021F4807143E80014002CF6D10168083133
:10C3300051E8003F23F0010341E80034002CF5D11F
:10C340000168083151E8003F23F0400341E8003420
:10C35000002CF5D12021C0F88C10C16E012908D124
:10C36000016851E8003F23F0100341E80034002C3D
:10C37000F6D10267C16E012902D0FCF79BFD10BD0A
:10C38000B0F85C10FCF792FA10BD10B5806B01217B
:10C390000167C16E012902D0FCF7A0FD10BDB0F805
:10C3A0005C104908FCF782FA10BD000010B5026865
:10C3B00052E8001F21F4907142E80013002BF6D1DF
:10C3C0000E4B0268083252E8001F194042E8001480
:10C3D000002CF6D1C16E012908D1026852E8001F75
:10C3E00021F0100142E80013002BF6D10021202299
:10C3F000C0F88C20C166416710BD0000FEFFFFEF52
:10C40000026852E8001F21F0C00142E80013002B2F
:10C41000F6D10168083151E8002F22F4000241E80A
:10C420000023002BF5D12021C0F8881070470000B0
:10C4300000680349884201D10020704702207047FC
:10C44000005000402DE9F04304468068E24E87B07A
:10C45000E24B2168D4E90427D4F81CC010430A68D1
:10C46000002547EA0C073843324002430A6020683F
:10C47000E268416821F44051114341602268A1699A
:10C480009A4201D0206A01439668DFF854C3D54F21
:10C49000D54806EA0C060E4396602168666ACA6AA9
:10C4A00022F00F023243CA622268BA420ED10068FB
:10C4B00000F0380018286FD07ADCB8B308286CD0A8
:10C4C00010286BD18BE0282868D18EE0C7498A42BA
:10C4D00009D1006800F0070006285FD2DFE800F00D
:10C4E000507D7F818385C2498A4209D1006800F06E
:10C4F000070006287BD2DFE800F04370727476787C
:10C50000BC498A4209D1006800F0070006286ED2B3
:10C51000DFE800F036636567696BB7498A420BD183
:10C52000006800F00700062861D200E043E0DFE881
:10C5300000F0275456585A5CB0498A4206D1006828
:10C5400000F0380018284CD0B7DD31E0AC498A4201
:10C5500009D1006800F00700062848D2DFE800F0A3
:10C56000103D3F414345A7498A420BD1006800F086
:10C57000070006283BD2DFE800F0033032343638BB
:10C58000002035E0A0498A4209D1006800F0380057
:10C59000182826D091DD0BE023E01EE027E09B4920
:10C5A0008A420AD1006800F03800182819D084DDCA
:10C5B000202888D11CE001201AE09A4217D18A482D
:10C5C000001D006800F00700062810D2DFE800F028
:10C5D000030507090B0D02200AE0042008E00820EB
:10C5E00006E0102004E0202002E0402000E080204F
:10C5F0008749DFF820829A42874A4FF400434FEA86
:10C6000021174FF000064ED110281AD006DC022860
:10C6100009D004280BD008287ED10DE020283ED078
:10C62000402879D13DE0F9F789FB014610E06846E2
:10C63000F9F796FB01990BE003A8F9F733FC04998D
:10C6400006E01068800605D51068C0F3C100C1403F
:10C65000002970D0606A676838F8102007EB47033C
:10C66000B1FBF2F0834257D8B0EB073F54D8002318
:10C6700008461946F3F73AFF02467808130E1202ED
:10C6800043EA012110183A4671410023F3F72EFFC7
:10C69000624AA0F5407191423ED821688FE0394648
:10C6A000D8E71946D6E7D4F81CC04FF6EF799C4579
:10C6B00046D1082819D005DC58B101280CD004282F
:10C6C00075D10DE0102815D0202835D040286ED126
:10C6D00034E0FAF7A5FA01E0FAF7B4FA014610E0FF
:10C6E0006846F9F73DFB01990BE003A8F9F7DAFB7F
:10C6F000049906E01068800604D51068C0F3C100F4
:10C70000C140C1B1636A606838F81330B1FBF3F11E
:10C71000490001EB500100E049E0B1FBF0F0A0F16D
:10C720001001494543D84FF6F0732168C0F3420227
:10C730001840104343E043E03946E3E71946E1E798
:10C74000082819D005DC58B101280CD004282ED1B6
:10C750000DE0102815D020282BD0402827D12AE022
:10C76000FAF75EFA01E0FAF76DFA014610E0684662
:10C77000F9F7F6FA01990BE003A8F9F793FB04998E
:10C7800006E01068800604D51068C0F3C100C140FF
:10C79000B1B1636A606838F81330B1FBF3F101EBB3
:10C7A0005001B1FBF0F0A0F11001494505D9012578
:10C7B00006E03946EDE71946EBE7216880B2C8602C
:10C7C0000120A4F86A00A4F8680028466667A667F6
:10C7D00007B0BDE8F0830000F369FFCF000C0058FC
:10C7E000FFF4FF110010014054440258004400407F
:10C7F00000480040004C0040005000400014014040
:10C8000000780040007C004000180140001C0140FE
:10C810000090D0033800010800440258FFFC0F00CC
:10C8200070B50446D0F8800000232225A165A4F845
:10C830005C20C4F89030C4F88C50F0B11F49C1633B
:10C84000D4F880101E480864D4F880101D48C864CD
:10C85000D4F8800003651346A56D2168D4F88000E4
:10C860002A462431F8F7C6F838B11021C4F89010E0
:10C870002020C4F88C00012070BD206940B12168DF
:10C8800051E8000F40F4807041E80002002AF6D120
:10C890002068083050E8001F41F0010140E8001214
:10C8A000002AF5D12068083050E8001F41F040010F
:10C8B00040E80012002AF5D1002070BD09C300082D
:10C8C0008BC30008BBC200082DE9F0479946174604
:10C8D0000D460446089E4FF0000833E0701C31D02E
:10C8E000F9F71EF9A0EB0900B04218D8BEB12068D4
:10C8F0000168490726D5802D24D0402D22D0C1695A
:10C90000C94309070DD4082505622046FFF74EFDEF
:10C91000C4F89050012084F88480BDE8F08703209B
:10C92000FBE7C069C04300050CD421684FF40060E8
:10C9300008622046FFF73AFD2021C4F8901084F8E1
:10C940008480ECE72068C06935EA000004D000204C
:10C95000B842C3D00020E0E70120F9E7FEE703B4C6
:10C9600001984100009850EAC12018BF04204A0DE8
:10C9700018BF40F0010040F2FF72B2EB515F08BFF8
:10C9800040F00200012808BF052002B070474100B6
:10C99000080218BF04200A0E18BF40F001004FF033
:10C9A0007F4232EA010108BF40F00200012808BFBF
:10C9B000052070476FEAD05010F0FF0000D0012032
:10C9C0007047090700284FEA116104DB00F1E020FD
:10C9D00080F80014704700F00F0000F1E02080F8AC
:10C9E000141D704710B54FF00E402DED028BB0EEC8
:10C9F000408A18EE104A00EB4400B0F1506F4AD85C
:10CA00004FF0FC40B0EB440F22D2B0EEC80ADFED8D
:10CA1000360A30EEC00ADFED350A60EE208A18EEE5
:10CA2000900A01F0B7FE01EE100A14F0004F1DBF8E
:10CA3000DFED2F0A9FED2F0AB1EE411ADFED2E0A2E
:10CA400008BF9FED2E0ADFED2E1A21EE218A05E0A8
:10CA5000DFED2C0A68EE088AB0EE600A9FED2A1A14
:10CA6000DFED2A1A30EE080A48EE811A9FED281AE7
:10CA700008EEA11ADFED271A48EE811A9FED261A5B
:10CA800008EEA11A68EE281ABDEC028B01EE810AAD
:10CA900030EE200A10BD4FF0E440B0EB440F0CD94B
:10CAA00018EE100AFFF773FF042808BF00F026FEF7
:10CAB000B0EE480ABDEC028B10BD4FF07F40B0EBEA
:10CAC000440F07D2B0EE480ABDEC028BBDE810401F
:10CAD00000F006BE0120F3F76FFEBDEC028BBDE84F
:10CAE000104000F003BE00000000803F0000003F47
:10CAF0000000C9BF22AAFDB90000C93F22AAFD3922
:10CB0000000000C00000000024FE1C3DC78AD83C85
:10CB10001E67383D1B93993DAFAA2A3E00000000D6
:10CB200070B565482DED020B2DED048B059D25F0AC
:10CB30000044A04218DC6148844202DC0AD1049817
:10CB400040B19DED040BBDEC048B02B0BDE870401C
:10CB500000F0B2BD002DCCBF9FED590B9FED5A0BDD
:10CB6000BDEC048B02B070BD5948A04215DD594898
:10CB7000A042D8BF4FF0FF3455DD9DED040B51ECC2
:10CB8000100BFFF7ECFE042808BF00F09DFD9DEDA3
:10CB9000040BBDEC048B02B070BD9DED040B51EC99
:10CBA000100B00F09FFECDE904014B489FED4C0BAC
:10CBB000A0421CDD4C48A0420BDD9DED042B00245F
:10CBC0009FED4B1B12EE010B32EE011B80EE012B91
:10CBD00027E09DED041B9DED042B012431EE401B4D
:10CBE00032EE000B81EE002B8DED042B1BE0424852
:10CBF000A0420FDD9DED042B02249FED411B9DED16
:10CC0000043B32EE412B03EE010B82EE001B8DED57
:10CC1000041B08E09DED040B9FED3B1B032481EEFC
:10CC2000002B8DED042B9DED040B3948062120EEE1
:10CC3000009B29EE098BB0EE480B784400F004FD10
:10CC400020EE099B3348B0EE480B0521784400F0F4
:10CC5000FBFC20EE080B002C0BDA9DED042B39EECB
:10CC6000001B9DED040BBDEC048B02B002EE410BEA
:10CC700070BD2948784439EE000B00EBC4009DEDEF
:10CC8000042B90ED001B254812EE001B9DED040BBC
:10CC900031EE400B784400EBC400002D90ED001BFA
:10CCA00031EE400BB8BFB1EE400BBDEC048B02B0CF
:10CCB00070BD000000000000000010440000F07F84
:10CCC000182D4454FB21F93F182D4454FB21F9BF82
:10CCD0000000DC3F0000203E0000F33F00000000A9
:10CCE000000000000000F03F0000E63F00000000F0
:10CCF0000000000000000040008003400000000031
:10CD0000000000000000F83F000000000000F0BF3D
:10CD100012370000D8360000903600005036000070
:10CD200070B5614E2DED040B2DED048B82B0DDF856
:10CD300024C0DDE907235C422CF000411C4341EA9A
:10CD4000D474069D22F00040B44205D86C422C43B6
:10CD500040EAD474B4420BD99DED081B9DED060B3F
:10CD600002B0BDEC048B04B0BDE8704000F0A7BC7D
:10CD7000ACF14054A4F17F641C430BD0022404EABC
:10CD8000AC7444EAD27405439FED498B9FED4A2B66
:10CD90000DD016E09DED060B51EC100B00F060FD80
:10CDA00041EC100B02B0BDEC048B04B070BD002C44
:10CDB00014BF012C9DED060BF4D0022C2ED0032CB9
:10CDC0002FD00B439FED3E1B9FED3F0B0AD0B1428E
:10CDD0001DD1B04209D121F0804120F0804009915D
:10CDE000079014E0002ADDDA15E0394B7B44002C73
:10CDF00008BF93ED000BD5D0012C04BF93ED000BC1
:10CE0000B1EE400BCED0022C08D0032C09D0B0429A
:10CE10000AD1002AC6DAB0EE410BC3E7B0EE480BE8
:10CE2000C0E7B0EE420BBDE7401A00159FED2A9B0C
:10CE30003C28C8BF8DED000B15DCBCF1000FBCBF5A
:10CE400010F13C0F8DED009B0DDB9DED061B9DED64
:10CE5000082B81EE020B51EC100B00F043FD00F0AB
:10CE6000FFFCCDE9000194B1012C0CD09DED001B1D
:10CE70009FED1B0B022C31EE400B0CBF38EE400B2C
:10CE800030EE480B8EE7019880F0004001909DED58
:10CE9000000BB4EE490BF1EE10FA04BF0220F3F7D9
:10CEA0008BFC9DED000B7DE70000F07F0000000093
:10CEB000182D4454FB210940182D4454FB2109C06E
:10CEC000182D4454FB21F9BF182D4454FB21F93F80
:10CED000903500000000000000000000000000008D
:10CEE000075C143326A6A13C70B54FF068422DEDC7
:10CEF000048BF0EE408A18EE900AB0EE608A18EECD
:10CF0000101A02EB4003B3F1654F3CBF02EB410244
:10CF1000B2F1654F7DD200BFC0F3C753C1F3C75212
:10CF20009A1A1B2A09DD10F0004F14BF9FED830AE7
:10CF30009FED830ABDEC048B70BD12F11A0F36DA37
:10CF400011F0004F09D010F0004F0CBF9FED7D0A8B
:10CF50009FED7D0ABDEC048B70BD88EE889A19EEBA
:10CF6000100AFFF714FD042808BF00F0C7FB18EEF5
:10CF7000900AFFF70CFD054618EE100AFFF707FDB3
:10CF8000044619EE100AFFF702FD042D18BF052D07
:10CF900008D1042C18BF052C04D1002804BF02209E
:10CFA000F3F70AFCB0EE490ABDEC048B70BD4200F9
:10CFB000B2EB410F3AD910F0004F19BFDFED630A11
:10CFC0009FED630ADFED630A9FED630AB0EE481A36
:10CFD0000A46B1EE688A80F00041F0EE418A1046C0
:10CFE0000A1A5200B2F1807F34D2484010F0004F4C
:10CFF000DFED5A1A9FED5A2A1DBF9FED5A1A70EEA7
:10D00000E10A30EE420A9FED581A08BF70EEA10AFD
:10D0100000E040E008BF30EE020AB0EE682A01EE00
:10D02000482A08EE818AC2EE081A15E011F0004F76
:10D0300004BF9FED4E0AF0EE400AD1D010F0004F31
:10D0400019BFDFED4B0A9FED4B0ADFED4B0A9FED59
:10D050004B0AC5E7C8EE881A21EEA11A9FED482AAF
:10D06000DFED482A41EE022A9FED472A01EE222AEF
:10D07000DFED462A41EE022A9FED452ABDEC048BE6
:10D0800001EE222A21EE811A01EE020A30EE210A77
:10D0900030EE200A70BD4FF07F42B2EB400F28BF48
:10D0A000B2EB410F09D2F0EE480AB0EE680ABDECCF
:10D0B000048BBDE8704000F016BB40EA01035B0042
:10D0C00008BF41F0FF410BD0B2EB400F08BFB2EBFD
:10D0D000410F08D120F0804008EE900A21F08041F5
:10D0E00008EE101A18E7B2EB400F12BF5FEA4103D7
:10D0F00040F0FF4001F000413FF40EAFB2EB410FB2
:10D1000012BF5FEA400200F0004041F0FF413FF4EF
:10D1100003AF4A0092EA40033FF5FEAE002AACBFDF
:10D120009FED1C0A9FED1C0A68EE808A28EE008A9B
:10D1300018EE900A18EE101AEEE60000DB0FC9BFD9
:10D14000DB0FC93FDB0F4940DB0F49C00000C9BFFF
:10D1500022AAFDB90000C93F22AAFD390060ED3EB8
:10D16000C30ACE37000000BF0000003F00000000EF
:10D17000000049C022AA7DBA0000494022AA7D3A97
:10D180002DAD65BD8FB8D53D0FB511BE61C84C3E04
:10D19000A8AAAABE0000804F0000802F10EE101A2F
:10D1A00008B5434A6846B2EB410F26D94FF0E64036
:10D1B000B0EB410F94BF00204FF0FF30009000987B
:10D1C000DFED3C0A002860DB10F0010F46D060EE76
:10D1D000000ADFED391A9FED391A10F0020F00EE48
:10D1E000E11ADFED371A40EE811A21EEA01AF0EEB7
:10D1F000400A40EE010A2ED041E0324B21F00042BD
:10D2000093423FD911F0004FDFED2F0A20EE201A94
:10D21000DFED2E0A19BF31EE601A71EE200A31EEF1
:10D22000201A71EE600ABDEEE01A11EE100A9FEDB1
:10D23000281A00F0030000EEC10A9FED261A0090A4
:10D2400000EEC10A9FED241A00EEC10A9FED231AD9
:10D2500000EEC10AB3E7F1EE600A10E020EE000A2A
:10D260009FED1F1ADFED1F1A10F0020F40EE011A9A
:10D270009FED1D1A00EE211A40EE010AEBD1B0EE2F
:10D28000600A08BD00F042FA99E710EE100A40006B
:10D29000B0F17F4FF3D307D14FF00100F3F78CFAD1
:10D2A000BDE8084000F022BABDE8084000F018BA16
:10D2B000B61F927E0000803F336D4C39DA82083C05
:10D2C000A0AA2ABE490E494683F9223F0000004B1E
:10D2D0000000C93F00A0FD390020A2331A61342CA0
:10D2E000B93AB2BACA9F2A3DDDFFFFBE10B52DED97
:10D2F000028BB0EE608AF0EE408A18EE101A18EE3B
:10D30000900A02F0B1FD00F07040B0F1005F0CD067
:10D3100018EE100A20F00040C0F1FF40C00F02BF1D
:10D32000B0EE480ABDEC028B10BDB0EE680ABDEC51
:10D33000028B10BD00B510EE101A2DED028B81B0DE
:10D34000524A6846B2EB410F2ED94FF0E640B0EB9F
:10D35000410F94BF00204FF0FF3000900098B0EED6
:10D36000408A00286ADB10F0010F4BD068EE080AF3
:10D370009FED471A9FED470A00EE810A9FED461A7E
:10D3800000EE801A9FED450A10F0020F00EE810AB0
:10D3900002BF01B0BDEC028B00BD00BF01B0B1EE19
:10D3A000400ABDEC028B00BD3D4B21F00042934290
:10D3B00041D911F0004FDFED3B0A20EE201ADFEDDE
:10D3C0003A0A19BF31EE601A71EE200A31EE201AC6
:10D3D00071EE600ABDEEE01A11EE100A9FED331AED
:10D3E00000F0030000EEC10A9FED311A009000EE3C
:10D3F000C10A9FED301A00EEC10A9FED2F1A00EE10
:10D40000C10AABE728EE080A9FED2C1ADFED2C0AC3
:10D4100010F0020F40EE410A9FED2A1A00EE201A8A
:10D4200061EE000AB0EE480A08EE200AB6D101B05B
:10D43000BDEC028B00BD00F069F98FE718EE100A11
:10D440004000B0F17F4F0DD218EE100AFFF79FFA9F
:10D45000042808BF00F052F9B0EE480A01B0BDEC54
:10D46000028B00BD09D10120F3F7A6F901B0BDEC94
:10D47000028B5DF804EB00F039B901B0B0EE480A58
:10D48000BDEC028B5DF804EB00F02AB9B61F927E6A
:10D49000B93AB2BACA9F2A3DDDFFFFBE0000803F05
:10D4A000490E494683F9223F0000004B0000C93F66
:10D4B00000A0FD390020A2331A61342C336D4C39A1
:10D4C000DA82083CA0AA2ABE00B510EE101A2DED93
:10D4D000028B81B04D4A6846B2EB410F3CD94FF008
:10D4E000E640B0EB410F94BF00204FF0FF300090BA
:10D4F0000098B0EE408A00285FDB28EE080ADFEDD6
:10D50000440A9FED441A00EE201ADFED430A40EE74
:10D51000010A9FED421A00EE201ADFED410A10F0D9
:10D52000010F40EE010A9FED3F1A00EE201A61EE56
:10D53000000AB0EE480A08EE200A02BF01B0BDECB6
:10D54000028B00BD9FED381A01B0C1EE000ABDECA0
:10D55000028BB0EE600A00BD344B21F000429342D2
:10D5600028D911F0004FDFED320A20EE201ADFED4E
:10D57000310A19BF31EE601A71EE200A31EE201A1D
:10D5800071EE600ABDEEE01A11EE100A9FED2A1A44
:10D5900000F0030000EEC10A9FED281A009000EE93
:10D5A000C10A9FED271A00EEC10A9FED261A00EE70
:10D5B000C10A9DE700F0AAF89AE718EE100A4000A9
:10D5C000B0F17F4F0DD218EE100AFFF7E0F90428F2
:10D5D00008BF00F093F8B0EE480A01B0BDEC028B32
:10D5E00000BD09D10120F3F7E7F801B0BDEC028BD3
:10D5F0005DF804EB00F07AB801B0B0EE480ABDEC7B
:10D60000028B5DF804EB00F06BB80000B61F927E51
:10D61000BBE9223C0C6D063B8A76CE3CACB5593D4D
:10D6200035A1083E29AAAA3E000080BF490E4946FE
:10D6300083F9223F0000004B0000C93F00A0FD39E4
:10D640000020A2331A61342C491E00EBC102B0EE57
:10D65000401B92ED000B31F006020DD0491E00EB8D
:10D66000C102B0EE403B92ED002B31F00602B0EE6D
:10D67000420B03EE010BF1D1022914D004290AD088
:10D68000062918BF704790ED0A2B00EE012B90ED94
:10D69000080B02EE010B90ED062B00EE012B90ED36
:10D6A000040B02EE010B90ED022B00EE012B90ED2E
:10D6B000000B02EE010B704730EE000B704730EEAE
:10D6C000010B7047000000009FED030B20EE000BE4
:10D6D0007047000000000000000000000000001083
:10D6E00030EE000A704730EE200A7047DFED020A84
:10D6F00080EEA00A70470000000000009FED020AC3
:10D7000020EE000A70470000000000102DE9F00133
:10D710004FF07F42B2EB410F9FBF4FF0FF310160EE
:10D72000BDE8F00170474FF0004242EA0123C1F327
:10D73000C752783A551112F01F0C434CCCF1200619
:10D740007C44C1F3C752A2F178024FEA621204EBA3
:10D75000820254F8254008BFD2E9015612D055681C
:10D7600004FA0CF425FA06F73C43976805FA0CF521
:10D7700027FA06F8D26807FA0CFCF24045EA0805D9
:10D780004CEA0206A4FB034CA5FB0352A6FB036371
:10D790001D449D4234BF012600261319334416B19F
:10D7A000934202D903E0934201D2012200E0002219
:10D7B000624402F1200C9206DC0C42EA443200EE94
:10D7C000102A5B03DFED210AF8EEC01A00EE103AD2
:10D7D0004FEA9C1C11F0004FB8EE400AC0F800C0A0
:10D7E00020EE201A00EE105ADFED190AB8EE400ABA
:10D7F00020EE200A71EE810A70EE800A10EE902A67
:10D8000002F500626FF30B0200EE902A70EEE11A4F
:10D8100031EEC11ADFED101A30EE411A9FED0D0AFC
:10D8200020EE800A01EE210A9FED0C1A00EE810A1B
:10D8300004BFBDE8F0017047CCF180510160BDE844
:10D84000F001B1EE400A7047442C000000000036A1
:10D850000000802C22AAFD29DB0FC92F0000C92F50
:10D8600010B541EC100BFFF75BF951EC100B10BD3C
:10D870002DE9F041040006D0184E306884420AD1E8
:10D880000020BDE8F081502080F31188BFF34F8F56
:10D89000BFF36F8FFEE701F03FF8776B6569B66BFA
:10D8A00001F05AF8BD4201D0B54201D10220E8E7AB
:10D8B0000B48854208D1A06A0028F7D194F8580097
:10D8C0000128F3D00320DCE705481438854202D054
:10D8D0000DB10120D5E70420D3E700001C0000248F
:10D8E0000C0F002482B0CDE9000121F0004001902E
:10D8F0009DED000B02B051EC100B7047012170EE52
:10D90000601A8140491E31EE600A00EE901AF8EE6E
:10D91000E00A61EEA00A80EE801ABDEEC10A10EEA8
:10D92000100A7047F8F70AF9FDF7BAFCFCF7A0FCFB
:10D93000FCF76EF8FBF780FFFBF7ACFFFBF7DEFFB1
:10D94000FCF714F8FCF7E4F8FCF716F9FCF740F9DB
:10D95000FCF7DAF9FCF78AF900F044F8FCF73EF836
:10D9600000F068F8FEE710B5EFF3058111B16FF034
:10D97000050404E04FF0000408B101F0A5F82046CA
:10D9800010BD38B50546EFF3058010B16FF0050402
:10D990000CE0002402F02AF8291A0090002903DD87
:10D9A000684601F0B7F801E06FF00304204638BD87
:10D9B00010B502F00DF838B1022804D00348006811
:10D9C000012800D0002010BD032010BD6C000024F1
:10D9D000EFF3058008B102F00FB802F007B84FF47A
:10D9E0007A707047EFF3058010B16FF00500704753
:10D9F0000449086810B14FF0FF30704701220A60F7
:10DA0000002070476C00002410B5EFF3058010B1C2
:10DA10006FF0050010BD01F0DBFF20B1022804D03B
:10DA20004FF0FF3010BD012010BD01F0CFF90020F4
:10DA300010BD000010B5EFF3058010B16FF00500C8
:10DA400010BD08480168012902D04FF0FF3010BD19
:10DA5000054A002182F8141D0221016001F072F9CB
:10DA6000002010BD6C0000240BE000E070B5EFF367
:10DA7000058010B16FF0050413E001F0A9FF4FF02D
:10DA8000FF3510B102280BD108E0012402F01AF989
:10DA9000012806D001F09CFF10B102E0002400E054
:10DAA0002C46204670BD0000F8B56FF003021D46FD
:10DAB0006FF002064FF00004EFF30583A3B1F0B15D
:10DAC000E9B1E5B9002200926A4601F0CBFC0128D9
:10DAD00017D10098B0B10C494FF080500860BFF3E7
:10DAE0004F8FBFF36F8F0DE048B141B12A4601F06F
:10DAF0001BFC012806D025B16FF0010402E014469A
:10DB000000E034462046F8BD04ED00E0F8B51446C8
:10DB10004FF00005EFF3058212BB08B301B3A4B1C7
:10DB2000D4E9023263B1502A1AD32269C2B100FB90
:10DB300001F66769B74213D3009501F04AFA07E08E
:10DB400072B9226962B9626952B9002201F020FA01
:10DB5000050005D00CB1216800E0002100F07EFF37
:10DB60002846F8BDF8B56FF003021D466FF00206B7
:10DB70004FF00004EFF30583ABB100B3F9B1F5B991
:10DB80000022009213466A4601F050FB012818D18A
:10DB90000098B8B10C494FF080500860BFF34F8F28
:10DBA000BFF36F8F0EE050B149B100232A4601F058
:10DBB0008DFA012806D025B16FF0010402E0144669
:10DBC00000E034462046F8BD04ED00E010B5EFF368
:10DBD000058111B16FF0050404E028B1002421464D
:10DBE00001F02AFA204610BD6FF00304FAE72DE990
:10DBF000F0410D46014621F001004FF0000401F014
:10DC00000101EFF305820AB1A41F16E048B1002913
:10DC100029466FF001066FF0020708D001F02EFDD3
:10DC200007E06FF0030408E035B1344605E001F089
:10DC300067FC0128F8D100E03C462046BDE8F081B1
:10DC400070B505464FF00004EFF3058050BB0DB1F1
:10DC5000686800E00020C10701D0012600E000262E
:10DC600000071FD46DB1D5E9021021B1502819D396
:10DC70001EB1042002E020B114E0012001F07BF984
:10DC800005E00EB1042000E0012001F069F9040074
:10DC900008D00DB1296800E0002100F0DFFE0EB1D0
:10DCA00044F00104204670BD014670B521F001002A
:10DCB0004FF0000401F00101EFF305820AB1A41F47
:10DCC00011E028B16FF0020529B101F00EFB07E069
:10DCD0006FF0030407E000231A46194601F0F6F935
:10DCE000012800D02C46204670BD00003EB504003F
:10DCF00001D0002903DA6FF0030001902BE04FF010
:10DD0000FF300190EFF30580D0B10025029502A805
:10DD10002B4601220090204601F0D2FD0022204631
:10DD200001AB1146009501F0CBFD029898B10B496B
:10DD30004FF080500860BFF34F8FBFF36F8F0AE042
:10DD400000232046012201F04BFD0022204601ABBA
:10DD5000114601F045FD01983EBD000004ED00E0D4
:10DD60002DE9F84F894605464FEA0206EFF3058094
:10DD700010B16FF005041EE0002D02DA6FF003040D
:10DD800019E05FEA897002D54FF0000800E0A8466C
:10DD90009246002401F02AFEE71E834600205346E7
:10DDA0006A46414601F094FE012807D016B36FF091
:10DDB00001040028F2D12046BDE8F88F00982C40DD
:10DDC0005FEAC97144EA00040BD035EA0400F2D0DE
:10DDD00056B101F00BFEA0EB0B00504506D9002018
:10DDE00006E02542E7D1F3E73C46E4E7AAEB000072
:10DDF0008246D3E73C46DCE701F0E4BD2DE9FF4174
:10DE00004FEA01034FF00005EFF30581039561BB75
:10DE100058B34FF080064FF018014FF000044AB39A
:10DE2000176807B13C4697691FB139467F1E382FE6
:10DE300002D21779FF0703D0002004B0BDE8F081BB
:10DE4000576907B1BE08D2F808C0BCF1000F0DD069
:10DE5000D5685C2D18D312693AB137B18DE8061038
:10DE60003246214601F091FC03900DE0D7685FB97E
:10DE700012694AB903AACDE90012B2B2214601F0F3
:10DE800057FC012800D003950398D6E770B50546E6
:10DE9000EFF3058010B16FF005040FE04DB1284697
:10DEA000FFF7E6FC042807D00024284600F078FE9F
:10DEB00004E06FF0030401E06FF00204204670BD3F
:10DEC0002DE9F041134C0F460546E6682068001D19
:10DED00000F0C4FC681C07D137B12168BDE8F041EF
:10DEE0000D48091D00F00CBD20683544B542456061
:10DEF000216805D2A06B091DBDE8F04100F0E8BC27
:10DF0000606B091D00F0E4FCA06A854200D2A562A6
:10DF1000BDE8F0811C0000240C0F00242DE9F04125
:10DF2000054600F0F9FC2D4C2D4FA068401CA06068
:10DF3000206810B1606930B32BE02560A06801282B
:10DF400027D1002606EB860007EB800000F0B2FC2C
:10DF5000761C382EF6D3234800F0ACFC2148143050
:10DF600000F0A8FC1F48283000F0A4FC1D483C30FD
:10DF700000F0A0FC1B48503000F09CFC1948606386
:10DF80001430A06305E0E86A2168C96A814200D8BC
:10DF90002560606A401C60626864E86A21698842A2
:10DFA00000D9206100EB8000291D07EB800000F004
:10DFB000A7FC00F0D1FC606900280CD02068E96A59
:10DFC000C06A884207D208494FF080500860BFF30A
:10DFD0004F8FBFF36F8FBDE8F08100001C0000245D
:10DFE0005C0A0024BC0E002404ED00E038B500F00B
:10DFF00093FC104C2068C8B90F4800F05BFC0E4839
:10E00000143000F057FC0C490020E160143121610C
:10E01000A1F582730090A1F1B40210210A2000F052
:10E02000D8FF206010B105A100F018FDBDE8384010
:10E0300000F092BC5800002410100024546D72515E
:10E040000000000030B4026C0B46002A0BD0D0E96F
:10E0500002411144C160A14201D30168C160184668
:10E0600030BCF2F7D9BA30BC70472DE9F041856B6E
:10E070001746026C0446002682B1C7B1E068F2F789
:10E08000CBFAE168206C2268091AE160914202D261
:10E09000A168081AE060022F16D017E02068A8B91E
:10E0A000A06801F05BFD06460020A0600EE06068FD
:10E0B000F2F7B2FAD4E90101226C104460608842A0
:10E0C00004D32068606001E005B16D1E6D1CA5637E
:10E0D0003046BDE8F08110B5044690F8590058B1BB
:10E0E00001280CD002280FD0502080F31188BFF3F4
:10E0F0004F8FBFF36F8FFEE7206B00F041FC20468F
:10E10000BDE8104000F03CBC10BD000011484FF4C9
:10E11000004110B5420706D00E49C01D20F007008F
:10E12000411AC1F500410C4C002301440839A4F107
:10E13000180221F00701C4E900030C1A11604B60BA
:10E140000B60C0E9001494604FF0004154605161CD
:10E1500010BD0000F016002488000024144E4FF07B
:10E160008058144CDFF85090A6F29C4712E000BF94
:10E1700000F0D2FBF068C568281D00F06FFBA068B6
:10E18000401EA0606068401E606000F0E5FB28460D
:10E19000FFF7A1FF60680028EAD138680128F9D9A3
:10E1A000C9F80080BFF34F8FBFF36F8FF2E7000015
:10E1B000F80E00241C00002404ED00E0002807D025
:10E1C0000021816001600B460A46C16000F07EBFFD
:10E1D0007047000070B51D46049C51B1C4F8002082
:10E1E000C4E90F010121204600F026FF84F84C50BD
:10E1F00070BD2460F4E72DE9F05F88469A469100EF
:10E200001546DDE90B940A9EA5228346206BF2F7A2
:10E210007AFA206B6FF0030101EB8501084420F0CE
:10E220000707780707D0502080F31188BFF34F8F7E
:10E23000BFF36F8FFEE7B8F1000F4FF000050ED06F
:10E240000020221818F8001082F8341018F8001076
:10E2500011B1401C1028F4D384F8435001E084F835
:10E260003450382E00D33726E662201DC4E91365EA
:10E2700000F02BFB04F1180000F027FB6565C6F1E8
:10E280003800A06184F858505246246159463846F7
:10E29000646200F067FAB9F1000F206001D0C9F89C
:10E2A0000040BDE8F09F000030B5114900E0114684
:10E2B0000A688242FBD34B685C18844203D14468ED
:10E2C000084623444B6043681D18954209D1084C09
:10E2D000183C2468A24209D052681A4442600A6875
:10E2E00012680260814200D0086030BD0460F9E726
:10E2F0008800002470B50D4D914241604FF000043C
:10E30000006106D88169D21A8A4206D2011D2869A5
:10E3100007E09A4203D2994201D3012403E0011D90
:10E32000E86800F0D5FA204670BD000058000024CF
:10E3300010B5044600F0F0FAA06B28B15FF00004BD
:10E3400000F00AFB204610BD0124F9E730B53C4D32
:10E3500089B06BE00498002806DA059ADDE9060129
:10E3600090470498002861DB069C606910B1201D6D
:10E3700000F074FA03A800F0D5F8024604980A28C1
:10E3800054D2DFE800F00505052D304705052D3096
:10E3900094F8280040F0010084F82800A06905994D
:10E3A0000B4601442046FFF7A5FF50B3216A2046E3
:10E3B000884794F82800400738D500200090059839
:10E3C0000023A16942181946204601F00DFDC0B98D
:10E3D000502080F31188BFF34F8FBFF36F8FFEE79C
:10E3E00094F828001EE094F8280040F0010084F81A
:10E3F00028000598A06128B1811813462046FFF730
:10E4000079FF13E0502080F31188BFF34F8FBFF3E3
:10E410006F8FFEE794F82800810703D4204600F0B0
:10E42000AFFA03E020F0010084F8280028680022F9
:10E4300004A900F079FF00288CD109B030BD00009C
:10E44000580000242DE9FC410F46054600F0BEFCB3
:10E4500001A800F067F80446019818B101F032FCF9
:10E46000BDE8FC81254EAFB130690068D0B300270C
:10E470003068291B3A4600F005FB01F023FC002818
:10E48000EED11F494FF080500860BFF34F8FBFF3AC
:10E490006F8FE5E7A542EBD801F014FCF068274642
:10E4A000C068C468201D00F0D9F994F8280041071D
:10E4B00019D5A0692B463A4641192046FFF71AFFA5
:10E4C000A8B100202A46034601460090204601F0EC
:10E4D0008BFC60B9502080F31188BFF34F8FBFF3DE
:10E4E0006F8FFEE707E020F0010084F82800216A22
:10E4F00020468847B4E70127BAE700005800002407
:10E5000004ED00E00648416B096829B1416BC96818
:10E51000C9684968816270474FF0FF31FAE700002F
:10E520001C00002470B5054601F060FA064E044652
:10E53000B068844203D200F009F8012000E0002016
:10E5400028602046B46070BD58000024F8B5194D0D
:10E5500020E0C068C4680668201D00F07FF9216AC9
:10E560002046884794F82800400713D5A069304416
:10E57000B04206D92461211D6060E86800F0A8F966
:10E5800008E000203246034601460090204601F094
:10E590002BFC38B1E86801680029DAD12969C5E99E
:10E5A0000310F8BD502080F31188BFF34F8FBFF3E5
:10E5B0006F8FFEE75800002408484068401C4FF069
:10E5C000500080F3118804D0BFF34F8FBFF36F8FDB
:10E5D000FEE7BFF34F8FBFF36F8FFEE7900000247D
:10E5E000074CE068016841B1C0680021D0F8000024
:10E5F000FFF728FFFFF7AAFEF3E701210020F7E766
:10E60000580000242DE9F041044600F085F994F902
:10E61000455004F1240609E0606A48B1304601F033
:10E6200019FB08B100F00CFB6D1E6DB2002DF3DC80
:10E630004FF0FF3684F8456000F08EF900F06CF979
:10E6400094F9445004F1100709E0206948B13846B4
:10E6500001F000FB08B100F0F3FA6D1E6DB2002D61
:10E66000F3DC84F84460BDE8F04100F075B90000C7
:10E670002DE9F0410027044600F0A8FB324E306837
:10E6800008B9FFF743FD706904424ED1C4B30834A2
:10E6900060070ED004F00700C0F1080004446007D2
:10E6A00007D0502080F31188BFF34F8FBFF36F8FD7
:10E6B000FEE72CB37068844237D8234818300146EF
:10E6C0000D6801E028460D466968A14202D229681A
:10E6D0000029F7D131688D4227D007682968016089
:10E6E00008376868011B10290FD92819420708D07C
:10E6F000502080F31188BFF34F8FBFF36F8FFEE779
:10E7000013E041606C60FFF7CFFD69687068401AE4
:10E710007060B268904200D2B0600020726911430C
:10E72000C5E90001F068401CF06001F0CBFA780701
:10E7300007D0502080F31188BFF34F8FBFF36F8F46
:10E74000FEE73846BDE8F0817000002404490868FF
:10E7500018B10868026D521C026508687047000015
:10E760001C00002470B5041F094E231F4FF0807554
:10E7700021F0010125601C1F1960A0F120010B1F71
:10E78000266044380A606FF002051D6070BD00000D
:10E79000B9E5000810B500EE100A2DED028BB1EEC0
:10E7A000C08A18EE100A20F00040C0F1FF40C00FF0
:10E7B0000AD010EE100A20F00040C0F1FF40C00F58
:10E7C00004BF0120F1F7F8FF18EE100ABDEC028B30
:10E7D00010BD00000848017800290CD10849012229
:10E7E0009FED060A02700023438081ED000A81ED4F
:10E7F000010A81ED020A704728040024000000008D
:10E80000C8BD002410B50446F7F78AF908494860E6
:10E8100001F110002178017161784171A1780170D6
:10E82000E17849004180217981716179C17110BD20
:10E83000BC00002401EE100A70EEC00A0120B8EE00
:10E84000C11A8840401E21EE201A00EE900AF8EE10
:10E85000E01AC1EE210A30EE800A7047D0E9013299
:10E8600001699A60D0E901235A604A68824201D165
:10E8700082684A60002202610868401E08600868D9
:10E880007047000010B5044C8023046004F15C0064
:10E890000860136010BD00003810002410B5044C4F
:10E8A0004FF48073046004F15C000860136010BDD5
:10E8B000941200244FF0FF3300F108010022C0E958
:10E8C00001130260C160016170470021016170475E
:10E8D00030B50B685A1C02D000F1080202E0026950
:10E8E00004E02246546825689D42FAD953684B607B
:10E8F00099608A60516008610168491C016030BDFF
:10E9000042684A6093688B609368596091600861BF
:10E910000168491C01607047502080F31188BFF3E3
:10E920004F8FBFF36F8F0A494868401C4860012829
:10E930000CD10848006810F0FF0F07D0502080F37A
:10E940001188BFF34F8FBFF36F8FFEE77047000052
:10E950009000002404ED00E00849486828B1401EFA
:10E96000486001D180F311887047502080F31188EE
:10E97000BFF34F8FBFF36F8FFEE7000090000024BE
:10E9800070B500282AD0164DA0F1080461686869A6
:10E99000014207D1502080F31188BFF34F8FBFF39E
:10E9A0006F8FFEE722683AB1502080F31188BFF3E1
:10E9B0004F8FBFF36F8FFEE78143616000F006FA6F
:10E9C00060686968084468602046FFF76DFC286944
:10E9D000401C2861BDE8704001F074B970BD0000B2
:10E9E000700000244FF0E020002101614FF47A72A2
:10E9F0008161072303490968B1FBF2F1491E4161B6
:10EA0000036170471400002410B5F1F72DFD114982
:10EA100010280ED300F1E0200A7890F8F00390421D
:10EA200007D2502080F31188BFF34F8FBFF36F8F51
:10EA3000FEE709488968006800F4E060884207D969
:10EA4000502080F31188BFF34F8FBFF36F8FFEE725
:10EA500010BD0000900000240CED00E0084B5FF0BA
:10EA6000000210B553F832401CB1521C082AF9D3E9
:10EA700010BD03EBC20443F83210606010BD00000B
:10EA80001C0A002470B515460E460446FFF744FFE5
:10EA900094F944100020491C01D184F8440094F9F1
:10EAA0004510491C01D184F84500FFF755FFA06BC4
:10EAB00028B904F124002A46314600F0DFF8204648
:10EAC000BDE87040FFF79EBD020010B514D00F489E
:10EAD000006B38B1502080F31188BFF34F8FBFF324
:10EAE0006F8FFEE700F072F900211046FFF7E8F99A
:10EAF00001F0E8F8002807D105494FF08050086080
:10EB0000BFF34F8FBFF36F8F10BD00001C000024B8
:10EB100004ED00E070B504000D460BD095B11E4A1F
:10EB2000106BB8B1502080F31188BFF34F8FBFF343
:10EB30006F8FFEE7502080F31188BFF34F8FBFF334
:10EB40006F8FFEE7502080F31188BFF34F8FBFF324
:10EB50006F8FFEE700F03AF92368D26859199342A3
:10EB600004D98B420AD9914202D807E08B42FAD9E4
:10EB7000881A21600021FFF7A3F900E0216001F06D
:10EB8000A1F8002807D105494FF080500860BFF375
:10EB90004F8FBFF36F8F70BD1C00002404ED00E0A9
:10EBA00070B50546FFF7B8FE1E4C05B92568281D4F
:10EBB000FFF754FEA86A18B105F11800FFF74EFEE2
:10EBC000606A401C60622068854207D11648291D92
:10EBD000FFF796FE6068401C606007E0A068401E7A
:10EBE000A0602846FFF777FAFFF78CFCFFF7B4FE2A
:10EBF0006069002814D02068854211D1206B38B19B
:10EC0000502080F31188BFF34F8FBFF36F8FFEE763
:10EC100006494FF080500860BFF34F8FBFF36F8FEE
:10EC200070BD00001C000024F80E002404ED00E07C
:10EC300002490A6A0260C968416070471C000024EA
:10EC400001490120C86170471C00002410B50C4622
:10EC500050B1094909681831FFF73AFE2046BDE86E
:10EC600010400121FFF72CB9502080F31188BFF329
:10EC70004F8FBFF36F8FFEE71C00002470B5144662
:10EC80000D4668B10A4909681831FFF739FE0CB121
:10EC90004FF0FF3521462846BDE87040FFF710B918
:10ECA000502080F31188BFF34F8FBFF36F8FFEE7C3
:10ECB0001C00002470B5002804463ED0226DA2B18D
:10ECC000E06C884200D30146E06A884235D0012AD0
:10ECD00033D11A4D2A6894420FD1502080F3118805
:10ECE000BFF34F8FBFF36F8FFEE7502080F3118883
:10ECF000BFF34F8FBFF36F8FFEE7A269E162002A77
:10ED000002DBC1F13801A1610D4E00EB80006169A9
:10ED100006EB8000814210D1201DFFF79FFDE06AC5
:10ED20002969884200D9286100EB8000211D06EB8B
:10ED30008000BDE87040FFF7E3BD70BD1C000024FB
:10ED40005C0A002430B587B0002405AA04A9039406
:10ED500003A80494FFF796FDDDE903010094002366
:10ED6000CDE90110174815A1059A00F00EFD164DCA
:10ED70000028E8621FD001F007F8012809D0401CE4
:10ED800019D1502080F31188BFF34F8FBFF36F8FDD
:10ED9000FEE7502080F31188BFF34F8FBFF36F8FD2
:10EDA00001214FF0FF30A8626961EC6007B0BDE857
:10EDB000304000F045B807B030BD000049444C4534
:10EDC000000000005DE100081C0000240248016B07
:10EDD000491C0163704700001C000024164810B550
:10EDE000016B11B10121C16110BD0021C161134A44
:10EDF000016901E0B9B1491E01EB810352F82330EA
:10EE0000002BF7D001EB810302EB830202F108042F
:10EE100053685B685360A34201D15B685360DA6852
:10EE20000260016110BD502080F31188BFF34F8F45
:10EE3000BFF36F8FFEE700001C0000245C0A002473
:10EE400037481CB5374902688A4207D1502080F301
:10EE50001188BFF34F8FBFF36F8FFEE73149006812
:10EE6000491E884207D1502080F31188BFF34F8F8D
:10EE7000BFF36F8FFEE72C49FF200A7801920870DC
:10EE800008788DF800009DF800209DF8000002F041
:10EE9000F002824207D0502080F31188BFF34F8FD9
:10EEA000BFF36F8FFEE79DF8002007201F4C02F094
:10EEB00050022270A06005E09DF8002052008DF8FD
:10EEC0000020401E9DF800201206F5D40328A06003
:10EED00007D0502080F31188BFF34F8FBFF36F8F9F
:10EEE000FEE74FF44070A060019808700C48203095
:10EEF000016841F470010160016841F070410160F6
:10EF0000FFF770FD00206060F1F776FA08480168AD
:10EF100041F040410160F1F75BFA00201CBD0000A8
:10EF200000ED00E071C20F4100E400E09000002419
:10EF300034EF00E0502010B580F31188BFF34F8FFD
:10EF4000BFF36F8F00F060FD18B104494FF080509F
:10EF50000860002080F3118810BD000004ED00E07F
:10EF600000210246012010B500F012F80446FFF718
:10EF700025F9204610BD38B500220B4611460090F9
:10EF8000012000F026F80446FFF718F9204638BDA6
:10EF9000F8B5050017460E4613D005FB06F05030B5
:10EFA000FFF766FB04000AD0002084F8460004F155
:10EFB00050023B46314628460094FFF70BF92046A5
:10EFC000F8BD502080F31188BFF34F8FBFF36F8FD0
:10EFD000FEE7F8B5069D18B153B1CAB181B120E082
:10EFE000502080F31188BFF34F8FBFF36F8FFEE780
:10EFF000502080F31188BFF34F8FBFF36F8FFEE770
:10F00000502080F31188BFF34F8FBFF36F8FFEE75F
:10F0100039B1502080F31188BFF34F8FBFF36F8F4A
:10F02000FEE750241C46012683F8466000932B46D9
:10F03000FFF7D0F82046F8BD2DE9F04704008A46D6
:10F0400029D0FFF769FC21680025D4E90F23D4F803
:10F0500040C004F1100810460E46401E4FF0FF3924
:10F0600002FB031200FB0C10BAF1000FA5636660EF
:10F0700084F8449084F84590C4E9022013D04046B7
:10F08000FFF718FC04F12400FFF714FCFFF764FC01
:10F090000120BDE8F087502080F31188BFF34F8F27
:10F0A000BFF36F8FFEE720690028EFD0404600F0E5
:10F0B000D1FD0028EAD004494FF080500860BFF32A
:10F0C0004F8FBFF36F8FE1E704ED00E02DE9FF47BD
:10F0D00004001D4682B08A464FF0000803D0BAF102
:10F0E000000F08D011E0502080F31188BFF34F8F3C
:10F0F000BFF36F8FFEE7206C38B1502080F311888A
:10F10000BFF34F8FBFF36F8FFEE7022D0AD1E06B85
:10F11000012807D0502080F31188BFF34F8FBFF331
:10F120006F8FFEE700F054FC3F4F4FF080564FF0DA
:10F13000000948B9049838B1502080F31188BFF312
:10F140004F8FBFF36F8FFEE7FFF7E6FBA06BE16B1E
:10F15000884207D3022D05D00498D0B1B8F1000F32
:10F160001AD01EE02A4651462046FEF77EFF616A0D
:10F1700019B104F1240000F06DFD20B13E60BFF331
:10F180004F8FBFF36F8FFFF7E7FB012006B0BDE89D
:10F19000F087FFF7E1FB22E06846FFF749FD4FF0FB
:10F1A0000108FFF7D9FBFFF711FEFFF7B5FB94F954
:10F1B0004400401C01D184F8449094F94500401C5F
:10F1C00001D184F84590FFF7C7FB04A9684600F019
:10F1D00073FA30B12046FFF715FA00F073FD0020F6
:10F1E000D4E7FFF799FBA06BE16B884213D1FFF7DF
:10F1F000B3FB049904F11000FFF728FD2046FFF748
:10F2000001FA00F05FFD00289ED13E60BFF34F8FF2
:10F21000BFF36F8F98E7FFF79FFB2046FFF7F2F9E8
:10F2200000F050FD90E7000004ED00E02DE9F0470C
:10F2300004001F469046894603D0B9F1000F08D05C
:10F2400011E0502080F31188BFF34F8FBFF36F8F11
:10F25000FEE7206C38B1502080F31188BFF34F8F48
:10F26000BFF36F8FFEE7022F0AD1E06B012807D0B2
:10F27000502080F31188BFF34F8FBFF36F8FFEE7ED
:10F28000FFF7C2FB5020EFF3118680F31188BFF324
:10F290004F8FBFF36F8FA06BE16B884206D3022FB5
:10F2A00004D0002086F31188BDE8F08794F945501A
:10F2B000A06B3A4649462046FEF7D7FE681C04D0AC
:10F2C0006D1C84F845500120ECE7606A0028FAD0F4
:10F2D00004F1240000F0BEFC0028F4D0B8F1000FC7
:10F2E000F1D00121C8F80010EDE710B5040009D0F5
:10F2F00000F068FBA168884214D1E068401EE0601D
:10F3000008D00DE0502080F31188BFF34F8FBFF37A
:10F310006F8FFEE7002320461A461946FFF7D6FEF8
:10F32000012010BD002010BD2DE9F74704008A46DA
:10F3300083B04FF0000603D0BAF1000F08D011E0FF
:10F34000502080F31188BFF34F8FBFF36F8FFEE71C
:10F35000206C38B1502080F31188BFF34F8FBFF37A
:10F360006F8FFEE700F034FBDFF8F4804FF080573A
:10F370004FF0000948B9059838B1502080F3118842
:10F38000BFF34F8FBFF36F8FFEE7FFF7C5FAA56B93
:10F39000C5B151462046FEF755FE6D1EA563206996
:10F3A00050B104F1100000F055FC28B1C8F800700D
:10F3B000BFF34F8FBFF36F8FFFF7CEFA012006B078
:10F3C000BDE8F087059808B11EB106E0FFF7C4FA62
:10F3D00027E06846FFF72CFC0126FFF7BDFAFFF790
:10F3E000F5FCFFF799FA94F94400401C01D184F828
:10F3F000449094F94500401C01D184F84590FFF7F2
:10F40000ABFA05A9684600F057F9002820460AD053
:10F41000FFF7F8F800F056FC2046FEF789FF0028B9
:10F42000B3D00020CBE7FEF783FF90B1059904F13C
:10F430002400FFF70BFC2046FFF7E4F800F042FC45
:10F440000028A2D1C8F80070BFF34F8FBFF36F8FB1
:10F450009BE72046FFF7D6F800F034FC95E7000064
:10F4600004ED00E02DE9F04704009046894603D002
:10F47000B9F1000F08D011E0502080F31188BFF3DC
:10F480004F8FBFF36F8FFEE7206C38B1502080F3B1
:10F490001188BFF34F8FBFF36F8FFEE7FFF7B4FA0A
:10F4A0005020EFF3118680F31188BFF34F8FBFF325
:10F4B0006F8FA76BFFB194F9445049462046FEF781
:10F4C000C1FD681CA7F10107A76304D06D1C84F877
:10F4D0004450012010E020690028FAD004F1100007
:10F4E00000F0B8FB0028F4D0B8F1000FF1D00121F2
:10F4F000C8F80010EDE7002086F31188BDE8F0871A
:10F500002DE9F3434FF000060400354683B009D0DF
:10F51000206C78B1502080F31188BFF34F8FBFF378
:10F520006F8FFEE7502080F31188BFF34F8FBFF33A
:10F530006F8FFEE700F04CFADFF83C814FF0805708
:10F540004FF0000948B9049838B1502080F3118871
:10F55000BFF34F8FBFF36F8FFEE7FFF7DDF9A06BAF
:10F56000C8B12168401EA06311B9FFF7EFF8A06091
:10F57000206950B104F1100000F06CFB28B1C8F80C
:10F580000070BFF34F8FBFF36F8FFFF7E5F90120D6
:10F5900005B0BDE8F083049808B166B10FE03DB155
:10F5A000502080F31188BFF34F8FBFF36F8FFEE7BA
:10F5B000FFF7D2F95EE06846FFF73AFB0126FFF756
:10F5C000CBF9FFF703FCFFF7A7F994F94400401CBF
:10F5D00001D184F8449094F94500401C01D184F88D
:10F5E0004590FFF7B9F904A9684600F065F80028CE
:10F5F000204612D0FFF706F800F064FB2046FEF725
:10F6000097FE0028A9D075B3FFF786F9606A58B352
:10F61000206B0068C0F1380128E0FEF789FEE0B1F8
:10F62000206838B9FFF778F9A06800F0D5FA0546E8
:10F63000FFF792F9049904F12400FFF707FB204635
:10F64000FEF7E0FF00F03EFB002886D1C8F800700E
:10F65000BFF34F8FBFF36F8F7FE72046FEF7D2FFD8
:10F6600000F030FB79E705E0FFE70021A068FFF735
:10F6700021FB9DE700208BE704ED00E070B504005E
:10F680000D4607D000F09EF9A16888420AD1E168D2
:10F6900001200EE0502080F31188BFF34F8FBFF39D
:10F6A0006F8FFEE729462046FFF72AFF002802D089
:10F6B000E168491CE16070BD2DE9F04105000C4690
:10F6C00012D0CCB1FFF728F9184E2068F268471C19
:10F6D0006B68A2EB030117D02F68366AB74215D0CA
:10F6E000934213D801251CE0502080F31188BFF30A
:10F6F0004F8FBFF36F8FFEE7502080F31188BFF369
:10F700004F8FBFF36F8FFEE700250AE0884205D9CF
:10F71000401A20602846FFF78BFAF5E700202060AA
:10F720000125FFF719F92846BDE8F0811C000024E7
:10F730002DE9FF5F994616468A4683469000DDE92B
:10F740000E87FEF795FF05001CD05C20FEF790FFAA
:10F75000040014D00020256384F859004B46CDE9FD
:10F760000087CDE90240324651465846FEF743FD38
:10F770002046FEF7D3FB012004B0BDE8F09F2846E9
:10F78000FFF7FEF84FF0FF30F6E7F0B585B0DDE9A2
:10F790000B740A9DA7B1DCB15C262763022684F8AE
:10F7A0005960002703970DF1100C0095CDE901C4B5
:10F7B000FEF721FD2046FEF7B1FB049805B0F0BD31
:10F7C000502080F31188BFF34F8FBFF36F8FFEE798
:10F7D000502080F31188BFF34F8FBFF36F8FFEE788
:10F7E0002DE9F0411F4690460D464FF0010690B1BD
:10F7F0000446FFF791F80FB1606D3860022294F86B
:10F80000580084F85820B8F1050F19D2DFE808F045
:10F81000230B0E141200502080F31188BFF34F8F7A
:10F82000BFF36F8FFEE7616D294301E0616D491CF5
:10F83000616510E0022801D065650CE0002634E027
:10F84000616D491C07D0502080F31188BFF34F8FA2
:10F85000BFF36F8FFEE7012827D1201DFEF7FEFFC3
:10F86000144DE06A2969884200D9286100EB8000C4
:10F87000114901EB8000211DFFF742F8A06A38B161
:10F88000502080F31188BFF34F8FBFF36F8FFEE7D7
:10F890002868E16AC06A814207D908494FF0805060
:10F8A0000860BFF34F8FBFF36F8FFFF755F83046F7
:10F8B000BDE8F0811C0000245C0A002404ED00E097
:10F8C0002DE9F04704001F4692460D46DDF82090D2
:10F8D0004FF001081AD0FFF797F85020EFF3118688
:10F8E00080F31188BFF34F8FBFF36F8F0FB1606D3F
:10F8F0003860022294F8580084F85820BAF1050FB5
:10F900001AD2DFE80AF0240B0E141200502080F304
:10F910001188BFF34F8FBFF36F8FFEE7616D2943EF
:10F9200001E0616D491C616511E0022801D0656547
:10F930000DE04FF000083AE0616D491C07D05020FF
:10F9400080F31188BFF34F8FBFF36F8FFEE701285D
:10F950002DD1A06A38B1502080F31188BFF34F8FAA
:10F96000BFF36F8FFEE7144D286B18B1134804F1F5
:10F9700018010DE0201DFEF771FFE06A2969884239
:10F9800000D9286100EB80000D4901EB8000211DAA
:10F99000FEF7B6FFE06A2968C96A884207D9B9F15B
:10F9A000000F4FF0010001D0C9F80000E86186F3B4
:10F9B00011884046BDE8F0871C000024E40E0024B6
:10F9C0005C0A002401480068704700001C00002405
:10F9D0000548416919B1006B18B10020704701203A
:10F9E00070470220704700001C0000240148C068D6
:10F9F000704700001C00002410B5FFF705F801480F
:10FA0000C06810BD1C0000242DE9F0412E4C206B75
:10FA1000002728B1A069401CA0613846BDE8F081EC
:10FA2000E668761CE66013D1606B006838B1502040
:10FA300080F31188BFF34F8FBFF36F8FFEE7606BCA
:10FA4000A16B6163A063206A401C2062FEF75AFD2F
:10FA5000DFF87880A06A864209D3606B0068A0B1A5
:10FA6000606BC068C5686868864211D2A062206871
:10FA7000C06A00EB800158F82100012800D9012755
:10FA8000E0690028C9D00127C7E74FF0FF30EDE754
:10FA9000281DFEF7E3FEA86A18B105F11800FEF76D
:10FAA000DDFEE86A2169884200D9206100EB80010F
:10FAB00008EB8100291DFEF723FF2068E96AC06A70
:10FAC0008142CAD30127C8E71C0000245C0A002435
:10FAD0002DE9F0411E46154688460746FEF71CFFF5
:10FAE0001C4C206890F85800022814D02068416D02
:10FAF000B94341652168012081F858005EB10121B8
:10FB00003046FEF7DDF914494FF080500860BFF32E
:10FB10004F8FBFF36F8FFEF71FFFFEF7FDFE15B18E
:10FB20002068406D2860206890F85800022801D0B5
:10FB3000002505E02068416D21EA080141650125A5
:10FB40002168002081F85800FEF706FF2846BDE82E
:10FB5000F08100001C00002404ED00E070B50446B4
:10FB60004FF0000190B31A4D2868844207D050200E
:10FB700080F31188BFF34F8FBFF36F8FFEE7206DC7
:10FB800038B1E36C401EE26A20659A421ED040B153
:10FB90001CE0502080F31188BFF34F8FBFF36F8FAD
:10FBA000FEE7201DFEF75AFEE06CC0F13801A161AE
:10FBB000E0622969884200D9286100EB800005498C
:10FBC00001EB8000211DFEF79BFE0121084670BD60
:10FBD0001C0000245C0A002470B5002804464FF085
:10FBE00000002BD0194DE16A2A68D26A914226D2D0
:10FBF000A069002804DB2868C06AC0F13800A06151
:10FC0000134E01EB8101606906EB8101884211D13D
:10FC1000201DFEF723FE2868C06AE0622969884239
:10FC200000D9286100EB8000211D06EB8000FEF763
:10FC300067FE02E02868C06AE062012070BD2968A2
:10FC4000E26CC96A8A42F8D370BD00001C0000242F
:10FC50005C0A002470B5C068C46854B104F118008F
:10FC60000646FEF7FBFD144D286B50B11348314694
:10FC700015E0502080F31188BFF34F8FBFF36F8FD3
:10FC8000FEE7201DFEF7EAFDE06A2969884200D9F7
:10FC9000286100EB80000A4901EB8000211DFEF77E
:10FCA0002FFEE06A2968C96A884203D90121E96107
:10FCB000084670BD002070BD1C000024E40E002426
:10FCC0005C0A00242DE9F0472C4D286B00242746C0
:10FCD00038B1FEF721FE286B401E2863286B40B127
:10FCE00047E0502080F31188BFF34F8FBFF36F8F31
:10FCF000FEE7234E0120A968D9B3A6F59169804695
:10FD00003068E0B1F068C46804F11800FEF7A6FDA1
:10FD1000201DFEF7A3FDE06A2969884200D9286109
:10FD200000EB800109EB8100211DFEF7E9FDE06A8F
:10FD30002968C96A8842E3D3C5F81C80E0E70CB1A2
:10FD4000FEF7E0FBAC694CB14FEA0806FFF75CFE3A
:10FD500000B1EE61641EF9D10020A861E86940B1EC
:10FD6000084901274FF080500860BFF34F8FBFF361
:10FD70006F8FFEF7F1FD3846BDE8F0871C000024C8
:10FD8000E40E002404ED00E010B586B0FEF72EF975
:10FD9000114C2068B8B10020039005AA049004A972
:10FDA00003A8FEF77BFDDDE90321022000238DE897
:10FDB00007000C4809A1059AFFF7E7FC606010B145
:10FDC00006B0012010BD502080F31188BFF34F8F83
:10FDD000BFF36F8FFEE7000058000024546D7220BF
:10FDE00053766300E1E500082DE9FF411E46134606
:10FDF00002004FF000000A9D16D0144C2768002F17
:10FE00000FD006290292CDE9001317DAFFF7E0FDC3
:10FE100002284FF000030FD0002220686946FFF748
:10FE200055F904B0BDE8F081502080F31188BFF38C
:10FE30004F8FBFF36F8FFEE72A46EEE7002332466F
:10FE400069463846FFF7F2F9EBE700005800002456
:10FE500000EE100A00EE901AB4EE600AF1EE10FA0D
:10FE600078BF704700F00DB810B5FFF7F1FFEFF362
:10FE7000008020F0104038BF40F0004080F3008840
:10FE800010BDBDE8104010B500F047F800000009B3
:10FE900000F007B84FF0404010F1004FEFF3008042
:10FEA0007047401058BFC0F14040491058BFC1F1E1
:10FEB00040418142EFF3008070474FF07E5209E0ED
:10FEC00011F0004204D54042C1F1000138BF491E83
:10FED00042F07E520B0002F1706212BF20235FEAF3
:10FEE00000017047B1FA81FCA3EB0C0301FA0CF19D
:10FEF00020FA03FC02EBC352C3F1200341EA0C01D8
:10FF000010FA03FC5CEA416C42EB112018BF5FF071
:10FF1000806C28BF20F0010070470EF1020E2EF019
:10FF2000030E5EF8044B244204D44FEA4102B2F1BE
:10FF30007F4F11D84FEA4003B3F17F4F0CD80ED159
:10FF40004FEAD07CB2F17F4F0CEB4C0C0CF1020C61
:10FF500008BF4CEBD17C04E04FF0080C01E04FEA05
:10FF6000D17C0CEB4C0324FA03F404F00704B4F145
:10FF7000040C06D20EEB840CBDE810404CF0010CD2
:10FF80006047DFE80CF0070802024FF00040A0F5E0
:10FF9000800010BD0846420018BFD2F1807288BFB1
:10FFA00000F0004010BD4FF04070E1EE100A7047C5
:10FFB000A80301080000000000000000000000008D
:10FFC0000000000000020000180000000000000017
:10FFD00000000000000610160006101600010203C3
:10FFE00004050607080C101418203040000000001B
:10FFF0000000000000000000000000000000000001
:020000040801F1
:1000000001000000020000000300000004000000E6
:1000100000000000050000000000000000000000DB
:1000200000000000060000000000000000000000CA
:1000300000000000070000000100020004000600AC
:1000400008000A000C0010002000400080000001A1
:100050000101010307010000080402040801010175
:10006000000000000102030401020304060708095E
:100070000001020304050607080C10141820304084
:100080000080000000000258010000000008025833
:10009000002000000008025800400000000802583C
:1000A0000080000000080258080000000008025804
:1000B0000004000000100258001000000010025858
:1000C0002C0800240C000000780800240400000024
:1000D00000000000010000000002000005210008EF
:1000E000010000000200000000020000872000085C
:1000F0000200000004000000000200001B210008B4
:100100000300000008000000000200003121000888
:100110000400000010000000000200005D20000844
:10012000050000002000000000020000C3200008BD
:10013000060000000000008000080000E920000820
:10014000070000000080000001080000F320000804
:1001500008000000800000000002000047210008A5
:100160000900000000010000010C000083200008CD
:100170000A00000030400000010100009D2000083E
:10018000000000000000803F0AD7233C0000000070
:100190000000803F0000803F0000000000000000E1
:1001A000C40301080000000000000000000000007F
:1001B000000000000004000030000000000000000B
:1001C00000000000D0030108000000000000000053
:1001D0000000000000000000000400001800000003
:1001E0000000000000000000D4030108000000002F
:1001F00000000000000000000000000000040000FB
:10020000180000000000000000000000E0030108EA
:1002100000000000000000000000000000000000DE
:1002200000040000180000000000000000000000B2
:10023000E8030108000000000000000000000000CA
:100240000000000000200000180000000000000076
:1002500000000000F803010800000000000000009A
:100260000000000000000000000400001800000072
:10027000000000000000000004040108000000006D
:10028000000000000000000000000000000400006A
:100290001800000000000000000000001004010829
:1002A000000000000000000000000000000000004E
:1002B0000004000018000000000000000000000022
:1002C000140401080000000000000000000000000D
:1002D00000000000000800001800000000000000FE
:1002E00000000000000000004FBB610567ACDD3F6F
:1002F000182D4454FB21E93F9BF681D20B73EF3F4D
:10030000182D4454FB21F93FE2652F227F2B7A3CC4
:10031000075C143326A6813CBDCBF07A8807703C7D
:10032000075C143326A6913CC4EB98999999C9BFF0
:10033000711623FEC671BCBF6D9A74AFF2B0B3BF25
:100340009AFDDE522DDEADBF2F6C6A2C44B4A2BFE5
:100350000D5555555555D53FFF8300922449C23F51
:100360006E204CC5CD45B73F513DD0A0660DB13F85
:10037000EB0D76244B7BA93F11DA22E33AAD903F97
:100380000000000000000000000000006E83F9A2E1
:100390002915444ED15727FCC0DD34F5999562DB11
:1003A0004190433CAB6351FE64656661756C745467
:1003B00061736B00445231365F5043004452313612
:1003C0005F5243005461736B5F496E6974000000B3
:1003D00072630000617474695F6573746900000082
:1003E000626C696E6B0000006374726C5F636861BD
:1003F00073736973000000006374726C5F67696DEA
:1004000062616C006374726C5F73686F6F7400007C
:10041000636D640073757065726361700000000045
:1004200040040108000000244C04000008030008F8
:10043000C80501084C0400243CEA000064030008DD
:1004400081320182103C90D0030401771AAA010185
:100450003C2D022B073DD0320625CDCC4C3F3A80B7
:100460000452052B803FD9292021339B43133F01A0
:100470002B0102101908111C0202010B290A7A0330
:100480000A3A041E1A020A3A0514290A5A060A21CF
:100490001A071E2920296447C03F9A99993E197866
:1004A0002D3E666666784ABF04397C3D40CDCCCC93
:1004B00020190C1908390459202B20404419204ECA
:1004C0003D0AD7233D2839B83DBFDB0FC91C9960D1
:1004D00019287A4C2059603D3F6666E62029440C75
:1004E000119A9919402904C1A940CBF041043A124C
:1004F000DE2112608A502C79E08950798019341AF3
:10050000806849FC612A2014398089D0B97CD9409F
:100510001AA0401A202C0910404924437A443C5E1A
:10052000DC3E1019E419401401020132015A02089C
:100530005A03083A04080D1D6F12833A78591009BE
:1005400010204978412B4842042956211A40142989
:1005500004111904237A465A05700D200602010180
:1005600070091F905F010203CDCC4C142AC028688B
:10057000083F0102040101022F83BB44136B241BBB
:1005800008A3041AEB04298213A9231B08D9041A0F
:100590004310692F81F20345BC0301081388BE1480
:1005A0002429221B0861041A2D041AB418294C6945
:1005B000185A311841180C63ADC1BA503A33BBD345
:0805C000F2C9C40112000000A1
:04000005080002CD20
:00000001FF
